:0400000014EF00F009
:10000800FACFE2F8FBCFE3F8E9CFE4F815EF35F0E3
:10001800D8CFC9F8E8CFCAF8E0CFCBF8C3EF34F0AF
:1000280007EE56F0000EF66E000EF76E010EF86E33
:1000380010EE51F036EC00F0F86A00EE00F017EE22
:1000480056F02FEC00F00EEE7EF010EE02F02FECE2
:1000580000F0A1EF1DF0EE6AE550E150FCE1E2503E
:10006800FAE112000900F5CFEEFFE550E150FAE1A0
:10007800E250F8E112000E010E01D96746EF00F0D8
:1000880048EF00F09DEF00F05AEC42F0070107013D
:100098001A5108010801A15F070107011B51080156
:1000A8000801A25B450E08010801A15D000E0801C8
:1000B800A259D8A062EF00F064EF00F09AEF00F0C8
:1000C8000801356F110E08010801376F0801355115
:1000D80039EC3FF0370EE96E080EEA6E010EE9269C
:1000E800000EEA22EF500801366F080136A57FEFAF
:1000F80000F081EF00F08DEF00F006010601D5B3A6
:1001080088EF00F08AEF00F08BEF00F08D7292EF2D
:1001180000F00601D5930601D5978D925AEC42F06E
:10012800A1C81AF7A2C81BF70601D595000E5EEF05
:1001380001F00601D58306010601D5B1A6EF00F04E
:10014800A8EF00F0ADEF00F02EEC3CF0000E5EEFF3
:1001580001F0FCC6DBF6FDC6DCF6DBC6E0FEDCC65D
:10016800E1FE140E08010801C46F000E0801C56FF6
:100178000801210E08010801C26F0801080E0801D4
:10018800C36F6DEC38F033C8BCF834C8BDF82FEC39
:1001980043F0BCC833F8BDC834F8CE0E08010801D6
:1001A800215D0A0E08012259D8B0DDEF00F0DFEF1B
:1001B80000F011EF01F00801080121B1E6EF00F0AD
:1001C800E8EF00F011EF01F00801080126BFEFEF9A
:1001D80000F0F1EF00F011EF01F00801080125B976
:1001E800F8EF00F0FAEF00F011EF01F0EF0E080160
:1001F8000801235D050E08012459D8B006EF01F067
:1002080008EF01F011EF01F00801080125BF0FEF19
:1002180001F011EF01F012EF01F0FF0021C8FCF628
:1002280022C8FDF6060E08010801B06F000E08018D
:10023800B16F2D0E0801356F080E366F35C8AEF850
:1002480036C8AFF81DC8ACF81EC8ADF858EC3AF07F
:100258001FC8E9FF20C8EAFFFF0EEF6E080108017A
:100268003451080AD8A43BEF01F03DEF01F059EFF3
:1002780001F0080108013351D8B445EF01F047EF08
:1002880001F052EF01F0080108013351060AD8A421
:1002980050EF01F052EF01F059EF01F01FC8E9FFEC
:1002A80020C8EAFF080133C8EFFF0601D591010E07
:1002B8005EEF01F012006FEC42F0250E0801080114
:1002C8000B6F000E08010C6F0001DB0E080108011E
:1002D800096F0001000E08010A6F95EC3AF0000161
:1002E8000001DB29D8A47BEF01F07DEF01F0ADEF31
:1002F80001F00801086F000E00010001E06F08011D
:1003080008510801086F000E00010001DF6F0801A5
:1003180008510801086F000E00010001DE6F080196
:1003280008510801086F540E00010001DD6F080133
:1003380008510801086FCA0E00010001DC6F0801AE
:1003480008510801086FAC0E00010001DB6F0801BD
:100358000851060E08010801B06F000E0801B16FC0
:100368000001DB0E08010801AE6F0001000E080154
:10037800AF6F0001990E08010801AC6F0001000E73
:100388000801AD6F58EC3AF0C00E00010001806F13
:10039800A80E0001816F000E0001826F330E00016C
:1003A800836FFF0E00010001846FFF0E0001856F4F
:1003B800FF0E0001866F000E0001876F000100012B
:1003C800EC29D8B4EAEF01F0ECEF01F00AEF02F003
:1003D80000010001ED29D8B4F4EF01F0F6EF01F0C7
:1003E8000AEF02F000010001EE29D8B4FEEF01F097
:1003F80000EF02F00AEF02F000010001EF29D8A493
:1004080008EF02F00AEF02F051EF02F00001988DB8
:100418000001988FC00E000100016C6FA80E00014A
:100428006D6F000E00016E6F330E00016F6FFF0ECF
:1004380000010001706FFF0E0001716FFF0E0001D7
:10044800726F000E0001736FC00E00010001746F1F
:10045800A80E0001756F000E0001766F010E0001F5
:10046800776FC00E00010001786FA80E0001796F48
:10047800000E00017A6F010E00017B6F000E000173
:1004880000017C6F000E00017D6F000E00017E6F81
:10049800000E00017F6F7DEF02F00001989D0001C2
:1004A800989FECC06CF0EDC06DF0EEC06EF0EFC040
:1004B8006FF0F0C070F0F1C071F0F2C072F0F3C0EC
:1004C80073F0F4C074F0F5C075F0F6C076F0F7C0BC
:1004D80077F0F8C078F0F9C079F0FAC07AF0FBC08C
:1004E8007BF0FCC07CF0FDC07DF0FEC07EF0FFC05C
:1004F8007FF012003FC8E9FF40C8EAFFEECF47F897
:10050800EECF48F8EECF49F8EECF4AF800010001E7
:100518006F5108014A1911E1000100016E510801EB
:1005280049190BE1000100016D510801481905E165
:10053800000100016C5108014719D8A4A6EF02F088
:10054800A8EF02F0ABEF02F0FF0E9AEF03F00801FC
:10055800080143690201000E08010801456F020104
:10056800020E0801466F0801476F000E08010801D6
:10057800446F08014751040E080108014465C7EF9C
:1005880002F0C9EF02F0CBEF02F058EF03F0020ED1
:10059800080108013D25E96E000E080108013E2109
:1005A800EA6E0C0E080108014525E16E000E0801EF
:1005B80008014621E26EE652EE52ED50E518EFCF03
:1005C800E8FFD8B4E718D8A4ECEF02F0EEEF02F099
:1005D80044EF03F03DC8E9FF3EC8EAFF0A0E0801F0
:1005E80008014525E16E000E080108014621E26E6A
:1005F800E652EE52ED50E518EFCFE8FFD8B4E71811
:10060800D8A409EF03F00BEF03F042EF03F03FC863
:10061800E9FF40C8EAFFEECF47F8EECF48F8EECF43
:1006280049F8EECF4AF845C8E9FF46C8EAFFEECFD9
:100638004BF8EECF4CF8EECF4DF8EECF4EF8080160
:100648004A5108014E190EE10801495108014D1996
:1006580009E10801485108014C1904E10801475112
:1006680008014B19D8A43BEF03F03DEF03F042EF2C
:1006780003F00801080144519AEF03F044C843F815
:10068800170E080108014527000E08014623080136
:100698000801442B040E08010801446556EF03F0D5
:1006A80058EF03F0CBEF02F0080108014329D8B452
:1006B80060EF03F062EF03F095EF03F00801080123
:1006C8004351170D0201000EF32408010801456F7C
:1006D8000801466B0201020E080146230A0E0801B2
:1006E8000801B06F000E0801B16F3FC8AEF840C8EE
:1006F800AFF845C8ACF846C8ADF858EC3AF03DC874
:10070800E9FF3EC8EAFF0A0E080108014525E16E27
:10071800000E080108014621E26EEECFE6FFEDCF9C
:10072800E5FF0801080143519AEF03F01200C2CF18
:1007380029F8C0CF2AF8D5CF2BF8D6CF2DF8D7CFA8
:100748002CF8010EC26E08012E6F3F0EC06E080114
:100758002E5108012E6F880ED56E08012E51080102
:100768002E6F000E080108011A6F08012E51000EA5
:1007780008010801216F000E0801226F000E080110
:10078800236F000E0801246F000E080108011D6F79
:10079800000E08011E6F7BEC22F00801080174C8E6
:1007A80025F80801080175C826F808010801276B13
:1007B8000801286B000ED76E000ED66EC2820400A8
:1007C800E6EF03F0C2B2EBEF03F0EDEF03F0E6EF74
:1007D80003F0D6CF1FF8D7CF20F87BEC22F074C8EF
:1007E8001BF875C81CF8080108011F510801080109
:1007F8002127080108012051080108012223000EC1
:10080800080108012323000E0801080124231A0EF9
:100818000801215DF20E080122599E0E0801235994
:10082800000E080108012459D8A01DEF04F01FEF9D
:1008380004F03DEF04F07BEC22F00801080174514C
:1008480008010801251B0801080175510801080164
:10085800261B7BEC22F008010801745108010801ED
:10086800271B08010801755108010801281B9FEF83
:1008780004F0080108012051080108011E1906E1C9
:10088800080108011F51080108011D19D8A44FEFDC
:1008980004F051EF04F053EF04F09DEF04F0080169
:1008A8001DC82EF808011EC82FF8080108011F519D
:1008B80008012E5F08010801205108012F5B08017B
:1008C80008011B5108012E27080108011C510801C5
:1008D8002F2308012EC830F808012FC831F8080165
:1008E8000801326B0801336B54EC36F01FC81DF851
:1008F80020C81EF80801D8900801253708012637B6
:1009080008012737080128377BEC22F00801080185
:1009180074AF91EF04F093EF04F096EF04F0080140
:1009280008012581080108011A3F9DEF04F09FEF97
:1009380004F0DEEF03F029C8C2FF2AC8C0FF2CC8A4
:10094800D7FF2DC8D6FF2BC8D5FF25C816F826C84F
:1009580017F827C818F828C819F8B3EF04F01200D8
:100968000C0E08010801796F000E08017A6FF9EC86
:1009780042F04BEC44F008010801756F75C878F82F
:10098800F00E080178170801D89078330801D8903C
:100998007831EC0F08010801756F080108017567C7
:1009A800D8EF04F0DAEF04F0E3EF04F0180E0801D2
:1009B8000801726F020E0801736FC0EF05F0070E91
:1009C80008010801C46F000E0801C56F000E080178
:1009D8000801C26F000E0801C36F6DEC38F0ABEF71
:1009E80005F04BEC44F008010801746F0801080198
:1009F800746701EF05F003EF05F005EF05F0B7EFB9
:100A080005F0080108017405D8A40DEF05F00FEFF3
:100A180005F011EF05F0ABEF05F00801080174517E
:100A2800020AD8A41AEF05F01CEF05F076EF05F0DE
:100A3800030E08010801756124EF05F026EF05F0A3
:100A480028EF05F0B7EF05F0000E08010801766FF2
:100A5800000E0801776F4BEC44F008010801746F31
:100A6800080108017451040AD8A43DEF05F03FEFCE
:100A780005F049EF05F04BEC44F008010801776FE9
:100A88004BEC44F008010801766F180E08010801C4
:100A9800765D020E08017759D8B055EF05F057EF8B
:100AA80005F059EF05F0B7EF05F0B50E080108019C
:100AB800765D050E08017759D8A065EF05F067EF58
:100AC80005F070EF05F0B40E08010801726F050E0D
:100AD8000801736FC0EF05F076C872F877C873F82D
:100AE800C0EF05F0020E0801080175617EEF05F000
:100AF80080EF05F082EF05F0B7EF05F04BEC44F01E
:100B080008010801746F08010801745108010801FF
:100B1800756191EF05F093EF05F095EF05F0B7EFEC
:100B280005F00801080174C8C4F808010801C56B7C
:100B3800000E08010801C26F000E0801C36F6DECBA
:100B480038F008010801745108010801755F0801AF
:100B58000801750708017529D8A4B5EF05F0B7EFA6
:100B680005F0F5EF04F0180E08010801726F020E87
:100B78000801736FC0EF05F01200000E06010601B0
:100B8800CE6F000E0601CF6F080E08010801C46F72
:100B9800000E0801C56F0801280E08010801C26F80
:100BA8000801080E0801C36F6DEC38F028C8BCF8BE
:100BB80029C8BDF82FEC43F0BCC828F8BDC829F8EF
:100BC8002AC8BCF82BC8BDF82FEC43F0BCC82AF8DB
:100BD800BDC82BF82CC8BCF82DC8BDF82FEC43F0C5
:100BE800F80E08010801BC25080108012C6FFF0E4A
:100BF80008010801BD2108012D6F080108012F51C6
:100C08002E11D8B40AEF06F00CEF06F093EF06F0B9
:100C18001DC8E9FF1EC8EAFF0801EECF30F8080139
:100C2800EECF31F80801EECF32F80801EECF33F8F5
:100C38001FC8E9FF20C8EAFF0801EECF34F8080111
:100C4800EECF35F80801EECF36F80801EECF37F8C9
:100C580008013C6F000E08010801386F08013C517B
:100C680008013C6F110E08010801396F08013C5159
:100C780021C83AF822C83BF83AC8BCF83BC8BDF8C6
:100C88002FEC43F0BCC83AF8BDC83BF80C0E08017D
:100C98000801BC6F000E0801BD6F0801300E080185
:100CA8000801BA6F0801080E0801BB6FF2EC1EF0CC
:100CB80008010801BA1D08010801246F080108018C
:100CC800BB1D0801256F000E08010801796F000E91
:100CD80008017A6FF9EC42F021C8A0F822C8A1F8FF
:100CE8000EEC10F0A0C826F8A1C827F8080108EEF5
:100CF80026F00801EE5208012551ED18080124C814
:100D0800E8FFD8B4EF18D8B48CEF06F08EEF06F0F1
:100D180093EF06F02EEC3CF0000EC5EF06F01FC86E
:100D280041F820C842F81DC83FF81EC840F808011D
:100D3800280E080108013D6F0801080E08013E6FE2
:100D48007EEC02F008010801236F0801080123293D
:100D5800D8A4B1EF06F0B3EF06F0B8EF06F02EEC2A
:100D68003CF0000EC5EF06F023C8A3F72CC8CEF65A
:100D78002DC8CFF607010F8107010F93010EC5EFAC
:100D880006F01200C8EF06F0C5CF12F81F0E0801D2
:100D9800121712C813F80801146B000EC7B4010E1D
:100DA80008011313000E1413080114511311D8A4C9
:100DB800E0EF06F0E2EF06F0C8EF06F0C580E5EFD9
:100DC80006F0C5B0EAEF06F0ECEF06F0E5EF06F046
:100DD800A1A6F1EF06F0F3EF06F0FAEF06F008012E
:100DE8000801106908011169C6EF07F010C82FF84B
:100DF80019EC3AF00009D8B404EF07F006EF07F051
:100E080010EF07F0C584FD0E08010801106FFF0EF2
:100E18000801116FC6EF07F0C5BC15EF07F017EF13
:100E280007F0B4EF07F011C82FF819EC3AF00009F1
:100E3800D8B421EF07F023EF07F02DEF07F0C584B2
:100E4800FD0E08010801106FFF0E0801116FC6EFB3
:100E580007F0C5BC32EF07F034EF07F0A8EF07F052
:100E6800C58237EF07F0C5B23CEF07F03EEF07F059
:100E780037EF07F0A1A643EF07F045EF07F04CEF77
:100E880007F008010801106908011169C6EF07F0A9
:100E9800080108011029080108012F6F19EC3AF020
:100EA8000009D8B45AEF07F05CEF07F066EF07F0D7
:100EB800C584FD0E08010801106FFF0E0801116FAF
:100EC800C6EF07F0C5BC6BEF07F06DEF07F09CEFBE
:100ED80007F0C58670EF07F0C5B675EF07F077EF36
:100EE80007F070EF07F0C58AC5887BEF07F0C5B833
:100EF80080EF07F082EF07F07BEF07F0C58485EFFE
:100F080007F0C5B48AEF07F08CEF07F085EF07F01C
:100F1800A1A691EF07F093EF07F09AEF07F0080109
:100F28000801106908011169C6EF07F0A6EF07F07C
:100F3800C584FE0E08010801106FFF0E0801116F2D
:100F4800C6EF07F0B2EF07F0C584FE0E08010801EE
:100F5800106FFF0E0801116FC6EF07F0BEEF07F024
:100F6800C584FE0E08010801106FFF0E0801116FFD
:100F7800C6EF07F00801C9CF10F808010801116B86
:100F8800C6EF07F01200A0C8E9FFA1C8EAFF0801F0
:100F9800EECFBCF80801EDCFBDF82FEC43F0A0C8A8
:100FA800E9FFA1C8EAFF0801BCC8EEFF0801BDC8F7
:100FB800EDFF020E08010801A025E96E000E0801E8
:100FC8000801A121EA6E0801EECFBCF80801EDCFB7
:100FD800BDF82FEC43F0020E08010801A025E96EC8
:100FE800000E08010801A121EA6E0801BCC8EEFF45
:100FF8000801BDC8EDFF040E08010801A025E96E2F
:10100800000E08010801A121EA6E0801EECFA2F83E
:101018000801EECFA3F80801EECFA4F80801EECF3F
:10102800A5F82BEC3EF0040E08010801A025E96E96
:10103800000E08010801A121EA6E0801A2C8EEFF0E
:101048000801A3C8EEFF0801A4C8EEFF0801A5C85F
:10105800EDFFED52ED52080E08010801A025E96EDA
:10106800000E08010801A121EA6E0801EECFA2F8DE
:101078000801EECFA3F80801EECFA4F80801EECFDF
:10108800A5F82BEC3EF0080E08010801A025E96E32
:10109800000E08010801A121EA6E0801A2C8EEFFAE
:1010A8000801A3C8EEFF0801A4C8EEFF0801A5C8FF
:1010B800EDFFED52ED520E0E08010801A025E96E74
:1010C800000E08010801A121EA6E0801EECFBCF864
:1010D8000801EDCFBDF82FEC43F00E0E0801080112
:1010E800A025E96E000E08010801A121EA6E080199
:1010F800BCC8EEFF0801BDC8EDFF100E08010801CD
:10110800A025E96E000E08010801A121EA6E080178
:10111800EECFBCF80801EDCFBDF82FEC43F0100E70
:1011280008010801A025E96E000E08010801A121A7
:10113800EA6E0801BCC8EEFF0801BDC8EDFF120E3B
:1011480008010801A025E96E000E08010801A12187
:10115800EA6E0801EECFBCF80801EDCFBDF82FEC20
:1011680043F0120E08010801A025E96E000E0801DF
:101178000801A121EA6E0801BCC8EEFF0801BDC83C
:10118800EDFF12001DC8E9FF1EC8EAFF0801EECFF7
:1011980028F80801EECF29F80801EECF2AF808014F
:1011A800EECF2BF81FC8E9FF20C8EAFF0801EECFF1
:1011B8002CF80801EECF2DF80801EECF2EF8080123
:1011C800EECF2FF80801486F000E08010801306FB4
:1011D800080148510801486F060E08010801316FDF
:1011E8000801485121C832F822C833F832C8BCF87F
:1011F80033C8BDF82FEC43F0BCC832F8BDC833F88B
:101208000C0E08010801BC6F000E0801BD6F080133
:10121800280E08010801BA6F0801080E0801BB6F03
:10122800F2EC1EF008010801BA1D08010801246F3C
:1012380008010801BB1D0801256F21C8A0F822C8B4
:10124800A1F80EEC10F0A0C826F8A1C827F80801EC
:101258000801275108010801251906E108010801BC
:101268002651080108012419D8B43DEF09F03FEFD1
:1012780009F043EF09F02EEC3CF0BBEF09F0000E4B
:1012880008010801796F000E08017A6FF9EC42F045
:10129800140E08010801C46F000E0801C56F08018B
:1012A800340E08010801C26F0801080E0801C36F57
:1012B8006DEC38F00801340E08010801A06F080130
:1012C800080E0801A16FC7EC07F0080140390F0BA1
:1012D8000801486F0801D89048370801D890483568
:1012E800EC0F08010801236F0801080123510801C8
:1012F8000801215D0801486F000E08010801225904
:101308000801496FEC0E0801482508010801216F02
:10131800FF0E080149210801226F1DC84CF81EC89C
:101328004DF80801340E080108014A6F0801080E3B
:1013380008014B6F91ECB2F00009D8B4A6EF09F0A0
:10134800A8EF09F0B7EF09F021C84CF822C84DF80A
:101358000801340E080108014A6F0801080E080147
:101368004B6F29EC80F02EEC3CF0BBEF09F012003B
:10137800070107019D29D8A4C4EF09F0C6EF09F0B9
:10138800EEEF09F0000E08010801536F000E080186
:10139800546F450E08010801516F000E0801526F85
:1013A8000801166F000E08010801506F0801165158
:1013B800000E080108014C6F000E08014D6F000E69
:1013C80008014E6F000E08014F6F22ECD7F007019D
:1013D80007019D6F070107019D29D8A4F6EF09F0C1
:1013E800F8EF09F0FAEF09F0B0EF0AF09DC74CF8F2
:1013F800D9EC39F008014D514C11D8A406EF0AF088
:1014080008EF0AF00AEF0AF0B0EF0AF00001000155
:101418006C510001000170150801166F00010001F0
:101428006D510001000171150801176F00010001DD
:101438006E510001000172150801186F00010001CA
:101448006F510001000173150801196F05010501AD
:10145800DA5100010001701508011A6F0501050134
:10146800DB5100010001711508011B6F0501050121
:10147800DC5100010001721508011C6F050105010E
:10148800DD5100010001731508011D6F0801195194
:1014980008011D190EE10801185108011C1909E17C
:1014A8000801175108011B1904E108011651080128
:1014B8001A19D8B462EF0AF064EF0AF068EF0AF07C
:1014C8008FEC41F0B0EF0AF0060E08010801B06F8A
:1014D800000E0801B16F990E0801166F000E176F04
:1014E80016C8AEF817C8AFF80801080E08010801B9
:1014F800AC6F0801080E0801AD6F58EC3AF06CC0EB
:101508000EF86DC00FF86EC010F86FC011F80A0E13
:1015180008010801BC6F000E0801BD6F0801080E24
:1015280008010801BA6F0801080E0801BB6FF2EC48
:101538001EF0BAC812F8BBC813F8D0920801080EFA
:1015480008010801146F0801080E0801156F15C875
:10155800F4FF14C8F3FFFF00120096EF0BF01C0E07
:1015680008010801C46F000E0801C56F08011D0EAF
:1015780008010801C26F0801080E0801C36F6DEC6D
:1015880038F02EEC3CF008011D0E080108017C6FB4
:101598000801080E08017D6F9EEC30F00801080173
:1015A8001D051E11D8A4DBEF0AF0DDEF0AF0F3EFFA
:1015B8000AF0080108012151060AD8A4E6EF0AF04A
:1015C800E8EF0AF0F3EF0AF0080108012251040AD3
:1015D800D8B4F1EF0AF0F3EF0AF0F5EF0AF0A2EF52
:1015E8000BF0080108012351020A2411D8A4FFEFC7
:1015F8000AF001EF0BF015EF0BF008EE25F014EEF2
:10160800DDF0060EEECFE6FFE82E06EF0BF02BC856
:10161800D9F42CC8DAF42DC8DBF42EC8DCF4A2EF18
:101628000BF00801080123052411D8A41EEF0BF0C4
:1016380020EF0BF05EEF0BF0000100016F51080185
:101648000801381914E1000100016E510801080170
:1016580037190DE1000100016D5108010801361923
:1016680006E1000100016C51080108013519D8B4E0
:1016780040EF0BF042EF0BF044EF0BF0A2EF0BF052
:101688002BC859F62CC85AF62DC85BF62EC85CF63E
:1016980008EE25F016EE5DF0060EEECFE6FFE82E1A
:1016A80051EF0BF00801396F010E07010701366F82
:1016B80008013951020E08010801236F000E0801C4
:1016C800246F06EE5DF018EE2FF0060EEECFE6FF63
:1016D800E82E6AEF0BF059C635F85AC636F85BC6DD
:1016E80037F85CC638F808011D0E08010801786F44
:1016F8000801080E0801796F98EC1BF00009D8A4BE
:1017080088EF0BF08AEF0BF08CEF0BF0A2EF0BF0E9
:101718000801396F000E07010701366F08013951BA
:10172800A0EF0BF0070107013651000A01E117D7B6
:10173800010AC0E0A0EF0BF0A2EF0BF01200FDECE5
:1017480040F00009D8A4ABEF0BF0ADEF0BF0AFEF12
:101758000BF089EF0CF07B0E08010801566FFF0EA5
:101768000801576F4CEC27F00009D8A4BEEF0BF026
:10177800C0EF0BF0C2EF0BF089EF0CF0C9EC26F0CC
:1017880065C832F866C833F867C834F868C835F8E9
:1017980008013229D8B43329D8B43429D8B4352922
:1017A800D8A4D9EF0BF0DBEF0BF0EBEF0BF0000157
:1017B800988D0001988F0801366F000E0801080106
:1017C800376F08013651ABEC42F089EF0CF0600E30
:1017D80008010801566FFF0E0801576F4CEC27F0FF
:1017E8000009D8A4FAEF0BF0FCEF0BF0FEEF0BF0BA
:1017F80089EF0CF0C9EC26F065C82EF866C82FF8FA
:1018080067C830F868C831F8500E08010801566FEB
:10181800FF0E0801576F4CEC27F00009D8A417EF0A
:101828000CF019EF0CF01BEF0CF089EF0CF0C9EC81
:1018380026F065C82AF866C82BF867C82CF868C867
:101848002DF8C50E08010801566FFF0E0801576FE5
:101858004CEC27F00009D8A434EF0CF036EF0CF06C
:1018680038EF0CF089EF0CF0C9EC26F065C822F8C7
:1018780066C823F867C824F868C825F8D40E080194
:101888000801566FFF0E0801576F4CEC27F000094E
:10189800D8A451EF0CF053EF0CF055EF0CF089EF92
:1018A8000CF0C9EC26F065C826F866C827F867C8A2
:1018B80028F868C829F80001989D32C86CF033C828
:1018C8006DF034C86EF035C86FF02EC870F02FC8B0
:1018D80071F030C872F031C873F02AC874F02BC8A0
:1018E80075F02CC876F02DC877F022C878F023C898
:1018F80079F024C87AF025C87BF026C87CF027C880
:101908007DF028C87EF029C87FF012000701070182
:101918007D51D8B492EF0CF094EF0CF0C1EF0CF0BD
:10192800070107017C51070107017A277E0E07018D
:1019380007017A65A2EF0CF0A4EF0CF0A9EF0CF008
:10194800070107017C69BDEF0CF0070107017A6701
:10195800B0EF0CF0B2EF0CF0BDEF0CF00801DA6F4D
:10196800010E070107017C6F0801DA510701070121
:101978007D077AC7BBFF23EF0DF0070107017E51F2
:10198800020AD8A4CAEF0CF0CCEF0CF0D0EF0CF0A0
:101998007BC7BBFF23EF0DF0070107017E05D8A425
:1019A800D8EF0CF0DAEF0CF021EF0DF0D1EC43F0AA
:1019B800070107017F5108010801DE5D0801DA6FA0
:1019C80007010701805108010801DF590801DB6F91
:1019D80007010701815108010801E0590801DC6F7E
:1019E80007010701825108010801E1590801DD6F6B
:1019F800F30EDA5D9E0EDB59000EDC59000E08016D
:101A0800DD59D8A00AEF0DF00CEF0DF01FEF0DF027
:101A1800070107017B51FF0A070107017B6F7BC79D
:101A2800BBFFD1EC43F0DEC87FF7DFC880F7E0C822
:101A380081F7E1C882F723EF0DF0000EBB6E0701B6
:101A480007018651D8B42BEF0DF02DEF0DF05AEFAA
:101A58000DF00701070185510701070183277E0E55
:101A68000701070183653BEF0DF03DEF0DF042EFF5
:101A78000DF007010701856956EF0DF00701070111
:101A8800836749EF0DF04BEF0DF056EF0DF00801AD
:101A9800DA6F010E07010701856F0801DA510701A6
:101AA8000701860783C7BEFF6BEF0DF0070107012B
:101AB8008751020AD8A463EF0DF065EF0DF069EFC6
:101AC8000DF084C7BEFF6BEF0DF0000EBE6E120066
:101AD80008010F6F000E080108010E6F08010F5171
:101AE8003DEF0EF0080108010D513A0AD8A47FEF26
:101AF8000DF081EF0DF0A0EF0DF007010701015186
:101B08000011D8A48AEF0DF08CEF0DF096EF0DF0D0
:101B180008010F6F020E070107012F6F08010F510F
:101B28009EEF0DF008010F6F010E070107012F6FDF
:101B380008010F514CEF0EF007010701003B0701A8
:101B4800013BF00E07010117070100510F0B0701B8
:101B58000113F00E070100170DC872F82DEC2DF0D7
:101B680008010F6F08010F510701070100134CEF1F
:101B78000EF0C2EF0DF0080108010E2B0101C80E8E
:101B8800080108010E25E96EEA6A0101010EEA2240
:101B9800EF50D8A4D2EF0DF0D4EF0DF0BFEF0DF059
:101BA8000101C80E080108010E25E96EEA6A010163
:101BB800010EEA2208010DC8EFFF0701070100071F
:101BC800D8A001070701070101510011D8A4EFEFC0
:101BD8000DF0F1EF0DF09EEF0DF0070107012F2B2F
:101BE8004CEF0EF0080108010D51690AD8B4FFEF57
:101BF8000DF001EF0EF006EF0EF0070107012F6957
:101C08009EEF0DF0070107012F2B4CEF0EF0080196
:101C180008010D51730AD8A414EF0EF016EF0EF058
:101C280020EF0EF008010F6F000E070107012F6F5C
:101C380008010F514CEF0EF007010701273B070180
:101C4800283BF00E07012817070127510F0B070142
:101C58002813F00E070127170DC872F82DEC2DF088
:101C680008010F6F08010F510701070127134CEFF7
:101C78000EF0070107012F51000A01E133D7010ACD
:101C880001E177D7030AAEE0010AC1E04CEF0EF09C
:101C98001200A1C768F8BEEC20F068C854F869C8FB
:101CA80055F80101000E08010801596F0101010EE4
:101CB80008015A6F3DEC37F01A0E08010801592740
:101CC800000E08015A230801080159510801545D02
:101CD800080108015A5108015559D8B076EF0EF09D
:101CE80078EF0EF07CEF0EF065EC3FF02DEF0FF083
:101CF80022EC2FF0E20E08010801576FFF0E0801D1
:101D0800586FA1C756F830EC42F00801546F000E26
:101D180008010801536F08015451130E0801080106
:101D2800536599EF0EF09BEF0EF09DEF0EF0D8EF94
:101D38000EF00401E30E080108015325E96EEA6A72
:101D48000401040EEA22EF5008010801586F0DEC57
:101D58003FF008010801576FA1C756F801EC15F0CC
:101D68000401E30E080108015325E96EEA6A04013B
:101D7800040EEA22EF5008010801646FE1EC3EF01E
:101D880008010801576FA1C756F801EC15F00801C2
:101D98000801532B130E080108015365D6EF0EF006
:101DA800D8EF0EF09DEF0EF00101000E08010801BA
:101DB800596F0101010E08015A6F3DEC37F0080117
:101DC8000801595108010801586F0DEC3FF008014E
:101DD8000801576FA1C756F801EC15F00101000E74
:101DE80008010801596F0101010E08015A6F3DEC05
:101DF80037F008010801595108010801646FE1EC46
:101E08003EF008010801576FA1C756F801EC15F01C
:101E18000801546F3A0E08010801576F0801545120
:101E2800A1C756F801EC15F00101000E08010801E0
:101E3800576F0101010E0801586FA1C756F845EC0C
:101E480042F0A1C768F8F6EC3BF065EC3FF016EC01
:101E580044F01200FC0E92160E01FE8B96928D92A3
:101E680036EF0FF00E010E01FDA13DEF0FF03FEF31
:101E78000FF036EF0FF00801096F000E060106019A
:101E8800D56F080109510601D581000E060106012A
:101E9800FC6F000E0601FD6F000E0E010E01E86FCB
:101EA800000E0E01E96FCD0E0E010E01EC6F0A0E49
:101EB8000E010E01ED6FCD0E0E010E01EA6F0A0E36
:101EC8000E01EB6FCE0E0E010E01E46F0A0E0E012D
:101ED800E56FCE0E0E010E01E26F0A0E0E01E36FE2
:101EE8000801096F000E08010801C06F08010951B7
:101EF80064EC44F00801096F0D0E0E010E01A06F8D
:101F08000801095100F00801096F320E0E010E0197
:101F1800A26F0801095100F00801096F120E0E01A5
:101F28000E01A46F0801095100F00801096F400E65
:101F38000E010E01A36F0801095100F00801096F95
:101F4800120E0E010E01A66F0801095100F00801DA
:101F5800096F0C0E0E010E01A76F0801095100F060
:101F68000801096FEE0E0E010E01AA6F0801095152
:101F780000F00801096F050E0E010E01AB6F080194
:101F8800095100F099C084FE00F09AC085FE00F067
:101F98009BC082FE00F09CC083FE00F09DC080FEC6
:101FA80000F09EC081FE00F0100E080108010B6FC2
:101FB800010E08010C6F0801096F100E08010801D5
:101FC8000A6F0801095199EC40F0720E08010801E6
:101FD8000B6F340E08010C6F0801096F140E08010D
:101FE80008010A6F0801095199EC40F0000E080138
:101FF80008010B6F000E08010C6F0801096F000E35
:10200800080108010A6F0801095199EC40F00E0116
:10201800DF851200F1C6A8F8F2C6A9F8F3C6AAF837
:10202800F4C6ABF8E0CEA2F8E1CEA3F8A9EF10F021
:10203800A0C8A6F8A1C8A7F8150E08010801A05D58
:10204800000E0801A159D8A02CEF10F02EEF10F0C7
:1020580035EF10F0140E08010801A66F000E0801F4
:10206800A76FA6C8C4F8A7C8C5F80801AC0E080130
:102078000801C26F0801080E0801C36F6DEC38F043
:1020880008010801A65108010801A05F080108011C
:10209800A75108010801A15B08010801A6A157EF93
:1020A80010F059EF10F069EF10F00801AC0E0801BC
:1020B8000801A625E96EEA6A0801080EEA22000E60
:1020C800EF6E08010801A64BA72B0801AC0E08010A
:1020D8000801A46F0801080E0801A56F9EEF10F013
:1020E8000801A4C8E9FF0801A5C8EAFF0801020E13
:1020F8000801A427000E0801A523EECFC0F8EDCFF4
:10210800C1F80801C05108010801A8270801C151F8
:1021180008010801A923000E08010801AA23000EDE
:1021280008010801AB23020E08010801A65F000E92
:102138000801A75B08010801A751A611D8A4A7EFB9
:1021480010F0A9EF10F074EF10F008010801A15188
:10215800A011D8A4B2EF10F0B4EF10F01CEF10F0FB
:10216800A2C8E0FEA3C8E1FE08010801A8510801C1
:102178000801AA2508010801A86F08010801A9514A
:1021880008010801AB210801A96F0801AA6BD8B0A2
:10219800AA2B0801AB6B080108EEAAF0EE50080163
:1021A8000801A827ED5008010801A9230801080122
:1021B800A81D08010801A06F08010801A91D080150
:1021C800A16FE7EF10F01200140E0801080158255E
:1021D800E96E000E080108015921EA6EEF50080166
:1021E800606F3F0E08016017180E0801602708018C
:1021F80060510801080158250801616FE86A080163
:1022080060BFE8680801080159210801626F61C8C8
:102218005EF862C85FF8140E080108015825E96ED7
:10222800000E080108015921EA6E080108015C51F5
:10223800EE2608015D51EE22000EEE22ED22ED524F
:10224800ED52B5EF11F008015AC8F6FF08015BC856
:10225800F7FF000EF86E5EC8E9FF5FC8EAFF0800E6
:10226800F5CFEFFF080108015A4B5B2B0801080165
:102278005E4B5F2B580E0801080158250801606F56
:10228800000E0801080159210801616F0801615118
:10229800080108015F1905E10801605108010801FA
:1022A8005E19D8A45AEF11F05CEF11F0B0EF11F0FD
:1022B800100E08010801582508010801836F000E57
:1022C8000801080159210801846F0C0E0801080152
:1022D800582508010801816F000E080108015921DD
:1022E8000801826F080E0801080158250801080135
:1022F8007F6F000E0801080159210801806F040E44
:10230800080108015825080108017D6F000E080121
:102318000801592108017E6F58C87BF859C87CF814
:10232800180E08010801582508010801796F000EE8
:1023380008010801592108017A6F80EC9BF0180EFA
:10234800080108015825080108015E6F000E080100
:102358000801592108015F6F080108015C07D8A02E
:102368005D07080108015D515C11D8A4BEEF11F0AA
:10237800C0EF11F027EF11F01200140E0801080148
:102388005825E96E000E080108015921EA6EEF5040
:102398000801606F3F0E08016017180E08016027DA
:1023A800080160510801080158250801616FE86AB1
:1023B800080160BFE8680801080159210801626F37
:1023C80061C85EF862C85FF8140E08010801582554
:1023D800E96E000E080108015921EA6E080108019A
:1023E8005C51EE2608015D51EE22000EEE22ED2230
:1023F800ED52ED5289EF12F05AC8E9FF5BC8EAFFC7
:102408005EC8E1FF5FC8E2FFEFCFE7FF0801080100
:102418005A4B5B2B080108015E4B5F2B580E0801D5
:10242800080158250801606F000E080108015921AC
:102438000801616F08016151080108015F1905E190
:1024480008016051080108015E19D8A42EEF12F0A6
:1024580030EF12F084EF12F0100E08010801582531
:1024680008010801836F000E0801080159210801BD
:10247800846F0C0E08010801582508010801816FB6
:10248800000E0801080159210801826F080E080191
:1024980008015825080108017F6F000E080108018E
:1024A80059210801806F040E080108015825080108
:1024B80008017D6F000E08010801592108017E6F8F
:1024C80058C87BF859C87CF8180E08010801582527
:1024D80008010801796F000E080108015921080157
:1024E8007A6F80EC9BF0180E080108015825080146
:1024F80008015E6F000E08010801592108015F6F8D
:10250800080108015C07D8A05D07080108015D51B2
:102518005C11D8A492EF12F094EF12F000EF12F0D1
:102528001200000E080108012D659DEF12F09FEFC3
:1025380012F0A1EF12F065EF13F02DC871F81DEC41
:102548002BF00BC00DF00CC00EF043EF13F0DCECD9
:1025580040F06CEC33F065EF13F06CEC33F065EFA2
:1025680013F008012E6F010E08010801736F0801AE
:102578002E5108012F6F110E08010801726F080112
:102588002F519FECA1F030502F10D8A4CEEF12F0AD
:10259800D0EF12F0D2EF12F0E5EF12F000EE29F0D2
:1025A80010EE07F0E652EE52ED50E518EFCFE8FFD7
:1025B800D8B4E718D8A4E3EF12F0E5EF12F0B5EFBE
:1025C80012F008012E6F080E176E08012E5165EFE4
:1025D80013F008012E6F010E08010801736F08013E
:1025E8002E5108012F6F110E08010801726F0801A2
:1025F8002F519FECA1F030502F10D8A406EF13F004
:1026080008EF13F00AEF13F01DEF13F000EE29F0B6
:1026180010EE07F0E652EE52ED50E518EFCFE8FF66
:10262800D8B4E718D8A41BEF13F01DEF13F0EDEFA3
:1026380012F008012E6F0C0E176E08012E5165EF6F
:1026480013F008012E6F0D0E176E08012E5165EF5D
:1026580013F008012E6F000E08010801736F0801BE
:102668002E5108012F6F140E08010801726F08011E
:102678002F519FECA1F06CEC33F065EF13F017507D
:10268800000A01E16AD7010A01E161D7030A01E101
:1026980064D7010A01E161D7060A01E15ED7030A9E
:1026A80001E15FD7010A01E15CD70F0AD2E0010A14
:1026B800D0E0020A8EE0070ACCE0020AC2E02DEF61
:1026C80013F012000801606F690E08010801646FB9
:1026D800080160518FEC3FF0080156515311541115
:1026E8005511D8A47AEF13F07CEF13F088EF13F0AC
:1026F8000801606F300E08010801646F080160511D
:102708008FEC3FF02CEF14F00801606F000E080109
:102718000801576F08016051070E08010801576545
:1027280098EF13F09AEF13F09CEF13F0C9EF13F042
:102738000801580E080108015725E96EEA6A0801E0
:10274800080EEA2253C864F8E1EC3EF0EF6E040E7E
:102758000801606FD8900801080156330801553305
:1027680008015433080153330801602FAEEF13F00A
:1027780008010801572B070E080108015765C7EF24
:1027880013F0C9EF13F09CEF13F00801606F080E07
:1027980008010801576F08016051080108015767CF
:1027A800D8EF13F0DAEF13F0DCEF13F001EF14F0C9
:1027B80057C860F8FF0E080160270801580E080185
:1027C8006025E96EEA6A0801080EEA22EF50300A2D
:1027D800D8B4F1EF13F0F3EF13F0F5EF13F001EFC6
:1027E80014F0080108015707080108015767FFEFAF
:1027F80013F001EF14F0DCEF13F00801080157673C
:1028080008EF14F00AEF14F00CEF14F02CEF14F0AA
:1028180057C860F8FF0E080160270801580E080124
:102828006025E96EEA6A0801080EEA22EF500801FD
:102838000801646F8FEC3FF0080108015707080191
:10284800080157672AEF14F02CEF14F00CEF14F07E
:102858000801606F730E08010801646F0801605178
:102868008FEC3FF01200140E08010801C46F000E2F
:102878000801C56F0801270E08010801C26F080189
:10288800080E0801C36F6DEC38F0080108012751E4
:10289800F00B400AD8B453EF14F055EF14F058EF8A
:1028A80014F0000E00EF15F01F0E080108012D1599
:1028B80008013B6FFF0E080108012E1508013C6F47
:1028C80008013C513B11D8B46CEF14F06EEF14F0D2
:1028D80071EF14F0000E00EF15F027C83BF80F0E4B
:1028E80008013B170801D8903B370801D8903B35C1
:1028F80006010601FA6F06010801FAC63FF8080149
:102908000801406B000E080108013D6F000E080128
:102918003E6FF0EC36F03DC825F83EC826F80601B3
:102928000801FAC67BF8080108017C6B64EC3CF0EE
:102938000801080126512511D8B4A5EF14F0A7EF16
:1029480014F0AAEF14F0000E00EF15F00801270E9E
:1029580008010801BA6F0801080E0801BB6F5FEC97
:102968002CF0080108011E511D11D8B4BEEF14F057
:10297800C0EF14F0D0EF14F01DC8E9FF1EC8EAFF3D
:10298800080137C8EEFF080138C8EEFF080139C84A
:10299800EEFF08013AC8EEFF1FC8E9FF20C8EAFFAA
:1029A800080133C8EEFF080134C8EEFF080135C836
:1029B800EEFF080136C8EEFF21C8E9FF22C8EAFF8A
:1029C800080130C8EFFF06010601FA5108010801A5
:1029D800295D08013B6F000E080108012A5908010A
:1029E8003C6F23C8E9FF24C8EAFF3BC8EEFF3CC898
:1029F800EDFF010E00EF15F01200000E08010801AE
:102A0800566509EF15F00BEF15F00DEF15F0C7EF50
:102A180015F056C871F81DEC2BF056C868F8BEECD6
:102A280020F068C858F869C859F8080108015951D0
:102A38005811D8A422EF15F024EF15F026EF15F061
:102A4800C7EF15F00801080158055911D8A42FEF50
:102A580015F031EF15F035EF15F056C868F8F6ECBB
:102A68003BF019B03AEF15F03CEF15F067EF15F0B1
:102A780000EE03F0EECF5AF8EDCF5BF801500801F5
:102A88005A5F025008015B5BD89008015B3108016E
:102A98005D6F08015A3108015C6F0801080158513F
:102AA80008015C5D08010801595108015D59D8A069
:102AB80060EF15F062EF15F067EF15F056C868F88B
:102AC800F6EC3BF01980010E08010801AA6F000E10
:102AD8000801AB6F08015A6F010E08010801A96FC0
:102AE80008015A510801570E08010801A76F08018B
:102AF800080E0801A86F1CC0A6F807C0A4F808C0F3
:102B0800A5F8A0EC23F000EE03F010EE07F0E62A9B
:102B1800000EE522E652EE52ED50E55C02E1EF5080
:102B2800E75CD8A09AEF15F09CEF15F0A0EF15F030
:102B380001C007F002C008F0080108015805591142
:102B4800D8A4A9EF15F0ABEF15F0B1EF15F056C802
:102B580068F8F6EC3BF0C5EF15F018BAB6EF15F0CB
:102B6800B8EF15F0C5EF15F0188A5AEC42F0060ECA
:102B780008010801A125136E000E08010801A22111
:102B8800146EC7EF15F0120006EE95F018EE0DF072
:102B9800140EEECFE6FFE82ECDEF15F00801216FF9
:102BA800140E08010801676F0801215108010D0E74
:102BB80008010801656F0801080E0801666F0EEC30
:102BC80018F00009D8A4EBEF15F0EDEF15F0EFEFD2
:102BD80015F08CEF16F0000E08010801676FFF0E64
:102BE8000801686F08010D0E08010801656F0801EA
:102BF800080E0801666F49EC29F008016651651155
:102C0800D8A409EF16F00BEF16F00FEF16F070ECE2
:102C180034F08CEF16F0B60E08010801676FFF0E4E
:102C28000801686F08010D0E08010801656F0801A9
:102C3800080E0801666F49EC29F008016651651114
:102C4800D8A429EF16F02BEF16F02FEF16F0CCECE6
:102C5800D3F08CEF16F09F0E08010801676FFF0E86
:102C68000801686F08010D0E08010801656F080169
:102C7800080E0801666F49EC29F0080166516511D4
:102C8800D8A449EF16F04BEF16F04FEF16F0A3EC6F
:102C98000BF08CEF16F0770E08010801676FFF0E36
:102CA8000801686F08010D0E08010801656F080129
:102CB800080E0801666F49EC29F008016651651194
:102CC800D8A469EF16F06BEF16F06FEF16F0C5ECAD
:102CD80029F08CEF16F00C0E08010801676FFF0E43
:102CE8000801686F08010D0E08010801656F0801E9
:102CF800080E0801666F49EC29F008016651651154
:102D0800D8A489EF16F08BEF16F08CEF16F0FF00C1
:102D18001200040E08010801C46F000E0801C56FF7
:102D28000801210E08010801C26F0801080E0801F8
:102D3800C36F6DEC38F0080108012151080A22110F
:102D4800D8A4A9EF16F0ABEF16F04DEF17F01FC897
:102D58003FF820C840F8140E080108013D6F000E26
:102D680008013E6FF0EC36F008013E513D11D8B431
:102D7800C0EF16F0C2EF16F0C4EF16F04DEF17F0E3
:102D88000801256F000E08010801216F080125516F
:102D9800080E080108012327080E0801080123610D
:102DA800D8EF16F0DAEF16F0E9EF16F0080108018F
:102DB800242B080108012467E4EF16F0E6EF16F06B
:102DC800E9EF16F008010801232BEBEF16F0CBEC26
:102DD8003DF00009D8B4F3EF16F0F5EF16F0EBEF7D
:102DE80016F0DD0E08010801AC6F0A0E0801AD6F80
:102DF8000BEC44F01FC8A3F820C8A4F80801256FFD
:102E0800010E08010801A26F080125511DC8A0F88C
:102E18001EC8A1F8CAEC18F0040E08010801C26F18
:102E2800000E0801C36F0801210E08010801C06FD8
:102E38000801080E0801C16FBBEC40F0FC0E080148
:102E480008011F2508010801B06FFF0E08010801DD
:102E580020210801B16FFF0E08010801AE6FFF0EB7
:102E68000801AF6FFF0E08010801AC6FFF0E0801E3
:102E7800AD6F3CECDDF041EF17F08EEC43F000094C
:102E8800D8B449EF17F04BEF17F041EF17F003EC08
:102E980039F0120027C838F828C839F867EC35F037
:102EA80008012D6F690E08010801646F08012D5192
:102EB8008FEC3FF0080108012A512911D8A467EFC7
:102EC80017F069EF17F075EF17F008012D6F300E46
:102ED80008010801646F08012D518FEC3FF003EFE2
:102EE80018F008012D6F000E080108012C6F080169
:102EF8002D51080108012B51080108012C5DD8A0AB
:102F080088EF17F08AEF17F08CEF17F0B4EF17F08F
:102F1800080108012C51080108012925E96E08015A
:102F2800000E080108012A21EA6EEF50300AD8B4D1
:102F3800A0EF17F0A2EF17F0A4EF17F0B4EF17F017
:102F4800080108012C2B080108012B510801080170
:102F58002C5DD8A0B2EF17F0B4EF17F08CEF17F094
:102F6800080108012B51080108012C5DD8A0BFEF0A
:102F780017F0C1EF17F0C3EF17F003EF18F00801CF
:102F880008012C51080108012925E96E0801000EE5
:102F9800080108012A21EA6EEF5008010801586F5C
:102FA8000DEC3FF008010801646F8FEC3FF0080159
:102FB80008012C51080108012925E96E0801000EB5
:102FC800080108012A21EA6EEF5008010801646F20
:102FD800E1EC3EF008010801646F8FEC3FF0080156
:102FE80008012C2B080108012B51080108012C5D50
:102FF800D8A001EF18F003EF18F0C3EF17F008019D
:103008002D6F730E08010801646F08012D518FECB4
:103018003FF0120008016B6F000E08010801696F8C
:1030280008016B5108016B6F000E080108016A6FF7
:1030380008016B5149EF18F00101000E0401040169
:10304800FF25E96EEA6A0101010EEA22EF50080144
:103058000801686F04010401FF2B08010801685189
:103068003A0AD8A43AEF18F03CEF18F03EEF18F0FF
:1030780053EF18F008016A3BF00E6A1768C872F837
:103088002DEC2DF0080108016A13C70E0401040194
:10309800FF6551EF18F053EF18F020EF18F0080112
:1030A8006AC86BF808016C6BFF0E080108016725F8
:1030B80008016D6F08016E6BFF0E08016E23080191
:1030C8006E51800A08016F6F08016B5108016D5D30
:1030D80008016C51800A08016F59D8B076EF18F0D2
:1030E80078EF18F081EF18F0080108016A5104011F
:1030F8000401FF27000EC9EF18F008016B6F000EDE
:1031080008010801696F08016B51AAEF18F0010165
:10311800000E04010401FF25E96EEA6A0101010EAF
:10312800EA22080108016951080108016525E16ED4
:103138000801000E080108016621E26EEFCFE7FFE3
:1031480004010401FF2B08010801692B080108018B
:103158006A5108010801695DD8A0B5EF18F0B7EF0A
:1031680018F08BEF18F0080108016A5108010801EE
:103178006525E96E0801000E080108016621EA6E5E
:10318800000EEF6E010EC9EF18F012000801B96FBA
:10319800140E06010601FA6F0801B9510801B96F4A
:1031A800450E08010801A56F0801B9510801B96F5A
:1031B800000E08010801A66F0801B951140E080194
:1031C8000801A32508010801A76F000E08010801DE
:1031D800A4210801A86F07010701204B212B20C754
:1031E800A9F821C7AAF8000E08010801AB6F000E64
:1031F8000801AC6F0801B96F640E08010801AD6FD2
:103208000801B951A2C8AEF8000E08010801AF6F55
:10321800000E0801B06F6CC0B1F86DC0B2F86EC096
:10322800B3F86FC0B4F8A0C8E9FFA1C8EAFF080165
:10323800EECFB5F80801EECFB6F80801EECFB7F833
:103248000801EECFB8F80801A50E08010801BA6F09
:103258000801080E0801BB6F5FEC2CF0140E080182
:103268000801BC6F000E0801BD6F0801A50E08011A
:103278000801BA6F0801080E0801BB6FF2EC1EF0D6
:10328800BAC8AFF8BBC8B0F8140E08010801A325E6
:1032980008010801BD6F000E08010801A4210801FA
:1032A800BE6F0801B96F000E08010801BC6F080164
:1032B800B951040E08010801A02508010801BA6FD8
:1032C800000E08010801A1210801BB6FC4EC33F00E
:1032D800140E08010801C26F000E0801C36F08012F
:1032E800A50E08010801C06F0801080E0801C16F8A
:1032F800BBEC40F080EF19F012004CC850F84DC8F4
:1033080051F8080150C8F6FF080151C8F7FF000E30
:10331800F86E08000801F5CF4FF808010801504B76
:10332800512B080108014F51D8B49DEF19F09FEFB8
:1033380019F0CBEF19F0080108014F512E0AD8B443
:10334800A8EF19F0AAEF19F0CBEF19F0080108015E
:103358004F512F0AD8B4B3EF19F0B5EF19F0CBEFEE
:1033680019F0080108014F512C0AD8B4BEEF19F022
:10337800C0EF19F0CBEF19F0080108014F513E0AD0
:10338800D8A4C9EF19F0CBEF19F085EF19F00801AF
:1033980008014C5108010801505D0801526F0801ED
:1033A8005205080108014E6F4EC853F867EC3DF00E
:1033B800080108014EC855F808010801566B4CC8A9
:1033C80053F84DC854F853EC31F0010E08010801C8
:1033D8005327000E0801542308010801535108011E
:1033E80008014C27080108015451080108014D2320
:1033F800080108014F51D8B404EF1AF006EF1AF08B
:1034080027EF1AF0080108014F512F0AD8B40FEF1F
:103418001AF011EF1AF027EF1AF0080108014F51BE
:103428002C0AD8B41AEF1AF01CEF1AF027EF1AF08A
:10343800080108014F513E0AD8A425EF1AF027EFDA
:103448001AF029EF1AF02BEF1AF085EF19F008019E
:10345800526F000E08010801536F0801525167ECC2
:103468003DF012004CC850F84DC851F850C8E9FF5B
:1034780051C8EAFFEF50080108014F6F0801080121
:10348800504B512B080108014F51D8B44EEF1AF098
:1034980050EF1AF07CEF1AF0080108014F512E0A7C
:1034A800D8B459EF1AF05BEF1AF07CEF1AF0080164
:1034B80008014F512F0AD8B464EF1AF066EF1AF0DA
:1034C8007CEF1AF0080108014F512C0AD8B46FEFAD
:1034D8001AF071EF1AF07CEF1AF0080108014F5149
:1034E8003E0AD8A47AEF1AF07CEF1AF03AEF1AF0F5
:1034F800080108014C5108010801505D0801526F8C
:1035080008015205080108014E6F4EC853F867ECD0
:103518003DF0080108014EC855F808010801566B2E
:103528004CC853F84DC854F8F9EC30F0010E0801B6
:1035380008015327000E08015423080108015351BC
:10354800080108014C270801080154510801080125
:103558004D23080108014F51D8B4B5EF1AF0B7EF61
:103568001AF0D8EF1AF0080108014F512F0AD8B401
:10357800C0EF1AF0C2EF1AF0D8EF1AF008010801EC
:103588004F512C0AD8B4CBEF1AF0CDEF1AF0D8EF80
:103598001AF0080108014F513E0AD8A4D6EF1AF0D4
:1035A800D8EF1AF0DAEF1AF0DCEF1AF03AEF1AF067
:1035B8000801526F000E08010801536F08015251AB
:1035C80067EC3DF012004CC8E9FF4DC8EAFFEECFAA
:1035D80050F8EECF51F8EECF52F8EECF53F8040181
:1035E8000401DC510801531911E104010401DB5104
:1035F800080152190BE104010401DA5108015119BB
:1036080005E104010401D95108015019D8B40FEF9C
:103618001BF011EF1BF083EF1BF004010401DC51D8
:1036280000010001771914E104010401DB510001D4
:10363800000176190DE104010401DA5100010001CD
:10364800751906E104010401D9510001000174193A
:10365800D8A431EF1BF033EF1BF094EF1BF04CC8EC
:10366800E9FF4DC8EAFFEECF50F8EECF51F8EECFA4
:1036780052F8EECF53F8000100016C5108015019BF
:103688000801546F000100016D510801511908012A
:10369800556F000100016E51080152190801566F5B
:1036A800000100016F51080153190801576F00010B
:1036B80000017051080154150801586F00010001FC
:1036C8007151080155150801596F00010001725127
:1036D8000801561508015A6F0001000173510801CD
:1036E800571508015B6F08015B51581159115A11A0
:1036F800D8B481EF1BF083EF1BF094EF1BF004EEBE
:10370800DDF008014EC8E1FF08014FC8E2FF060ED0
:10371800EECFE6FFE82E8CEF1BF0010E97EF1BF0C3
:10372800000E97EF1BF012009AEF1BF0CBEC3DF068
:103738000009D8B4A2EF1BF0A4EF1BF09AEF1BF01E
:10374800CF0E08010801AC6F0A0E0801AD6F0BEC33
:1037580044F078C8E9FF79C8EAFF010EEE6E000E62
:10376800ED6E020E080108017825E96E000E0801C9
:1037780008017921EA6E000EEE6E080EED6E040E59
:10378800080108017825E96E000E08010801792171
:10379800EA6E060EEF6E050E080108017825E96E3F
:1037A800000E080108017921EA6E040EEF6E060E7C
:1037B80008010801B06F000E0801B16F990E0801E9
:1037C8007A6F000E7B6F7AC8AEF87BC8AFF8080E28
:1037D80008010801782508010801AC6F000E0801EE
:1037E800080179210801AD6F58EC3AF00E0E080176
:1037F80008017825E96E000E080108017921EA6EB2
:1038080000016CC0EEFF00016DC0EEFF00016EC04C
:10381800EEFF00016FC0EEFF78C87CF879C87DF82C
:103828009EEC30F01C0E08010801BD6F000E080167
:10383800BE6F08017A6F060E08010801BC6F080107
:103848007A51120E08010801782508010801BA6F9B
:10385800000E0801080179210801BB6FC4EC33F0A0
:103868001C0E08010801C26F000E0801C36F78C85A
:10387800C0F879C8C1F8BBEC40F003EC39F0010E90
:1038880046EF1CF0120008011B6F000E080108012A
:10389800186F08011B510801080116AF56EF1CF0FC
:1038A80058EF1CF067EF1CF008010801156D0801BE
:1038B800161FD8B0162B08011B6F010E080108014E
:1038C800186F08011B510801080114AF6EEF1CF0B6
:1038D80070EF1CF07BEF1CF008010801136D080164
:1038E800141FD8B0142B010E08010801181B000E74
:1038F80008010801196F000E08011A6F0801080174
:1039080016511511D8B48BEF1CF08DEF1CF0DCEFBD
:103918001CF008011B6F010E08010801176F080150
:103928001B51A0EF1CF00801D890080115370801B9
:10393800163708010801172B0801080116AFA7EF71
:103948001CF0A9EF1CF097EF1CF00801D8900801B3
:10395800193708011A37080108011551080108012B
:10396800135D080108011651080108011459D8A06F
:10397800C0EF1CF0C2EF1CF0D1EF1CF008010801E9
:10398800155108010801135F0801080116510801C3
:103998000801145B0801080119810801D890080181
:1039A80016330801153308010801172FA9EF1CF079
:1039B800080108011851D8B4E4EF1CF0E6EF1CF038
:1039C800EDEF1CF008010801196D08011A1FD8B0A5
:1039D8001A2B19C813F81AC814F8F3EF1CF01200C0
:1039E800990E08010801566FFF0E0801576F4CEC3D
:1039F80027F00009D8A403EF1DF005EF1DF007EF2D
:103A08001DF0A0EF1DF0C9EC26F065C8F8F566C8F2
:103A1800F9F567C8FAF568C8FBF5CF0E0801080183
:103A2800566FFF0E0801576F4CEC27F00009D8A419
:103A380020EF1DF022EF1DF024EF1DF0A0EF1DF088
:103A4800C9EC26F065C814F766C815F78C0E08018E
:103A58000801566FFF0E0801576F4CEC27F000095C
:103A6800D8A439EF1DF03BEF1DF03DEF1DF0A0EF9E
:103A78001DF0C9EC26F065C818F766C819F76DEC93
:103A880044F00801556F000E08010801536F080142
:103A98005551090E08010801536555EF1DF057EF00
:103AA8001DF059EF1DF09EEF1DF00801556F020E35
:103AB80008010801566F0801555177EC44F039ECBC
:103AC8002AF00801556F000E08010801546F08011B
:103AD80055510A0E08010801546575EF1DF077EF7E
:103AE8001DF079EF1DF091EF1DF00E0E0801556FD6
:103AF800850EE82E7DEF1DF0552F7DEF1DF000D0CF
:103B080008010801542B0A0E0801080154658FEFBB
:103B18001DF091EF1DF079EF1DF008010801532BFE
:103B2800090E0801080153659CEF1DF09EEF1DF07A
:103B380059EF1DF05FEC44F01200000E0801080177
:103B4800006F000E0801016F000E0801026F000EE1
:103B58000801036F000E0E010E01B66F000E0E0174
:103B68000E01B76F000E926E000E936E000E946EEB
:103B7800000E956E000E966E000E976E000E986EF3
:103B8800000E806E000E816E000E826E000E836E37
:103B9800000E846E000E856E0801046F400E9B6E49
:103BA800080104510801046F0F0EC16E0801045189
:103BB80042EC44F09CEC43F002EC3DF069EC44F03C
:103BC8005FEC01F0FEECE7F080EC43F0D1EC3AF06A
:103BD800420E080108010B6F370E08010C6F08012F
:103BE800046F140E080108010A6F0801045199ECCA
:103BF80040F0CBECCCF07DEC44F0C4EC43F0080191
:103C08000801005108010801A15D0801046F0801BD
:103C18000801015108010801A2590801056F0801AE
:103C28000801025108010801A3590801066F08019B
:103C38000801035108010801A4590801076FF20E91
:103C4800045D9E0E0559000E0659000E080107591D
:103C5800D8A031EF1EF033EF1EF03DEF1EF0C4EC9C
:103C680043F0A1C800F8A2C801F8A3C802F8A4C884
:103C780003F81AECC7F050ECE2F0EFECC4F019ECE2
:103C8800B6F046EC26F00400FDEF1DF014EF00F04E
:103C980012C817F811C816F882EC2FF008010801AD
:103CA800136F0701070113675CEF1EF05EEF1EF04C
:103CB80066EF1EF00801146F000E070107013B6F45
:103CC80008011451080108011351FE0AD8A46FEF26
:103CD8001EF071EF1EF07AEF1EF0FE0E08010801CB
:103CE800116FFF0E0801126FF1EF1EF008010801B5
:103CF8001329D8A482EF1EF084EF1EF08BEF1EF07C
:103D080008010801116908011269F1EF1EF00701A5
:103D180007011151040AD8A494EF1EF096EF1EF083
:103D2800A2EF1EF007013B3BF00E3B170801146F92
:103D3800000E07010701116F08011451080108015D
:103D48001351D8B4AAEF1EF0ACEF1EF0C1EF1EF06D
:103D580011C714F8010E0801156F0801142BB8EFEC
:103D68001EF0D890080115370801142FB5EF1EF082
:103D780008011551070107013B1307010701132B20
:103D880007010701112B080E070107011361CFEF87
:103D98001EF0D1EF1EF0D8EF1EF0080108011169DE
:103DA80008011269F1EF1EF00801146F000E0701F7
:103DB8000701136F080114510801146F000E070161
:103DC8000701116F08011451070108013BC711F8D9
:103DD80008010801126BF1EF1EF01200D8900801DB
:103DE8000801BD3108010801BF6F08010801BC3195
:103DF8000801BE6FBAC8C0F8BBC8C1F8000E0801F8
:103E08000801C26F000E0801C36F000E0801C46FDD
:103E1800000E0801C56F34EF1FF00801C0C8E9FFA4
:103E28000801C1C8EAFF0801020E0801C027000EF8
:103E38000801C123EECFC6F8EDCFC7F80801C65177
:103E480008010801C2270801C75108010801C32356
:103E5800000E08010801C423000E08010801C5234B
:103E680008010801BE07D8A0BF070801BE29D8B4B9
:103E7800BF29D8A442EF1FF044EF1FF011EF1FF045
:103E880008010801BCA14BEF1FF04DEF1FF060EFD8
:103E98001FF0C0C8E9FFC1C8EAFFEF500801C66FAC
:103EA8000801C65108010801C227000E0801C323F2
:103EB8000801C4230801C52308010801C2510801EB
:103EC8000801C42508010801C26F08010801C3518F
:103ED80008010801C5210801C36F0801C46BD8B0E7
:103EE800C42B0801C56B080108EEC4F0EE500801A8
:103EF8000801C227ED5008010801C3230801080181
:103F0800C21D08010801BA6F08010801C31D080194
:103F1800BB6F8FEF1FF01200000E08010801376F0A
:103F2800000E0801386F000E0801396F000E0801F5
:103F38003A6F08013551321133113411D8B4A7EF53
:103F48001FF0A9EF1FF01CEF20F008013B6F010ED6
:103F580008010801366F08013B51C0EF1FF0080146
:103F6800D89008013237080133370801343708017F
:103F7800353708010801362B0801080135AFC7EFAE
:103F88001FF0C9EF1FF0B3EF1FF00801D890080128
:103F98003737080138370801393708013A37080137
:103FA80008013251080108012E5D0801080133514A
:103FB800080108012F5908010801345108010801B6
:103FC8003059080108013551080108013159D8A0B4
:103FD800F0EF1FF0F2EF1FF00DEF20F008010801DD
:103FE8003251080108012E5F080108013351080108
:103FF80008012F5B08010801345108010801305BF2
:1040080008010801355108010801315B0801080160
:1040180037810801D8900801353308013433080185
:1040280033330801323308010801362FC9EF1FF076
:1040380037C82EF838C82FF839C830F83AC831F8D8
:1040480026EF20F0120007010701A529D8A42FEFB9
:1040580020F031EF20F056EF20F0FEC653F8FFC6EF
:1040680054F8FEC651F8FFC652F80801336F040E23
:1040780008010801506F08013351630E0801346FBD
:10408800060E356F080134C84CF8080135C84DF8DC
:10409800080108014E6B08014F6B22ECD7F00701AD
:1040A8000701A56F07010701A529D8A45EEF20F035
:1040B80060EF20F062EF20F0BDEF20F0A5C74CF8CC
:1040C80093EC39F008014D514C11D8A46EEF20F053
:1040D80070EF20F072EF20F0BDEF20F0DEEC43F03F
:1040E80036C82FF837C830F82FC859F830C85AF8EA
:1040F8003DEC37F059C82DF85AC82EF8000E0801C3
:104108000801316F000E0801326FA3EF20F008019B
:1041180008013151080108012F25E96E080108013D
:104128003251080108013021EA6EEF5008010801F8
:10413800536F67EC3DF008010801314B322B080141
:1041480008013251800A0801336F08012D51080116
:104158000801315D080108012E51800A0801335910
:10416800D8A0B9EF20F0BBEF20F08BEF20F053EC94
:1041780021F01200000E080108016865C6EF20F062
:10418800C8EF20F0D1EF20F0000E08010801686F99
:10419800000E0801696F52EF21F068C871F81DEC34
:1041A8002BF017C06AF8080108016A51070AD8B449
:1041B800E0EF20F0E2EF20F0F6EF20F00801080130
:1041C8006A510B0AD8B4EBEF20F0EDEF20F0F6EFD0
:1041D80020F0000E08010801686F000E0801696FE1
:1041E80052EF21F000EE09F010EE07F0E652EE5221
:1041F800ED50E55C02E1EF50E75CD8A006EF21F056
:1042080008EF21F039EF21F000EE07F0EECF6BF860
:10421800EDCF6CF8095008016B5F0A5008016C5B20
:1042280000EE03F0EECF6DF8EDCF6EF80150080107
:104238006D5F025008016E5BFF0E08016D250801D5
:104248006F6FFF0E08016E210801706F08016B5136
:1042580008016F5D08010801686F08016C510801C9
:1042680070590801696F52EF21F000EE09F0EECFA6
:104278006BF8EDCF6CF8075008016B5F0850080128
:104288006C5BFF0E08016B2508010801686FFF0EC3
:1042980008016C210801696F52EF21F01200070133
:1042A80007010D51170D0201000EF3240801080142
:1042B8004E6F08014F6B0201020E08014F23080ED2
:1042C80006010601BC25080108014C6F000E060115
:1042D8000601BD2108014D6F0C0E080108014E258D
:1042E800E96E000E080108014F21EA6E0801EECFC1
:1042F800BCF80801EDCFBDF82FEC43F0BCC850F86E
:10430800BDC851F80A0E080108014E25E96E000ED5
:10431800080108014F21EA6E0801EECFBCF8080138
:10432800EDCFBDF82FEC43F0BCC852F8BDC853F828
:104338004CC8BCF84DC8BDF82FEC43F0BCC854F8C5
:10434800BDC855F8000E08010801566F000E080197
:10435800576FDD0E08010801AC6F0A0E0801AD6F3A
:104368000BEC44F04CC8A3F84DC8A4F80801586FEA
:10437800110E08010801A26F080158514EC8A0F893
:104388004FC8A1F8CAEC18F0080E08010801C26F5E
:10439800000E0801C36F0801500E08010801C06F24
:1043A8000801080E0801C16FBBEC40F003EC39F0BE
:1043B800000E06010601BC6F000E0601BD6F070165
:1043C8000701A069120070EF22F06DC8B0F86EC83E
:1043D800B1F86BC8AEF86CC8AFF868C8ACF869C873
:1043E800ADF858EC3AF07AEF22F008010801682994
:1043F800D8B46929D8B403EF22F005EF22F00BEF07
:1044080022F068C8ACF869C8ADF80BEC44F0100E9F
:10441800080108016F6F000E0801706F63EF22F04A
:10442800080108016F51080108016D5D08010801C4
:104438007051080108016E59D8B025EF22F027EF16
:1044480022F02BEF22F06DC86FF86EC870F86FC8B5
:10445800B0F870C8B1F86BC8AEF86CC8AFF808010E
:10446800710E08010801AC6F0801080E0801AD6F54
:1044780058EC3AF06FC8C2F870C8C3F80801710E5A
:1044880008010801C06F0801080E0801C16FBBECE4
:1044980040F0080108016F51080108016B27000E60
:1044A800080108016C23080108016F51080108017F
:1044B8006D5F080108017051080108016E5B080171
:1044C80008016E516D11D8A46CEF22F06EEF22F046
:1044D80014EF22F07AEF22F0080108016A51000A6D
:1044E80084E0010A01E171D77AEF22F01200080195
:1044F800776F000E08010801766F080177510E0EDC
:104508000801080176658BEF22F08DEF22F08FEF1E
:1045180022F007EF23F0010E070107018C150801AF
:10452800776F000E070107018D150801786F000EDF
:10453800070107018E150801796F000E07010701B1
:104548008F1508017A6F08017751000808017B6F01
:10455800000E0801785508017C6F000E0801795596
:1045680008017D6F000E08017A5508017E6F010E63
:1045780008017B1508017F6F000E08017C150801F2
:10458800806F000E08017D150801816FD00E0801AB
:104598007E150801826F07018CC783F807018DC754
:1045A80084F807018EC785F807018FC786F8D89069
:1045B8000801863385338433833308017F5108012A
:1045C8008319070107018C6F0801805108018419BC
:1045D80007018D6F080181510801851907018E6F48
:1045E800080182510801861907018F6F0801080127
:1045F800762B0E0E08010801766505EF23F007EF0C
:1046080023F08FEF22F08CC774F88DC775F80DEF83
:1046180023F01200010E08010801566F000E080170
:10462800576F0801080162690801080163690801F8
:1046380008016469080108016569080108016669DB
:104648000801080167694CC84EF84DC84FF84CC8B6
:10465800E9FF4DC8EAFFEECF6CF8EECF6DF8EECF6C
:104668006EF8EECF6FF8000100016C5108016C196B
:104678000801706F000100016D5108016D190801F2
:10468800716F000100016E5108016E190801726F07
:10469800000100016F5108016F190801736F0001D3
:1046A80000017051080170150801746F00010001C4
:1046B8007151080171150801756F000100017251EF
:1046C800080172150801766F000100017351080195
:1046D80073150801776F08017751741175117611F8
:1046E800D8B479EF23F07BEF23F084EF23F00001B7
:1046F800740E080108014E6F0001000E08014F6F8B
:104708004EC8E9FF4FC8EAFF0801EECF68F8080174
:10471800EECF69F80801EECF6AF80801EECF6BF822
:104728000801500E08010801786F0801080E0801F9
:10473800796F98EC1BF0120022EF24F0D2EF23F0EF
:10474800AAC8B0F8ABC8B1F8A7C8AEF8A8C8AFF8FF
:10475800A4C8ACF8A5C8ADF858EC3AF0DBEF23F0E4
:1047680008010801A429D8B4A529D8B4BEEF23F0BC
:10477800C0EF23F0C6EF23F0A4C8ACF8A5C8ADF885
:104788000BEC44F0AAC8C2F8ABC8C3F8A7C8C0F875
:10479800A8C8C1F8BBEC40F0DBEF23F00801080122
:1047A800A651000ADDE0010ACBE0DBEF23F02CEF95
:1047B80024F019EF24F008010801A729D8B4A82982
:1047C800D8B4E9EF23F0EBEF23F0F1EF23F0A7C81B
:1047D800ACF8A8C8ADF82CEC44F0AAC8C4F8ABC82B
:1047E800C5F8A4C8C2F8A5C8C3F86DEC38F0DBEF6B
:1047F80023F0AAC8B0F8ABC8B1F8A7C8AEF8A8C8E3
:10480800AFF8A4C8ACF8A5C8ADF83CECDDF00DEFE6
:1048180024F08EEC43F00009D8B415EF24F017EF1C
:1048280024F00DEF24F0DBEF23F008010801A65176
:10483800000ADFE0010ABFE0DBEF23F0080108010E
:10484800A951000AB6E0010A01E178D72CEF24F05B
:1048580012002FEF24F0C5CF2CF81F0E08012C17DB
:104868002CC82DF808012E6B000EC7B4010E0801E4
:104878002D13000E2E1308012E512D11D8A447EF29
:1048880024F049EF24F02FEF24F0C5804CEF24F0FA
:10489800C5B051EF24F053EF24F04CEF24F0A1A65B
:1048A80058EF24F05AEF24F05CEF24F0B6EF24F030
:1048B80029C82FF819EC3AF00009D8B466EF24F0AB
:1048C80068EF24F06BEF24F0C584B6EF24F0C5BC84
:1048D80070EF24F072EF24F09EEF24F02AC82FF82E
:1048E80019EC3AF00009D8B47CEF24F07EEF24F0FC
:1048F80081EF24F0C584B6EF24F0C5BC86EF24F020
:1049080088EF24F099EF24F02BC82FF819EC3AF02F
:104918000009D8B492EF24F094EF24F097EF24F034
:10492800C584B6EF24F09CEF24F0C584B6EF24F0DC
:10493800A1EF24F0C584B6EF24F0C584A4EF24F0D9
:10494800C5B4A9EF24F0ABEF24F0A4EF24F0A1A69E
:10495800B0EF24F0B2EF24F0B4EF24F0B6EF24F077
:10496800B6EF24F0120007010701A451070107015F
:104978009F63C1EF24F0C3EF24F0C5EF24F03EEFAE
:1049880025F0070107019F51FE0AD8B4CEEF24F0A5
:10499800D0EF24F019EF25F0270E08010801AA6FBF
:1049A800000E0801AB6F0801A06F010E0801080195
:1049B800A96F0801A0511D0E08010801A76F000E7C
:1049C8000801A86F070107019F511C0DF3CFA1F83B
:1049D8001B0E0801A1270401BD0E0801A125E96EDF
:1049E800EA6A0401040EEA22EF5008010801A66FE2
:1049F800070107019F511C0D0401BD0EF324E96E48
:104A0800EA6A0401040EEA22EECFA2F8EDCFA3F879
:104A1800D90E0801A22508010801A46FFF0E08019C
:104A2800A3210801A56FA0EC23F0A4C79FF7270EC8
:104A380008010801AA6F000E0801AB6F1CC0A9F895
:104A4800D90E012408010801A76FFF0E02200801F2
:104A5800A86F0801A06F010E08010801A66F0801E0
:104A6800A0511D0E08010801A46F000E0801A56FD2
:104A7800A0EC23F012000701D89033370801080191
:104A8800F051D8B44AEF25F04CEF25F06FEF25F040
:104A980007010701262B070107012651030AD8A49D
:104AA80058EF25F05AEF25F060EF25F0070E0701C3
:104AB800070133136DEF25F0030E07010701266583
:104AC80068EF25F06AEF25F06DEF25F00701070183
:104AD800338177EF25F00801F16F000E0701070118
:104AE800266F0801F1510701D890393707010701EE
:104AF8003F2B0701070133AF84EF25F086EF25F040
:104B08008BEF25F00701070139818BEF25F00701AD
:104B180007013F51080AD8A494EF25F096EF25F035
:104B2800C2EF25F00801F16F000E070107013F6F82
:104B38000801F151B30E06010601D825E96E020EEF
:104B480006010601D921EA6E070139C7EFFF060100
:104B58000601D84BD92B06010601D951020AD811F2
:104B6800D8A4B9EF25F0BBEF25F0C2EF25F0000E71
:104B780006010601D86F000E0601D96F1200D9CEC2
:104B8800A4F8EECEA2F8EFCEA3F808010801A451CC
:104B98000E010E01D963D3EF25F0D5EF25F0C3EF51
:104BA80025F0ECCEA4F8EDCEA5F808010801A25135
:104BB80008010801A45D08010801A35108010801C2
:104BC800A559D8B0EAEF25F0ECEF25F00BEF26F069
:104BD8000801A2C8A6F80801A3C8A7F80801080197
:104BE800A4510801A65F08010801A5510801A75BA7
:104BF8000801A651CD0808010801A06F0801A751B6
:104C0800D8A0E82A0A080801A16F45EF26F0080194
:104C18000801A55108010801A31906E108010801C6
:104C2800A45108010801A219D8A41DEF26F01FEF0E
:104C380026F028EF26F0CD0E08010801A06F0A0E15
:104C48000801A16F45EF26F00801A4C8A6F80801DD
:104C5800A5C8A7F808010801A2510801A65F080124
:104C68000801A3510801A75BFF0E0801A62508014A
:104C78000801A06FFF0E0801A7210801A16F45EFE9
:104C880026F01200BFEF26F04A0E08010801536F04
:104C9800A50E0801546F4A0E08010801516FA50EB0
:104CA8000801526F0801096F040E08010801506FCE
:104CB80008010951000E080108014C6F000E080197
:104CC8004D6F000E08014E6F000E08014F6F22EC69
:104CD800D7F006010601E66F06010601E629D8A409
:104CE80078EF26F07AEF26F07CEF26F0C8EF26F072
:104CF8000801096F010E070107013E6F08010951FC
:104D0800C8EF26F0E6C64CF8D9EC39F008014D5149
:104D18004C11D8A492EF26F094EF26F096EF26F0E7
:104D2800C8EF26F065EC3FF0A9EF26F00801080E61
:104D3800080108014D6F0801080E08014E6F35EC97
:104D48003DF008C864F88FEC3FF0E6C64CF8D9ECA3
:104D580039F008014D514C11D8A4B5EF26F0B7EF42
:104D680026F09AEF26F08FEC41F0C8EC15F065ECD0
:104D78003FF0C8EF26F0070107013E51000A84E022
:104D8800010AC0E0C8EF26F01200000E0801080171
:104D98006D6F000E08016E6F000E08016F6F000E38
:104DA8000801706F77EC41F00009D8A4DEEF26F017
:104DB800E0EF26F0EFEF26F0000E08010801656F1E
:104DC800000E0801666F000E0801676F000E0801EB
:104DD800686F4BEF27F004010401FF2B37EF27F032
:104DE8000101000E04010401FF25E96EEA6A0101D0
:104DF800010EEA22EF500801716F08017151080194
:104E08000801696F08016A6B08016B6B08016C6B1C
:104E180004010401FF2B08016951730A6A116B111F
:104E28006C11D8A41AEF27F01CEF27F01EEF27F01B
:104E380041EF27F00801040ED89008016D370801EA
:104E48006E3708016F3708017037E82E20EF27F01A
:104E580069C872F82DEC2DF00801716F08017151C5
:104E6800080108016D13C70E04010401FF653FEF37
:104E780027F041EF27F0F4EF26F06DC865F86EC80B
:104E880066F86FC867F870C868F84BEF27F012002B
:104E98002DC7FFF4BEEF27F00801646F0C0E080160
:104EA8000801676F080164510801580E08010801DC
:104EB800656F0801080E0801666F0EEC18F000090E
:104EC800D8A469EF27F06BEF27F06EEF27F0000EFC
:104ED800CBEF27F00801580E08010801676F080199
:104EE800080E0801686F56C865F857C866F849EC97
:104EF80029F0080166516511D8A485EF27F087EFDE
:104F080027F08AEF27F0010ECBEF27F077EC41F07E
:104F18000009D8B492EF27F094EF27F098EF27F024
:104F2800C9EC26F0A9EF27F00801646F000E08010C
:104F38000801676F08016451000E08010801656FD8
:104F4800000E0801666F0EEC18F00101000E040156
:104F58000401FF25E96EEA6A0101010EEA22730ED7
:104F6800EF62B9EF27F0BBEF27F0BEEF27F0000E96
:104F7800CBEF27F0C70E04010401FF65C6EF27F049
:104F8800C8EF27F050EF27F0000ECBEF27F0120004
:104F980058C8E9FF59C8EAFF010EEE6E230EEE6EFF
:104FA800450EEE6E670EED6EED52ED52040E0801E1
:104FB80008015825E96E000E080108015921EA6E1A
:104FC800890EEE6EAB0EEE6ECD0EEE6EEF0EED6E42
:104FD800ED52ED52080E080108015825E96E000E41
:104FE800080108015921EA6EFE0EEE6EDC0EEE6E27
:104FF800BA0EEE6E980EED6EED52ED520C0E0801E3
:1050080008015825E96E000E080108015921EA6EC9
:10501800760EEE6E540EEE6E320EEE6E100EED6ED5
:10502800ED52ED52100E080108015825E96E000EE8
:10503800080108015921EA6EF00EEE6EE10EEE6EDF
:10504800D20EEE6EC30EED6EED52ED52140E080147
:1050580008015825E96E000E080108015921EA6E79
:10506800000EEE6E000EEE6E000EEE6E000EED6E91
:10507800ED52ED52580E080108015825E96E000E50
:10508800080108015921EA6E010EEF6E12000DC8E1
:1050980013F894EC2DF013C810F814C811F808018F
:1050A800080111511011D8A45CEF28F05EEF28F028
:1050B80061EF28F0000EC9EF28F00DC871F81DEC5B
:1050C8002BF0080108010F510E11D8B46EEF28F02B
:1050D80070EF28F08BEF28F0010E08010801AA6F85
:1050E800000E0801AB6F1CC0A9F80DC0A7F80EC0D0
:1050F800A8F80801126F010E08010801A66F08013F
:1051080012510EC8A4F80FC8A5F8A0EC23F000EEC1
:105118000DF0EE2A000EED2210EE05F0E652EE52EA
:10512800ED50E55C02E1EF50E75CD8B09EEF28F067
:10513800A0EF28F0A4EF28F003C00DF004C00EF093
:105148000801080110051111D8A4ADEF28F0AFEF40
:1051580028F0B2EF28F01984C6EF28F018BAB7EF94
:1051680028F0B9EF28F0C6EF28F0188A5AEC42F078
:105178001F0E08010801A125136E000E0801080181
:10518800A221146E010EC9EF28F012000094000E3F
:10519800070107010E6F009253C8E9FF54C8EAFFE0
:1051A800EF5007010701126FB180DBEF28F000A272
:1051B800E0EF28F0E2EF28F0DBEF28F09D92010EF7
:1051C80008010801556F000E0801566F25EF29F0F8
:1051D800080108015551080108015325E96E080125
:1051E80008015651080108015421EA6E010EEF62C8
:1051F80000EF29F002EF29F005EF29F0008421EFF4
:1052080029F00092080108015551080108015325A9
:10521800E96E080108015651080108015421EA6E97
:10522800EF5007010701126F1AEF29F000A21FEFD4
:1052380029F021EF29F01AEF29F008010801554B50
:10524800562B080108015551080108015325E96E3C
:10525800080108015651080108015421EA6EEF506F
:10526800D8A439EF29F03BEF29F0ECEF28F09D8224
:1052780000923FEF29F000A244EF29F046EF29F011
:105288003FEF29F0B190899812004DEF29F04DEFCA
:1052980029F008010801675108016A6F080108012F
:1052A800685108016B6F0801674B682B6AC8F6FFE5
:1052B8006BC8F7FF000EF86E0E0EF76403D00800F7
:1052C800F55005D0F6CFE9FFF7CFEAFFEF50080118
:1052D8006C6F080165C8F6FF080166C8F7FF000E85
:1052E800F86E0E0EF76403D00800F55005D0F6CF1F
:1052F800E9FFF7CFEAFFEF5008016D6F08016C5125
:1053080008016D5D08010801696F080169678FEF81
:1053180029F091EF29F0B7EF29F00801080165514C
:1053280008016A6F08010801665108016B6F0801DE
:10533800654B662B6AC8F6FF6BC8F7FF000EF86E60
:105348000E0EF76403D00800F55005D0F6CFE9FF3C
:10535800F7CFEAFFEF500009D8A4B5EF29F0B7EF6F
:1053680029F04BEF29F008010801695108010801EB
:10537800656F0801666B080165BF6607C4EF29F011
:1053880012000001000198ADCCEF29F0CEEF29F012
:10539800FDEF29F000010001EC690001ED69000151
:1053A800EE690001EF6900010001F0690001F1698F
:1053B8000001F2690001F36900010001F4690001CC
:1053C800F5690001F6690001F76900010001F86953
:1053D8000001F9690001FA690001FB690001000197
:1053E800FC690001FD690001FE690001FF6925EF04
:1053F8002AF06CC0ECF06DC0EDF06EC0EEF06FC03E
:10540800EFF070C0F0F071C0F1F072C0F2F073C04C
:10541800F3F074C0F4F075C0F5F076C0F6F077C01C
:10542800F7F078C0F8F079C0F9F07AC0FAF07BC0EC
:10543800FBF07CC0FCF07DC0FDF07EC0FEF07FC0BC
:10544800FFF0250E08010801246F000E0801256FE2
:105458000001DB0E08010801226F0001000E08019F
:10546800236F4DEC39F0FF0012008988050E080102
:10547800566F300EE82E3EEF2AF0562F3EEF2AF0F8
:1054880089982B0E0801566F560EE82E49EF2AF020
:10549800562F49EF2AF004000801566F020E080142
:1054A8000801586F08015651FBC557F840EC30F019
:1054B8000801566F080E08010801586F0801565177
:1054C800FAC557F840EC30F00801566F080E08018D
:1054D8000801586F08015651F9C557F840EC30F0EB
:1054E8000801566F080E08010801586F0801565147
:1054F800F8C557F840EC30F0B4EC3EF0070107016E
:1055080018051911D8A48BEF2AF08DEF2AF091EF26
:105518002AF05AEC3EF093EF2AF0B4EC3EF0080182
:10552800566F040E08010801586F0801565114C738
:1055380057F840EC30F08988050E0801566F300E98
:10554800E82EA4EF2AF0562FA4EF2AF0899812002B
:105558000801326F000E08010801316F080132514D
:105568002EC8E9FF2FC8EAFFEF5008010801356F80
:105578002CC8E9FF2DC8EAFF0801EECF33F808016F
:10558800EDCF34F887EC3EF0D8B0CDEF2AF0D0EF6D
:105598002AF0010ED1EF2AF0000E08010801306F41
:1055A80008010801312B2EC835F82FC836F82CC849
:1055B80033F82DC834F899EC3CF02EC8E9FF2FC811
:1055C800EAFFEF5008010801356F2CC8E9FF2DC824
:1055D800EAFF0801EECF33F80801EDCF34F887EC85
:1055E8003EF0D8B0FAEF2AF0FDEF2AF0010EFEEFF8
:1055F8002AF0000E080108013019D8B406EF2BF084
:1056080008EF2BF00DEF2BF00801080131511CEFCA
:105618002BF0080108013129D8A415EF2BF017EF5A
:105628002BF01AEF2BF0000E1CEF2BF0D4EF2AF022
:10563800120008010801715107010701A46327EF4F
:105648002BF029EF2BF02BEF2BF08AEF2BF0070133
:105658000701A451FE0AD8B434EF2BF036EF2BF033
:1056680056EF2BF01C0E08010801B06F000E080160
:10567800B16F010E08010801AE6F000E0801AF6F8F
:1056880007010701A4511C0D0401BD0EF3240801F4
:105698000801AC6F0801AD6B0401040E0801AD23CD
:1056A80058EC3AF071C8A4F7080108017151FE0AD4
:1056B800D8A461EF2BF063EF2BF065EF2BF08AEFA6
:1056C8002BF01C0E08010801B06F000E0801B16F25
:1056D8000801080171511C0DBD0E0801726F040EFE
:1056E800736FF35008017227E86AF3BEE86808018F
:1056F800732372C8AEF873C8AFF8010E0801080129
:10570800AC6F000E0801AD6F58EC3AF012008DEF47
:105718002BF0C5CF2AF81F0E08012A172AC82BF824
:1057280008012C6B000EC7B4010E08012B13000EE4
:105738002C1308012C512B11D8A4A5EF2BF0A7EF9F
:105748002BF08DEF2BF0C580AAEF2BF0C5B0AFEF93
:105758002BF0B1EF2BF0AAEF2BF0A1A6B6EF2BF0B0
:10576800B8EF2BF0BAEF2BF0F7EF2BF029C82FF892
:1057780019EC3AF0C0EF2BF0DBEF2BF0C582C5EF48
:105788002BF0C5B2CAEF2BF0CCEF2BF0C5EF2BF006
:10579800A1A6D1EF2BF0D3EF2BF0D5EF2BF0F7EF3D
:1057A8002BF029C82FF819EC3AF0DBEF2BF0C5BC29
:1057B800E0EF2BF0E2EF2BF0C2EF2BF0C584E5EF22
:1057C8002BF0C5B4EAEF2BF0ECEF2BF0E5EF2BF064
:1057D800A1A6F1EF2BF0F3EF2BF0F5EF2BF0F7EF9D
:1057E8002BF0F7EF2BF0120006010601CE5106014F
:1057F8000601D25D06010601CF5106010601D35903
:10580800D8B009EF2CF00BEF2CF018EF2CF00701B3
:105818000701A351070107010D19D8B416EF2CF0A1
:1058280018EF2CF01AEF2CF05EEF2CF006010601B1
:10583800D25106010601CE5D08010801516F06012B
:105848000601D35106010601CF590801526F08011C
:1058580008014F5108010801515D08010801505124
:10586800080108015259D8B03CEF2CF03EEF2CF05B
:1058780042EF2CF051C84FF852C850F84FC8C4F83E
:1058880050C8C5F84DC8C2F84EC8C3F86DEC38F01A
:10589800C2C84FF8C3C850F8080108014F510601A3
:1058A8000601D22708010801505106010601D32339
:1058B8005EEF2CF01200020E08010801BA25E96E0D
:1058C800000E08010801BB21EA6E0801EECFBCF802
:1058D8000801EDCFBDF82FEC43F0020E08010801D6
:1058E800BA25E96E000E08010801BB21EA6E08011D
:1058F800BCC8EEFF0801BDC8EDFF040E0801080191
:10590800BA25E96E000E08010801BB21EA6E0801FC
:10591800EECFBCF80801EDCFBDF82FEC43F0040E34
:1059280008010801BA25E96E000E08010801BB212B
:10593800EA6E0801BCC8EEFF0801BDC8EDFF0A0EFB
:1059480008010801BA25E96E000E08010801BB210B
:10595800EA6E0801EECFBCF80801EDCFBDF82FECD8
:1059680043F00A0E08010801BA25E96E000E080185
:105978000801BB21EA6E0801BCC8EEFF0801BDC8DA
:10598800EDFF120012C816F811C815F80CECE7F074
:1059980008010801136F080108011351FE0AD8A471
:1059A800D8EF2CF0DAEF2CF0E3EF2CF0FE0E080124
:1059B8000801116FFF0E0801126F2CEF2DF008017E
:1059C80008011329D8A4EBEF2CF0EDEF2CF0F4EF3D
:1059D8002CF0080108011169080112692CEF2DF05B
:1059E8000701D8903533080108011351D8B4FFEFE7
:1059F8002CF001EF2DF004EF2DF007010701358F92
:105A080007010701292B070107012C2B080E0701A5
:105A180007012C6112EF2DF014EF2DF01BEF2DF084
:105A2800080108011169080112692CEF2DF008011D
:105A3800146F000E070107012C6F080114510701AC
:105A4800080135C711F808010801126B2CEF2DF079
:105A580012005FEF2DF0000E93EF2DF0010E93EF83
:105A68002DF0020E93EF2DF0030E93EF2DF0040EA0
:105A780093EF2DF0050E93EF2DF0060E93EF2DF01A
:105A8800070E93EF2DF0080E93EF2DF0090E93EF0C
:105A98002DF00A0E93EF2DF00B0E93EF2DF00C0E58
:105AA80093EF2DF00D0E93EF2DF00E0E93EF2DF0DA
:105AB8000F0E93EF2DF0080108017251300ACBE068
:105AC800010ACCE0030ACDE0010ACEE0070ACFE0E4
:105AD800010AD0E0030AD1E0010AD2E00F0AD3E0BC
:105AE800010AD4E0780AD5E0030AD6E0010AD7E033
:105AF800070AD8E0010AD9E0030ADAE0270AC9E070
:105B0800030ACAE0010ACBE0070ACCE0010ACDE0AB
:105B1800030ACEE090EF2DF0000E93EF2DF0120067
:105B2800000E0801080113659CEF2DF09EEF2DF083
:105B3800A7EF2DF0000E08010801136F000E0801F1
:105B4800146FF9EF2DF013C871F81DEC2BF000EE6F
:105B58000DF010EE0BF0E652EE52ED50E55C02E16E
:105B6800EF50E75CD8A0BBEF2DF0BDEF2DF0C8EFEC
:105B78002DF00D500B5C08010801136F0E500C58E6
:105B88000801146FF9EF2DF000EE0BF0EECF15F8C9
:105B9800EDCF16F803500801155F04500801165B95
:105BA80000EE05F0EECF17F8EDCF18F80D5008010C
:105BB800175F0E500801185B0801155108011725D9
:105BC8000801196F080116510801182108011A6FF8
:105BD800010E0801192508010801136F000E0801BC
:105BE8001A210801146FF9EF2DF0120045EF2EF07D
:105BF80013C8E9FF14C8EAFFEF50D8B406EF2EF037
:105C080008EF2EF021EF2EF0080115C8F6FF080165
:105C180016C8F7FF000EF86E0800F5CF19F813C87C
:105C2800E9FF14C8EAFFEF5008011919D8B41FEFAB
:105C38002EF021EF2EF03DEF2EF013C8E9FF14C827
:105C4800EAFFEF500801196F080115C8F6FF0801AF
:105C580016C8F7FF000EF86E0800F5500801195D28
:105C680008010801136F0801146BD8A014075EEF30
:105C78002EF008010801134B142B08010801154BDD
:105C8800162B080108011707D8A0180708011729BB
:105C9800D8B41829D8A453EF2EF055EF2EF0FCEF06
:105CA8002DF0000E08010801136F000E0801146F93
:105CB8005EEF2EF01200800E08010801276F000E1B
:105CC8000801286F0801080128512711D8A46FEF8F
:105CD8002EF071EF2EF073EF2EF0BCEF2EF00801CE
:105CE800000E080122BF010E08010801256F0801F6
:105CF800266B08010801235108010801271500092E
:105D0800D8B489EF2EF08BEF2EF097EF2EF0080124
:105D1800080126512511000ED8B4010E080108010A
:105D2800256F0801266B0801D89022370801080161
:105D380026512511D8B4A3EF2EF0A5EF2EF0ABEF26
:105D48002EF008010801245108010801221B08014E
:105D5800D890080128330801273308010801285181
:105D68002711D8A4BAEF2EF0BCEF2EF073EF2EF067
:105D7800080108012251C1EF2EF0120027C82EF8A1
:105D880028C82FF825C82CF826C82DF8ACEC2AF01E
:105D9800080108012A6F1D0E080108012A65D7EFBE
:105DA8002EF0D9EF2EF0E6EF2EF0290E08010801AB
:105DB8002A61E1EF2EF0E3EF2EF0E6EF2EF0000E71
:105DC80021EF2FF027C82EF828C82FF825C82CF85F
:105DD80026C82DF8ACEC2AF008010801296F090E35
:105DE800080108012A65FBEF2EF0FDEF2EF01EEFEB
:105DF8002FF0150E080108012A6105EF2FF007EFB3
:105E08002FF01EEF2FF0090E0801080129650FEF8A
:105E18002FF011EF2FF01EEF2FF0150E08010801DB
:105E2800296119EF2FF01BEF2FF01EEF2FF0010E55
:105E380021EF2FF0020E21EF2FF012000601000EC5
:105E480008010801586F0601060E0801596FCCECCD
:105E580027F00101000E08010801596F0101010E28
:105E680008015A6F3DEC37F059C856F85AC857F828
:105E780056C85CF857C85DF80101000E0801080112
:105E88005A6F0101010E08015B6F0601000E08013F
:105E98000801586F0601060E0801596FC1EC11F090
:105EA800200E080108015C6F000E08015D6F470EA7
:105EB800080108015A6FFE0E08015B6F0601000E0B
:105EC80008010801586F0601060E0801596FE8EC31
:105ED80010F00401E30E080108015A6F0401040ED2
:105EE80008015B6F0601000E08010801586F0601E2
:105EF800060E0801596F89ECB9F012000D0E080161
:105F0800080117658AEF2FF08CEF2FF0B4EF2FF010
:105F1800160E08010801176194EF2FF096EF2FF085
:105F2800B4EF2FF006010601C4A19DEF2FF09FEFFB
:105F38002FF0A2EF2FF0FE0EE0EF2FF0020E060179
:105F48000601C42506010601C46F000E06010601FC
:105F5800C5210601C56F080108011651E0EF2FF0B1
:105F6800050E080108011765BCEF2FF0BEEF2FF0F2
:105F7800DDEF2FF00C0E080108011761C6EF2FF0B6
:105F8800C8EF2FF0DDEF2FF006010601C44BC52B3B
:105F980006010601C4B1D3EF2FF0D5EF2FF0DAEFE9
:105FA8002FF0080108011651E0EF2FF0FF0EE0EF87
:105FB8002FF0FE0EE0EF2FF01200080108010D2966
:105FC800D8B40E29D8A4EBEF2FF0EDEF2FF0F4EFB3
:105FD8002FF0080108010D6908010E693FEF30F044
:105FE800080108011051800A0801116F08010D51BC
:105FF800080108010F5D080108010E51800A080117
:106008001159D8A00AEF30F00CEF30F01FEF30F044
:10601800080108010D51080108010F5D0801080178
:106028000D6F080108010E510801080110590801F7
:106038000E6F3FEF30F0000E0801116F020E126F65
:10604800080108010D510801115F080108010E51EE
:106058000801125B080108010F5108011125080108
:1060680008010D6F080108011051080112210801EB
:106078000E6F3FEF30F0120008015B6F010E080150
:1060880008015A6F08015B5108015B6F000E080197
:106098000801596F08015B5158C85BF8FF0E0801E9
:1060A8005B27010E08015C6F08015B2B5FEF30F086
:1060B800D89008015C3708015B2F5CEF30F00801CD
:1060C8005C51080108015A6F08015B6F000E080156
:1060D8000801596F08015B5190EF30F00801080181
:1060E8005751080108015A150009D8B47EEF30F05D
:1060F80080EF30F084EF30F05AEC3EF086EF30F06D
:10610800B4EC3EF00801D89008015A3108010801A2
:106118005A6F08010801592B080108015851080154
:106128000801595DD8A09BEF30F09DEF30F072EF79
:1061380030F012007CC8E9FF7DC8EAFF0801EECF05
:10614800BCF80801EDCFBDF82FEC43F07CC8E9FF9F
:106158007DC8EAFF0801BCC8EEFF0801BDC8EDFF15
:10616800020E080108017C25E96E000E08010801ED
:106178007D21EA6E0801EECFBCF80801EDCFBDF82D
:106188002FEC43F0020E080108017C25E96E000E91
:10619800080108017D21EA6E0801BCC8EEFF08016C
:1061A800BDC8EDFF060E080108017C25E96E000E4A
:1061B800080108017D21EA6E0801EECFBCF808014C
:1061C800EDCFBDF82FEC43F0060E080108017C2541
:1061D800E96E000E080108017D21EA6E0801BCC8BD
:1061E800EEFF0801BDC8EDFF120004010401FB51D8
:1061F800C00808010801576F04010401FC51D8A028
:10620800E82A05080801586F0801080155510801D6
:106218000801575D0801080156510801080158593D
:10622800D8B019EF31F01BEF31F01FEF31F057C83C
:1062380055F858C856F808010801555104010401D9
:10624800FB2708010801565104010401FC2304013D
:106258000401FB5106010601BC5D04010401FC5167
:1062680006010601BD59D8B03CEF31F03EEF31F0E0
:1062780042EF31F0FBC4BCF6FCC4BDF655C8C2F809
:1062880056C8C3F853C8C0F854C8C1F8BBEC40F0AE
:1062980055C853F856C854F852EF31F012000401AB
:1062A8000401FB51C00808010801576F04010401EB
:1062B800FC51D8A0E82A05080801586F0801080110
:1062C800555108010801575D080108015651080198
:1062D80008015859D8B073EF31F075EF31F079EF04
:1062E80031F057C855F858C856F8080108015551F3
:1062F80004010401FB2708010801565104010401A7
:10630800FC2304010401FB5106010601BC5D0401E4
:106318000401FC5106010601BD59D8B096EF31F0D1
:1063280098EF31F09CEF31F0FBC4BCF6FCC4BDF62D
:1063380055C85BF856C85CF853C859F854C85AF899
:106348002EEC40F055C853F856C854F8ACEF31F06D
:1063580012000F0E080108012465B5EF31F0B7EF00
:1063680031F0D8EF31F00A0E080108012561BFEFBE
:1063780031F0C1EF31F0D8EF31F00A0E0801080111
:106388002661C9EF31F0CBEF31F0D8EF31F00A0ECA
:10639800080108012761D3EF31F0D5EF31F0D8EFCC
:1063A80031F0000E06EF32F00A0E080108012461F0
:1063B800E0EF31F0E2EF31F003EF32F00A0E0801BE
:1063C80008012561EAEF31F0ECEF31F003EF32F02C
:1063D8000F0E080108012665F4EF31F0F6EF31F0F1
:1063E80003EF32F00A0E080108012761FEEF31F0D1
:1063F80000EF32F003EF32F0010E06EF32F0020E3A
:1064080006EF32F012000F0E080108011F650FEFAA
:1064180032F011EF32F032EF32F00A0E08010801C3
:10642800206119EF32F01BEF32F032EF32F00F0E2D
:1064380008010801216523EF32F025EF32F032EF31
:1064480032F00A0E0801080122612DEF32F02FEF19
:1064580032F032EF32F0000E60EF32F00A0E08012F
:1064680008011F613AEF32F03CEF32F05DEF32F095
:106478000F0E08010801206544EF32F046EF32F0B4
:106488005DEF32F00F0E0801080121654EEF32F082
:1064980050EF32F05DEF32F00A0E08010801226178
:1064A80058EF32F05AEF32F05DEF32F0010E60EF44
:1064B80032F0020E60EF32F012000D0E08010801F2
:1064C8001F6169EF32F06BEF32F08CEF32F00D0E96
:1064D80008010801206173EF32F075EF32F08CEF9C
:1064E80032F00D0E0801080121617DEF32F07FEFD7
:1064F80032F08CEF32F0100E08010801226587EFA8
:1065080032F089EF32F08CEF32F0010EBAEF32F050
:106518000D0E080108011F6194EF32F096EF32F07A
:10652800B7EF32F0100E0801080120659EEF32F037
:10653800A0EF32F0B7EF32F00D0E0801080121612B
:10654800A8EF32F0AAEF32F0B7EF32F00D0E0801E3
:1065580008012261B2EF32F0B4EF32F0B7EF32F057
:10656800000EBAEF32F0020EBAEF32F01200000E4F
:1065780008010801156F000E0801166F000E0801CA
:10658800176F000E0801186F080108010DA1CFEF61
:1065980032F0D1EF32F0E9EF32F008010801115181
:1065A800080108011527080108011251080108010E
:1065B80016230801080113510801080117230801CF
:1065C800080114510801080118230801D89008018E
:1065D8001137080112370801133708011437080169
:1065E800D8900801103308010F3308010E33080151
:1065F8000D33080110510D110E110F11D8A407EF1A
:1066080033F009EF33F0C8EF32F015C80DF816C8AB
:106618000EF817C80FF818C810F813EF33F0120067
:10662800C2C8F7F4C3C8F8F4C4C8F9F4C5C8FAF482
:10663800C6C8C8F8080E08010801C86126EF33F07B
:1066480028EF33F02AEF33F042EF33F0FAC4C7F8FB
:10665800F9C4FAF4F8C4F9F4F7C4F8F4C7C8F7F4BD
:10666800080E08010801C85F080E08010801C86182
:1066780040EF33F042EF33F02AEF33F0080108011E
:10668800C86749EF33F04BEF33F04DEF33F061EF6C
:1066980033F00401D890FABFD880F737F837F937C4
:1066A800FA3708010801C80708010801C8675FEF41
:1066B80033F061EF33F04DEF33F0F7C4C2F8F8C4AC
:1066C800C3F8F9C4C4F8FAC4C5F86BEF33F0120084
:1066D800B7EC24F02DC01AF02EC01BF001C007F053
:1066E80002C008F001C009F002C00AF003C00BF0B4
:1066F80004C00CF003C00DF004C00EF00801736F65
:106708000D0E08010801726F0801735118A68FEF6A
:1067180033F091EF33F099EF33F00801736F040E03
:1067280008010801726F0801735172C817F01890B8
:10673800189218940B000E001898189A189C189E16
:10674800199019921994199619883F903F923F967B
:106758003F9801C029F002C02AF07BEC22F074C8EF
:1067680021F075C822F07BEC22F074C823F075C8BC
:1067780024F03D683E68010E2F6E000E306E120048
:10678800CF0E0E010E01E26F0A0E0E01E36F080133
:10679800DC0E0801BD270A0E0801BE23BDC8E6FEAF
:1067A800BEC8E7FE060E08010801C26F000E080108
:1067B800C36FBAC8C0F8BBC8C1F8BBEC40F0060E3E
:1067C80008010801C26F000E0801C36F0001990E8D
:1067D80008010801C06F0001000E0801C16FBBEC81
:1067E80040F00801BF6F080E08010801C06F0801DA
:1067F800BF5164EC44F00801BF6F060E08010801A0
:10680800C06F0801BF5108010801BC670EEF34F0E2
:1068180010EF34F018EF34F00801BF6F000E0801D4
:106828000801C06F0801BF5164EC44F01200070171
:1068380007013A6722EF34F024EF34F04EEF34F0DA
:1068480008011F6F010E070107013A6F08011F5168
:1068580008011F6F000E080108011E6F08011F5173
:10686800000E080108011E653CEF34F03EEF34F0DD
:1068780040EF34F04EEF34F04468080108011E2B55
:10688800000E080108011E654CEF34F04EEF34F09D
:1068980040EF34F04428D8B454EF34F056EF34F0D5
:1068A8005BEF34F044C04CF8A3EC36F044680801C0
:1068B8001F6F010E00010001456F08011F510801FB
:1068C8001F6F000E00010001466F08011F510001F3
:1068D80046890001468312000A0E08010801B06FBC
:1068E800000E0801B16F06010601E651170D000EF2
:1068F8000801226F020E236FF35008012227E86A6D
:10690800F3BEE8680801232322C8AEF823C8AFF80D
:106918000601630E08010801AC6F0601060E0801A6
:10692800AD6F58EC3AF006010601E651170DF3CFAA
:1069380022F80A0E080122270201000E080122256A
:10694800E96EEA6A0201020EEA220601EECFFEF6BD
:106958000601EDCFFFF607010701A529D8B4B7EF67
:1069680034F0B9EF34F0C2EF34F0A5C74CF8A3EC1B
:1069780036F007010701A569C2EF34F01200FACF1B
:10698800CCF8FBCFCDF8E9CFCEF8EACFCFF8E1CFFE
:10699800D0F8E2CFD1F8D9CFD2F8DACFD3F8F3CF05
:1069A800D4F8F4CFD5F8F6CFD6F8F7CFD7F8F8CF94
:1069B800D8F8F5CFD9F8F2A4E4EF34F0E6EF34F0E4
:1069C800E8EF34F004EC42F09EA2EDEF34F0EFEF84
:1069D80034F0F2EF34F08AEC0CF09E92D9C8F5FF4F
:1069E800D8C8F8FFD7C8F7FFD6C8F6FFD5C8F4FF50
:1069F800D4C8F3FFD3C8DAFFD2C8D9FFD1C8E2FFA1
:106A0800D0C8E1FFCFC8EAFFCEC8E9FFCDC8FBFF79
:106A1800CCC8FAFFCBC8E0FFCAC8E8FFC9C8D8FF8E
:106A28001000EACFE5F8E1CFE6F8E2CFE7F8D9CFF2
:106A3800E8F8DACFE9F8F3CFEAF8F4CFEBF8F6CFD5
:106A4800ECF8F7CFEDF8F8CFEEF8F5CFEFF8A4A60D
:106A580030EF35F032EF35F03DEF35F0E20E786E7D
:106A6800000E81B8010E08010801F06F3FEC25F017
:106A7800A496A1A242EF35F044EF35F04AEF35F085
:106A8800B368C40EB26ECEEC3CF0A192EFC8F5FF2D
:106A9800EEC8F8FFEDC8F7FFECC8F6FFEBC8F4FF47
:106AA800EAC8F3FFE9C8DAFFE8C8D9FFE7C8E2FF98
:106AB800E6C8E1FFE5C8EAFFE4C8E9FFE3C8FBFF71
:106AC800E2C8FAFF110038C859F839C85AF83DEC3D
:106AD80037F008010801595108010801586F0DECF9
:106AE8003FF0080108013B6F38C859F839C85AF80F
:106AF8003DEC37F008010801595108010801646F9D
:106B0800E1EC3EF0080108013A6F080108013B5129
:106B1800300AD8B492EF35F094EF35F098EF35F0AD
:106B28003BC864F88FEC3FF03AC864F88FEC3FF04C
:106B380008013C6F3A0E08010801646F08013C51D6
:106B48008FEC3FF038C85AF839C85BF80101000EDD
:106B580008010801586F0101010E0801596F89ECFD
:106B680037F0120053C859F854C85AF83DEC37F0BA
:106B780008010801595108010801586F0DEC3FF050
:106B880008010801566F53C859F854C85AF83DEC23
:106B980037F008010801595108010801646FE1EC58
:106BA8003EF008010801556F080108015651300AE6
:106BB800D8B4E1EF35F0E3EF35F0E7EF35F056C83C
:106BC80064F88FEC3FF055C864F88FEC3FF008018B
:106BD800576F3A0E08010801646F080157518FEC8E
:106BE8003FF053C85AF854C85BF80101000E080179
:106BF8000801586F0101010E0801596F89EC37F03F
:106C080012000801276F000E06010601D66F080161
:106C18002751000E06010601CA6F000E0601CB6F50
:106C2800000E0601CC6F000E0601CD6F000E0501A7
:106C38000501FC6F000E0501FD6F000E0501FE6FDA
:106C4800000E0501FF6F010E07010701906F000E8E
:106C58000701916F000E0701926F000E0701936FF5
:106C68000801276F000E070107010A6F0801275165
:106C7800000E07010701166F000E0701176F0801C4
:106C8800276F000E06010601E86F08012751080169
:106C9800276F000E070107010C6F0801275112002A
:106CA8008CC735F88DC736F88EC737F88FC738F8D0
:106CB80008013351301131113211D8A466EF36F082
:106CC80068EF36F075EF36F0010E08010801306FF5
:106CD800000E0801316F000E0801326F000E080126
:106CE800336F30C88CF731C88DF732C88EF733C888
:106CF8008FF70801396F000E08010801346F080189
:106D080039510F0E0801080134658DEF36F08FEF09
:106D180036F091EF36F0A0EF36F07BEC22F0080168
:106D28000801342B0F0E0801080134659EEF36F078
:106D3800A0EF36F091EF36F0A2EF36F01200040E15
:106D4800080108014C65ABEF36F0ADEF36F0AFEF58
:106D580036F0EFEF36F0080108014C51170DF3CF6C
:106D68004DF80C0E08014D270201000E08014D25B3
:106D7800E96EEA6A0201020EEA22000EEE6E000EC9
:106D8800ED6E080108014C51170D0201000EF324A5
:106D9800E96EEA6A0201020EEA22000EEE6E000EA9
:106DA800EE6E000EEE6E000EED6EED52ED52080125
:106DB80008014C51170DF3CF4DF80E0E08014D2761
:106DC8000201000E08014D25E96EEA6A0201020E71
:106DD800EA22040EEF6E12000601DBC645F8060132
:106DE800DCC646F8080108013D510801452708019D
:106DF80008013E5108014623140E080145250801E3
:106E08000801436F000E080146210801446FCE0EA9
:106E180008010801435D0A0E08014459D8A017EF7C
:106E280037F019EF37F020EF37F00801CE0E0801E0
:106E3800435F0A0E0801445BE0CE41F8E1CE42F818
:106E480043C8E0FE44C8E1FE3FC8A0F840C8A1F826
:106E58000EEC10F0A0C843F8A1C844F841C8E0FE01
:106E680042C8E1FE43C83DF844C83EF83CEF37F05D
:106E7800120059C85BF85AC85CF845EF37F045EF7F
:106E880037F0080108015B5108015D6F080108012E
:106E98005C5108015E6F08015B4B5C2B5DC8F6FF17
:106EA8005EC8F7FF000EF86E0E0EF76403D00800F8
:106EB800F55005D0F6CFE9FFF7CFEAFFEF5000090C
:106EC800D8A469EF37F06BEF37F043EF37F00801DC
:106ED8005BC85DF808015CC85EF8080108015951F3
:106EE80008015D5F080108015A5108015E5BFF0E49
:106EF80008015D2508010801596FFF0E08015E2190
:106F080008015A6F88EF37F0120058C85CF859C862
:106F18005DF893EF37F0080108015C4B5D2B5CC806
:106F2800E9FF5DC8EAFFEF50D8A49DEF37F09FEF67
:106F380037F08FEF37F0A1EF37F0080108015A5109
:106F480008015E6F080108015B5108015F6F0801C5
:106F58005A4B5B2B5EC8F6FF5FC8F7FF000EF86E52
:106F680008015CC8E1FF08015DC8E2FF08010801EB
:106F78005C4B5D2B0E0EF76403D00800F55005D06E
:106F8800F6CFE9FFF7CFEAFFEF50E76EE750D8A456
:106F9800D0EF37F0D2EF37F09FEF37F0D4EF37F07C
:106FA800120008014C0E080108014D6F0801080E77
:106FB80008014E6F35EC3DF00009D8A4E6EF37F034
:106FC800E8EF37F0EAEF37F020EF38F00801080172
:106FD8004C51C00BC00AD8A4F4EF37F0F6EF37F0E5
:106FE80003EF38F008014C0E080108014D6F080145
:106FF800080E08014E6F35EC3DF020EF38F008011F
:1070080008014C670AEF38F00CEF38F00EEF38F053
:1070180020EF38F0080108014CC84FF808010801B2
:10702800506B000E080108014D6F000E08014E6FED
:10703800F8EC2BF0D5EF37F0120024C82EF825C84D
:107048002FF822C82CF823C82DF8ACEC2AF0080138
:107058000801266F24C82EF825C82FF822C82CF856
:1070680023C82DF8ACEC2AF008010801276F0D0E93
:1070780008010801266543EF38F045EF38F052EF74
:1070880038F00D0E0801080127654DEF38F04FEF75
:1070980038F052EF38F0000E6CEF38F00B0E0801A4
:1070A800080126615AEF38F05CEF38F069EF38F0E4
:1070B8000D0E08010801276564EF38F066EF38F017
:1070C80069EF38F0010E6CEF38F0020E6CEF38F013
:1070D8001200C4C8C6F8C5C8C7F808010801C351DA
:1070E800C211D8B47AEF38F07CEF38F09DEF38F061
:1070F8008BEF38F061CF7EFEC2C8E9FFC3C8EAFF54
:107108000E017ECEEFFF08010801C24BC32B080118
:107118000801C607D8A0C7070801C629D8B4C729D7
:10712800D8A499EF38F09BEF38F07EEF38F0B1EF44
:1071380038F0A1EF38F061CF7EFE08010801C607DC
:10714800D8A0C7070801C629D8B4C729D8A4AFEF63
:1071580038F0B1EF38F09FEF38F0C4C8C2F8C5C8AE
:10716800C3F8B7EF38F0120022EC2FF00801146FC3
:10717800000E08010801136F08011451130E0801CD
:1071880008011365CAEF38F0CCEF38F0CEEF38F0CD
:10719800FFEF38F00501E40E080108011325E96E38
:1071A800EA6A0501050EEA22EF500801146F04018E
:1071B800E30E080108011325E96EEA6A0401040ECA
:1071C800EA22EF5008011419D8B4EDEF38F0EFEFC8
:1071D80038F0F2EF38F0000E02EF39F0080108013C
:1071E800132B130E080108011365FDEF38F0FFEFAC
:1071F80038F0CEEF38F0010E02EF39F012000E0130
:10720800DF8F0E01DF9F080E08010801A06F0DEF48
:1072180039F008010801A0070801A029D8A417EF30
:1072280039F019EF39F00DEF39F00E01FC93060132
:107238000601D5B322EF39F024EF39F044EF39F0E5
:1072480006010601D5B52BEF39F02DEF39F044EFE3
:1072580039F05AEC42F0A1C81AF7A2C81BF7060188
:10726800D58506010601D5A73CEF39F03EEF39F088
:1072780041EF39F08D8242EF39F08D920601D577D2
:107288000E01DF87C4EC43F0A1C81EF7A2C81FF7A0
:1072980012000801276F000E08010801266F080177
:1072A80027517CEF39F022C8E9FF23C8EAFFEF50E5
:1072B800080108012B6F26C82AF80801276FA00EBD
:1072C80008010801296F080127512DEC24F0080155
:1072D8000801224B232B0801276FA00E0801080183
:1072E800296F080127518BEC2BF008010801262B88
:1072F800080126C827F80801286B0801080124514D
:107308000801275D08010801255108012859D8A05E
:1073180090EF39F092EF39F057EF39F01200CBECDB
:107328003DF00009D8A49BEF39F09DEF39F0A6EFA6
:1073380039F0000E080108014C6F000E08014D6F6E
:10734800D8EF39F007010701A051080108014C19CD
:10735800D8B4B1EF39F0B3EF39F0C5EF39F04CC814
:10736800A0F7000E06010601BC6F000E0601BD6FF6
:10737800000E080108014E6F000E08014F6FBFECA8
:1073880042F04CC80DF706010601BC51C0080801BF
:1073980008014C6F06010601BD51D8A0E82A05086E
:1073A80008014D6FD8EF39F012004CC80DF70701EE
:1073B8000701A351080108014C19D8B4E6EF39F0C8
:1073C800E8EF39F0F1EF39F0000E080108014C6FD1
:1073D800000E08014D6F18EF3AF0070107010FA1E1
:1073E800F8EF39F0FAEF39F005EF3AF007010F91AD
:1073F800000E080108014E6F000E08014F6F83EC64
:1074080042F006010601D25106010601CE5D0801CF
:1074180008014C6F06010601D35106010601CF5938
:1074280008014D6F18EF3AF012002FC8C9FFC6AE19
:1074380020EF3AF022EF3AF025EF3AF0FF0E57EF3F
:107448003AF027EF3AF0C7B02CEF3AF02EEF3AF0C7
:1074580027EF3AF030EF3AF0C5CF30F81F0E0801A9
:10746800301730C831F80801326B000EC7B4010E6E
:1074780008013113000E3213080132513111D8A41A
:1074880048EF3AF04AEF3AF030EF3AF0C5AC4FEF38
:107498003AF051EF3AF054EF3AF0FE0E57EF3AF067
:1074A800000E57EF3AF01200AEC8B4F8AFC8B5F8FE
:1074B800ACC8B2F8ADC8B3F882EF3AF00801B4C866
:1074C800F6FF0801B5C8F7FF000EF86EB2C8E1FF75
:1074D800B3C8E2FF0E0EF76403D00800F55005D0DC
:1074E800F6CFE9FFF7CFEAFFEF50E76E0801080192
:1074F800B44BB52B08010801B24BB32B08010801A6
:10750800B007D8A0B1070801B029D8B4B129D8A4C8
:1075180090EF3AF092EF3AF062EF3AF094EF3AF0E7
:10752800120008010E6F000E080108010D6F080116
:107538000E51BAEF3AF00DC811F808010E6FA00EFF
:1075480008010801106F08010E51C6EC06F0080189
:107558000801105109C8E9FF0AC8EAFFEF6E0801DF
:107568000801094B0A2B080108010D2B08010DC859
:107578000EF808010F6B080108010B5108010E5D98
:10758800080108010C5108010F59D8A0CEEF3AF0B4
:10759800D0EF3AF09FEF3AF012000801086F000EA2
:1075A80007010701556F080108510001988F9BECEE
:1075B80003F016C830F817C831F818C832F819C8D7
:1075C80033F854EC36F02EEC0FF01DEC41F0B8EC2B
:1075D8003FF0C9ECDFF00801086F000E0801080150
:1075E8001D6F080108511BEC34F00001000198BD23
:1075F80000EF3BF002EF3BF00CEF3BF00801086FA7
:10760800000E08010801096F080108511AEC42F040
:1076180012000401B30E08010801336F0401040EBF
:107628000801346F2DC831F82EC832F812ECD2F0A8
:107638000009D8B422EF3BF024EF3BF030EF3BF0E9
:10764800070108830801306F070E07010701A66FBD
:107658000801305147EF3BF02DC806F72EC807F751
:10766800000E07010701226F000E0701236F0801B2
:10767800306F000E07010701A66F080130512FC8AF
:107688003CF70701089312000401B30E0801080132
:10769800336F0401040E0801346F2DC831F82EC869
:1076A80032F892ECCEF00009D8B45DEF3BF05FEF12
:1076B8003BF06BEF3BF0070108830801306F070EC2
:1076C80007010701A66F0801305182EF3BF0000E59
:1076D80007010701066F000E0701076F2DC822F783
:1076E8002EC823F70801306F000E07010701A66FA7
:1076F800080130512FC83CF7070108931200000E0B
:1077080008010801646F000E0801656F080108018F
:1077180060A191EF3BF093EF3BF09FEF3BF0080146
:107728000801625108010801642708010801635132
:107738000801080165230801D8900801623708018B
:1077480063370801D89008016133080160330801E4
:10775800080161516011D8A4B4EF3BF0B6EF3BF0DB
:107768008AEF3BF064C860F865C861F8BCEF3BF08D
:107778001200320E080108015D6F000E08015E6FED
:10778800000E080108015B6F000E08015C6F010123
:10779800C80E08010801596F0101010E08015A6F4E
:1077A80053EC40F0000E07010701276F000E070198
:1077B800286F08010D6F000E070107012E6F0801E1
:1077C8000D5108010D6F000E070107011D6F08011B
:1077D8000D5108010D6F000E070107012F6F0801F9
:1077E8000D511200000E080108016865FEEF3BF01C
:1077F80000EF3CF002EF3CF02DEF3CF068C871F868
:107808001DEC2BF0B7EC24F000EE29F010EE07F099
:10781800E652EE52ED50E518EFCFE8FFD8B4E7187E
:10782800D8B419EF3CF01BEF3CF02DEF3CF0080109
:10783800696F010E08010801736F08016951080199
:107848006A6F100E08010801726F08016A519FECF7
:10785800A1F0120006010601D5A135EF3CF037EF83
:107868003CF039EF3CF063EF3CF00601D581FF0EA8
:1078780006010601FC25080108014C6FFF0E0601F0
:107888000601FD2108014D6FCE0E080108014C5D6F
:107898000A0E08014D59D8A054EF3CF056EF3CF0C1
:1078A8005DEF3CF0CD0E080108014C6F0A0E08018F
:1078B8004D6F0E01FE8D4CC8ECFE4DC8EDFE12005A
:1078C8000601DBC67FF80601DCC680F8080108015E
:1078D8007B5108017F27080108017C51080180239A
:1078E800140E08017F25080108017D6F000E0801AC
:1078F800802108017E6FCE0E080108017D5D0A0E09
:1079080008017E59D8A08BEF3CF08DEF3CF094EF46
:107918003CF00801CE0E08017D5F0A0E08017E5B6F
:107928007DC8E0FE7EC8E1FE120035C8E9FF36C812
:10793800EAFFD890EF3635C8E9FF36C8EAFFEF50BE
:10794800D8A4A9EF3CF0ABEF3CF0CDEF3CF035C844
:10795800E9FF36C8EAFF010EEF6E33C8E9FF34C805
:10796800EAFFEE50ED10D8A4BCEF3CF0BEEF3CF0BF
:10797800C6EF3CF033C8E9FF34C8EAFF000EEE6EEC
:10798800020EED6E33C8E9FF34C8EAFFEE06000EBA
:10799800ED5A1200070107010E67D5EF3CF0D7EF4B
:1079A8003CF0F4EF3CF00082070107011267DFEFBB
:1079B8003CF0E1EF3CF0E3EF3CF001EF3DF012C7A3
:1079C8000EF7000E07010701126F00B4EEEF3CF04E
:1079D800F0EF3CF0F3EF3CF08978F4EF3CF00094E2
:1079E800070107010E51D8B4FCEF3CF0FEEF3CF064
:1079F80001EF3DF0070107010E0712009E92CB68C8
:107A0800CA82CA9CCA8ACA88CA869F929D82CA8428
:107A1800000EBD6E000EBA6EBA86BA84BA9EBA9CC3
:107A2800BD86BD84BD9EBD9CBD86BD84BA86BA8414
:107A3800BD9ABD98BA9ABA98000EBE6E000EBB6E7B
:107A48000801086F000E07010701866F0801085139
:107A58000801086F000E070107017D6F0801085132
:107A6800120006010601CE5106010601D25D06018B
:107A78000601CF5106010601D359D8B046EF3DF0B3
:107A880048EF3DF055EF3DF007010701A35107010D
:107A980007010D19D8B453EF3DF055EF3DF058EFFD
:107AA8003DF0000E66EF3DF04BEC44F04DC8E9FFA9
:107AB8004EC8EAFFEF6E06010601D24BD32B010E2A
:107AC80066EF3DF01200C00E04010401FB5D050ED7
:107AD8000401FC59D8A073EF3DF075EF3DF077EF46
:107AE8003DF098EF3DF053C8C0F864EC44F0040151
:107AF8000401FB4BFC2B04010401FB5106010601A8
:107B0800BC5D04010401FC5106010601BD59D8B051
:107B180090EF3DF092EF3DF096EF3DF0FBC4BCF6E0
:107B2800FCC4BDF698EF3DF012000D0E08010801E7
:107B38002C61A1EF3DF0A3EF3DF0B0EF3DF00D0E4D
:107B4800080108012D61ABEF3DF0ADEF3DF0B0EF5E
:107B58003DF0000ECAEF3DF0180E080108012C6533
:107B6800B8EF3DF0BAEF3DF0C7EF3DF00D0E08015C
:107B780008012D61C2EF3DF0C4EF3DF0C7EF3DF0C5
:107B8800010ECAEF3DF0020ECAEF3DF012000E01E1
:107B98000E01DFB7D2EF3DF0D4EF3DF0D7EF3DF067
:107BA800010EFAEF3DF0C4EC43F0070107011E5146
:107BB80008010801A15F070107011F510801080119
:107BC800A25B7A0E08010801A15D000E0801A25906
:107BD800D8A0F1EF3DF0F3EF3DF0F7EF3DF00E01E7
:107BE800DF9703EC39F0000EFAEF3DF012000801C0
:107BF8000801695167C8E9FF68C8EAFFEF6207EF43
:107C08003EF009EF3EF00FEF3EF067C867F868C82E
:107C180068F82AEF3EF0080167C8E9FF080168C85C
:107C2800EAFF08010801674B682BEF50D8A41FEF43
:107C38003EF021EF3EF0FBEF3DF0000E0801080199
:107C4800676F000E0801686F2AEF3EF01200080106
:107C58000801A55108010801A21B08010801A25149
:107C680008010801A51B08010801A5510801080120
:107C7800A21B08010801A45108010801A31B08015F
:107C88000801A35108010801A41B08010801A45117
:107C980008010801A31BA2C8A2F8A3C8A3F8A4C896
:107CA800A4F8A5C8A5F859EF3EF012008988050E7A
:107CB80008015D6F300EE82E5FEF3EF05D2F5FEF3D
:107CC8003EF08998150E08015D6F6C0EE82E6AEF7C
:107CD8003EF05D2F6AEF3EF08988050E08015D6F62
:107CE800300EE82E75EF3EF05D2F75EF3EF0899867
:107CF800050E08015D6F300EE82E80EF3EF05D2F17
:107D080080EF3EF01200B30E080108013325E96E3A
:107D1800020E080108013421EA6EEF50080108013B
:107D2800366F080108013651080135C837F80801CF
:107D3800386B37BF380708013717000E38170801A6
:107D480038513711D8B4ABEF3EF0ADEF3EF0B0EF9D
:107D58003EF0D880B3EF3EF0D890B3EF3EF012007B
:107D68008988050E08015D6F300EE82EB9EF3EF0E8
:107D78005D2FB9EF3EF08998050E08015D6F300E52
:107D8800E82EC4EF3EF05D2FC4EF3EF08988050E63
:107D980008015D6F300EE82ECFEF3EF05D2FCFEF7C
:107DA8003EF08998150E08015D6F6C0EE82EDAEF2B
:107DB8003EF05D2FDAEF3EF012000F0E08010801C9
:107DC8006417300E08010801642508010801656F71
:107DD8000801666B000E08016623090E08010801F8
:107DE8006465F9EF3EF0FBEF3EF007EF3FF0370E2A
:107DF80008010801642508010801656F0801666B20
:107E0800000E080166230801080165510CEF3FF0D8
:107E180012000801583B0F0E5817300E08010801D0
:107E2800582508010801596F08015A6B000E08010E
:107E38005A23090E08010801586525EF3FF027EF7E
:107E48003FF033EF3FF0370E0801080158250801CD
:107E58000801596F08015A6B000E08015A230801DE
:107E68000801595138EF3FF0120037C8B4FE00F04E
:107E780008013B6F010E0E010E01B26F08013B5164
:107E880000F047EF3FF00E010E018AB14EEF3FF0D0
:107E980050EF3FF047EF3FF008013B6F000E0E0137
:107EA8000E01B26F08013B5100F0B8CE39F800F06E
:107EB800B9CE3AF839C837F83AC838F864EF3FF01D
:107EC8001200C80E080108015D6F000E08015E6F00
:107ED800000E080108015B6F000E08015C6F0101CC
:107EE800000E08010801596F0101010E08015A6FBF
:107EF80053EC40F00801566F000E04010401FF6FB7
:107F0800080156510801566F000E06010601D76F89
:107F1800080156511200000E08010801696F000E91
:107F280008016A6F0101000E08010801676F01016D
:107F3800010E0801686FFBEC3DF067C865F868C87A
:107F480066F80801080166516511D8B4AEEF3FF034
:107F5800B0EF3FF0B7EF3FF065C8E9FF66C8EAFF4A
:107F6800080164C8EFFF120008010A6F000E08013B
:107F78000801096F08010A51040E08010801096582
:107F8800C8EF3FF0CAEF3FF0CCEF3FF0DDEF3FF036
:107F980009C84CF8A3EC36F008010801092B040EB7
:107FA800080108010965DBEF3FF0DDEF3FF0CCEF9A
:107FB8003FF007010F8312000801116F000E07013F
:107FC80007012A6F080111510801116F000E0701FE
:107FD8000701106F08011151000E06010601C46F58
:107FE800000E0601C56F0801116F000E0701070199
:107FF800136F080111510801116F000E07010701E5
:10800800116F0801115112000801116F000E0701CC
:1080180007012C6F080111510801116F000E0701AB
:1080280007010B6F080111510801116F000E0701BC
:108038000701296F080111510801116F000E07018E
:1080480007012B6F08011151070107019869070102
:108058009969120042EF40F0080159C8F6FF08017B
:108068005AC8F7FF000EF86E08000E01F5CF7EFE25
:1080780008010801594B5A2B7ECE61FF08010801FF
:108088005B07D8A05C0708015B29D8B45C29D8A491
:1080980050EF40F052EF40F030EF40F0120059C876
:1080A8005FF85AC860F864EF40F05FC8E9FF60C83D
:1080B800EAFF08015BC8EFFF080108015F4B602B6E
:1080C800080108015D07D8A05E0708015D29D8B43A
:1080D8005E29D8A472EF40F074EF40F059EF40F0F9
:1080E80076EF40F01200A1C768F8BEEC20F07D0ED4
:1080F80008010801685D000E08016959D8B087EFCA
:1081080040F089EF40F08BEF40F098EF40F065ECDD
:108118003FF0BB0E08010801536FFF0E0801546FB2
:10812800B6EC35F04DEC0EF012000AC8B4FE0BC8E0
:108138007EFE0CC87FFEF250C00B080108010D6FCF
:108148003F0EF2167ECEB6FE00F07FCEB7FE0801D7
:1081580008010D51F212B1EF40F00E010E018AB183
:10816800B8EF40F0BAEF40F0B1EF40F01200CBEFBB
:1081780040F0C0C8E9FFC1C8EAFFEF500E010E0188
:108188007E6F08010801C04BC12B7ECE61FF08013C
:108198000801C207D8A0C3070801C229D8B4C32957
:1081A800D8A4D9EF40F0DBEF40F0BDEF40F012006B
:1081B80007010701A229D8B4E4EF40F0E6EF40F048
:1081C800EDEF40F0A2C74CF8A3EC36F00701070129
:1081D800A2690801306F070E07010701A66F0801A1
:1081E80030510701089107010831010BFCEF40F0FD
:1081F80012000101000E04010401FF25E96EEA6A7C
:108208000101010EEA22EF50680AD8B40EEF41F0DE
:1082180010EF41F013EF41F0000E1CEF41F00401A4
:108228000401FF29070107012D6F010E1CEF41F022
:10823800120004010401DD6904010401DE6904017E
:108248000401DF6904010401E06904010401E16932
:1082580004010401E269000E04010401D96F000E53
:108268000401DA6F000E0401DB6F000E0401DC6FFD
:108278001200000E080108010D6545EF41F047EFB7
:1082880041F04AEF41F0000E5BEF41F00DC871F884
:108298001DEC2BF01750070AD8B455EF41F058EFF2
:1082A80041F0010E59EF41F0000E5BEF41F0120072
:1082B80037EC44F027EC20F02CC82DF874EC44F08F
:1082C80051EC43F00009D8A46CEF41F06EEF41F097
:1082D80072EF41F065EC3FF076EF41F037EC44F097
:1082E8004DEC0EF012000101000E04010401FF25FF
:1082F800E96EEA6A0101010EEA22EF50690AD8B470
:1083080088EF41F08BEF41F0010E8CEF41F0000E49
:108318008EEF41F01200070107010FB396EF41F00D
:1083280098EF41F0A6EF41F02EEC3CF0000E06016C
:108338000601CE6F000E0601CF6F07010701A36982
:1083480007010F831200F28A00F0F29AD6CFFAF1F1
:10835800D7CFFBF1EDC6FCF1EEC6FDF1EFC6FEF19D
:10836800F0C6FFF1F2B4BBEF41F0BDEF41F0A7EF6B
:1083780041F0F28A1200F28A00F0F29AD6CFFAF1AE
:10838800D7CFFBF1EDC6FCF1EEC6FDF1EFC6FEF16D
:10839800F0C6FFF1F2B4D3EF41F0D5EF41F0BFEFF3
:1083A80041F0F28A120008010D6F010E0701070162
:1083B8007E6F08010D51070107017B69BB68C4EC9A
:1083C80043F0A1C87FF7A2C880F7A3C881F7A4C863
:1083D80082F71200000E080108010D65F6EF41F062
:1083E800F8EF41F0FAEF41F003EF42F00DC871F8F1
:1083F8001DEC2BF018960DC82DF895EC12F0120014
:10840800F2A409EF42F00BEF42F019EF42F0010E2F
:1084180006010601ED27000E0601EE23000E0601F7
:10842800EF23000E0601F023F29412004428D8B47A
:1084380020EF42F022EF42F027EF42F044C04CF820
:10844800A3EC36F0446808010A6F000E0001000131
:10845800456F08010A51120057C859F858C85AF808
:108468003DEC37F059C85CF85AC85DF857C85AF857
:1084780058C85BF856C859F88CECE3F044EF42F062
:10848800120057C859F858C85AF83DEC37F059C87F
:108498005CF85AC85DF857C85AF858C85BF856C807
:1084A80059F883ECDEF059EF42F01200A7EC41F0E6
:1084B800FBC1A5F8FCC1A6F8FDC1A7F8FEC1A8F844
:1084C800A5C8A1F8A6C8A2F8A7C8A3F8A8C8A4F880
:1084D8006EEF42F01200948694883F0EC716000E85
:1084E800C66E000EC56EC686C78E82868288C68A0C
:1084F8000801096F430EC86E080109511200080EE1
:10850800080108014E2508010801796F000E0801CD
:1085180008014F2108017A6FF9EC42F04EC8D2F6F3
:108528004FC8D3F612000801226F010E0801080196
:10853800376F0801225139EC3FF0370EE96E080E0B
:10854800EA6EEF30E832010BAAEF42F012000001A8
:1085580000014567B2EF42F0B4EF42F0BEEF42F0DF
:108568000801386F010E00010001456F08013851FC
:10857800000146911200F90E080108014E25080174
:108588000801AC6F0A0E080108014F210801AD6F00
:108598000BEC44F04EC8FBF44FC8FCF412000AC8B8
:1085A80059F80BC85AF83DEC37F059C855F85AC86D
:1085B80056F80AC853F80BC854F8F9EC30F0E5EF50
:1085C80042F012000AC859F80BC85AF83DEC37F0C7
:1085D80059C855F85AC856F80AC853F80BC854F879
:1085E80053EC31F0F8EF42F0120006010601FA519F
:1085F800080108017925080108017B6F000E0801B0
:1086080008017A2108017C6F64EC3CF01200A1C7D4
:1086180068F8BEEC20F065EC3FF0680E0801080130
:10862800536FFF0E0801546FB6EC35F021EC44F09F
:1086380012000701070108A124EF43F026EF43F0D9
:1086480029EF43F0000E2EEF43F007010881010ED9
:108658002EEF43F01200BCC8BFF8BDC8C0F8C0C8B0
:10866800BEF8BFC8C0F8BEC8BFF8BFC8BCF8C0C80D
:10867800BDF83FEF43F0120032C838F833C839F874
:1086880067EC35F034C853F835C854F836C855F88F
:1086980037C856F866EC13F0120006010601E551DA
:1086A800030AD8B45AEF43F05DEF43F0010E5EEFD2
:1086B80043F0000E60EF43F0120006010601D751A7
:1086C800040AD8B46AEF43F06DEF43F0010E6EEF81
:1086D80043F0000E70EF43F012002EC834F82FC894
:1086E80035F830C836F831C837F82CC832F82DC8F4
:1086F80033F840EC43F01200000ED76E000ED66E31
:10870800F194F294F28A0801086F870ED56E080179
:10871800085112000E010E01DFAB95EF43F098EF00
:1087280043F0010E99EF43F0000E9BEF43F0120067
:1087380076927690769C769A768876967684A496C3
:108748007768A38697949388A586120030C838F86E
:1087580031C839F867EC35F032C853F833C854F8E3
:10876800B6EC35F0120026C82BF824C829F825C81D
:108778002AF822C827F823C828F84EEC17F0120068
:10878800A7EC41F0FAC1A1F8FBC1A2F8FCC1A3F81B
:10879800FDC1A4F8D0EF43F01200BFEC41F0FAC1DC
:1087A800DEF8FBC1DFF8FCC1E0F8FDC1E1F8DDEF60
:1087B80043F012000101000E08010801366F0101A3
:1087C800010E0801376FE9EF43F0120008010E6F40
:1087D800020E070107017E6F08010E510DC87BF7D5
:1087E80012002EC832F82FC833F82CC830F82DC81C
:1087F80031F8AAEC43F0120008010E6F020E0701CF
:108808000701876F08010E510DC884F71200E2CEE8
:10881800AEF8E3CEAFF8ACC8E2FEADC8E3FE15EFA4
:1088280044F01200C4EC43F0A1C8E9F6A2C8EAF685
:10883800A3C8EBF6A4C8ECF6120008012C6F680E6A
:1088480008010801646F08012C518FEC3FF01200F9
:10885800E0CEAEF8E1CEAFF8ACC8E0FEADC8E1FEC0
:1088680036EF44F0120008012D6F730E080108015D
:10887800646F08012D518FEC3FF012009792929887
:108888008998B19AB198A082A282B190120061CF62
:108898007EFE0E010E017E5152EF44F012000001DF
:1088A8004651010B58EF44F01200070107012E5101
:1088B8005EEF44F012007AEC44F0B1907684120036
:1088C800C0C87EFE7ECE61FF1200D08EF28EF28C82
:1088D8001200769471EC44F012008E828E9412008D
:1088E8002DC87DF7120056C886F712008E928E8426
:0888F8001200BCEC09F01200B3
:10FE16002F7365727665722F61737369676E3F65BE
:10FE26006D6265646465643D312670726F746F63DC
:10FE36006F6C56657273696F6E3D32266D61633DF8
:10FE46000048415052414455395055535445575531
:10FE56003355334136484550415145465245504544
:10FE6600500000005E01E8036700535741513854C3
:10FE76004845433245424139484546454A3552553B
:10FE860053544548455939323754000D0A436F6E6D
:10FE96006E656374696F6E3A20636C6F73650D0AE5
:10FEA6000D0A0020485454502F312E300D0A486F49
:10FEB60073743A200073656C666C6561726E696E68
:10FEC6006776320054656C6C537469636B4E657467
:10FED6003A0054656C6C537469636B204E6574000C
:10FEE60073656C666C6561726E696E6700657665D2
:10FEF60072666C6F7572697368007265676C697398
:10FF060074656E657200646973636F6E6E656374A3
:10FF16000066696E656F666673657400636F646517
:10FF26007377697463680070726F746F636F6C00C7
:10FF36005265676973746572006D616E646F6C7982
:10FF46006E0076657273696F6E00676174657761BE
:10FF5600790061726374656368006E65746D6173C0
:10FF66006B0052617744617461006F7265676F6EF2
:10FF760000736176656970007365637265740073FA
:10FF8600656E736F72006D6574686F6400636C6193
:10FF9600737300686F7573650073657469700068C4
:10FFA60061737461006D6F64656C006461746100F7
:10FFB60073656E640050696E6700686173680064FB
:10FFC6006E7331007368613100756E697400646E1A
:10FFD60073320047455420006D61630032383A00A1
:10FFE6006B65790041434B00783130003137006F43
:0AFFF6007300520050005300000099
:020000040001F9
:1000000074656D706572617475726568756D69642B
:10001000697479006170692E74656C6C6475732EF7
:10002000636F6D000000010000000000000000018F
:100030000000000000009E9FFE4101000000FFFF45
:10004000F3FFFFFFFF80FFFFFEFEFFFEFFFFFEFF4F
:1000500007000D0E080108014A25E96E000E08018F
:1000600008014B21EA6EEF50080108014F6F080E9E
:10007000080108014A25E96E000E080108014B211C
:10008000EA6E0801EECF66F80801EECF67F80801C6
:10009000EECF68F80801EECF69F8040E08010801F8
:1000A0004A25E96E000E080108014B21EA6E08019D
:1000B000EECF5AF80801EECF5BF80801EECF5CF8FE
:1000C0000801EECF5DF81890189218940B000E00FE
:1000D00018B86DEF80F06FEF80F085EF80F0C4EC22
:1000E00043F0740E08010801A1250F6E350E0801BA
:1000F0000801A221106E060E08010801A321116E4D
:10010000000E08010801A421126EDDEF81F0080144
:1001100008014FA58EEF80F090EF80F094EF80F013
:100120006CEC33F0D6EF8DF0080108014FA99BEF7E
:1001300080F09DEF80F0BBEF80F066C821F067C8CB
:1001400022F068C823F069C824F008016A6F000E25
:1001500008010801736F08016A5108016B6F040EF2
:1001600008010801726F08016B519FECA1F06CEC63
:1001700033F0D6EF8DF0080108014FA3C2EF80F0F5
:10018000C4EF80F0F8EF80F0010E080108015A2555
:10019000256E000E080108015B21266E000E080185
:1001A00008015C21276E000E080108015D21286E00
:1001B000B4EC04F072C840F073C841F008016A6FF3
:1001C000010E08010801736F08016A5108016B6F85
:1001D000120E08010801726F08016B519FECA1F02B
:1001E00008016A6F060E176E08016A51FAEF80F077
:1001F0006CEC33F0D6EF8DF0080108014FA503EF4A
:1002000081F005EF81F007EF81F0D6EF8DF0080166
:1002100008014FA90EEF81F010EF81F056EF81F049
:1002200008010801695124180EE10801080168510C
:10023000231809E1080108016751221804E10801A7
:10024000080166512118D8B428EF81F02AEF81F017
:1002500056EF81F021C05AF822C05BF823C05CF849
:1002600024C05DF866C821F067C822F068C823F092
:1002700069C824F008016A6F010E08010801736F54
:1002800008016A5108016B6F040E08010801726FC2
:1002900008016B519FECA1F05AC821F05BC822F015
:1002A0005CC823F05DC824F0D6EF8DF0080108018A
:1002B0004FA35DEF81F05FEF81F0D9EF81F0010E88
:1002C000080108015A25256E000E080108015B216E
:1002D000266E000E080108015C21276E000E080141
:1002E00008015D21286E0E0E080108014A25E96EFD
:1002F000000E080108014B21EA6EEECF2FF0EDCF82
:1003000030F0B4EC04F072C840F073C841F008015A
:1003100008014FA98EEF81F090EF81F0C1EF81F0DD
:1003200008016A6F010E08010801736F08016A5124
:1003300008016B6F100E08010801726F08016B5104
:100340009FECA1F008016A6F070E176E08016A5151
:10035000C4EC43F0740E08010801A1250F6E350EA0
:1003600008010801A221106E060E08010801A32150
:10037000116E000E08010801A421126E1898D9EF21
:1003800081F008016A6F010E08010801736F08010E
:100390006A5108016B6F120E08010801726F0801A3
:1003A0006B519FECA1F008016A6F060E176E0801F1
:1003B0006A51D6EF8DF0E6EF81F01750040A01E1A3
:1003C000A6D6010A01E118D7DBEF81F04CC854F83A
:1003D0004DC855F8080108014FA1F1EF81F0F3EF86
:1003E00081F0F7EF81F008010801544B552B08010B
:1003F00008014FA3FEEF81F000EF82F004EF82F0DE
:1004000008010801544B552B00EE0DF010EE0BF0D7
:10041000E652EE52ED50E55C02E1EF50E75CD8A009
:1004200014EF82F016EF82F03DEF82F000EE0BF059
:10043000EECF6AF8EDCF6BF80D5008016A5F0E50F1
:1004400008016B5B00EE05F0EECF6CF8EDCF6DF8B8
:10045000035008016C5F045008016D5B08016A518C
:1004600008016C5D08010801526F08016B51080119
:100470006D590801536F54EF82F000EE0DF0EECF8E
:100480006AF8EDCF6BF80B5008016A5F0C50080159
:100490006B5BFF0E08016A2508010801526FFF0E11
:1004A00008016B210801536F2550080108015A5DAE
:1004B00008010801626F2650080108015B59080114
:1004C000636F2750080108015C590801646F2850C8
:1004D000080108015D590801656F62C856F863C8D4
:1004E00057F808016A6F000E080108014E6F0801F5
:1004F0006A510801080155515411D8B482EF82F0B5
:1005000084EF82F094EF83F00801080153515211F7
:10051000D8B48DEF82F08FEF82F092EF83F0080174
:10052000080165BF96EF82F098EF82F0CBEF82F082
:1005300008010801525108016A6F0801080153516E
:1005400008016B6F08016C6B08016D6B08016A5143
:1005500008010801625D08016B5108010801635937
:1005600008016C5108010801645908016D51080126
:1005700008016559D8B0BFEF82F0C1EF82F0CBEF30
:1005800082F008016A6F010E080108014E6F080130
:100590006A513DEF83F00801080154510801080138
:1005A000622508016A6F0801080155510801080118
:1005B000632108016B6F000E080108016421080126
:1005C0006C6F000E08010801652108016D6F0801BC
:1005D0006D51800A800F08E1000E6C5D05E1000E90
:1005E0006B5D02E1010E6A5DD8A0F9EF82F0FBEFCE
:1005F00082F03DEF83F00801080154510801080121
:10060000525D08016A6F080108015551080108018F
:10061000535908016B6F08016C6B08016BBF6C07C5
:1006200008016C5108016D6F08016D51800A0801C5
:100630006E6F08010801625108016A5D0801080136
:10064000635108016B5908010801645108016C5994
:10065000080108016551800A08016E59D8A033EFDE
:1006600083F035EF83F03DEF83F008016A6F010EF0
:10067000080108014E6F08016A5108010801525132
:1006800008016A6F08010801535108016B6F0801E6
:100690006C6B08016D6B080108016551800A080147
:1006A0006E6F08016A5108010801625D08016B5113
:1006B00008010801635908016C51080108016459D7
:1006C00008016D51800A08016E59D8B06AEF83F0B5
:1006D0006CEF83F092EF83F0080156C86AF80801C6
:1006E00057C86BF808010801545108016A2708012E
:1006F0000801555108016B2308016B51800A800FD6
:10070000010ED8B46A5DD8A088EF83F08AEF83F039
:1007100092EF83F008016A6F010E080108014E6F25
:1007200008016A51E4EF83F0080165516211631119
:100730006411D8A49EEF83F0A0EF83F0AAEF83F0BA
:1007400008016A6F010E080108014E6F08016A5125
:10075000E4EF83F00801080165BFB1EF83F0B3EF68
:1007600083F0E4EF83F008010801525108016A6F39
:1007700008010801535108016B6F08016C6B0801F7
:100780006D6B08016A5108010801625D08016B5137
:1007900008010801635908016C51080108016459F6
:1007A00008016D51080108016559D8B0DAEF83F0EE
:1007B000DCEF83F0E4EF83F008016A6F010E0801BB
:1007C00008014E6F08016A51080108014E67EBEFFE
:1007D00083F0EDEF83F00AEF84F0080108014FB5D4
:1007E000F4EF83F0F6EF83F008EF84F008016A6F0E
:1007F000010E08010801736F08016A5108016B6F4F
:10080000100E08010801726F08016B519FECA1F0F6
:10081000D6EF8DF0080108014F51060BD8B413EF45
:1008200084F015EF84F019EF84F06CEC33F0D6EF20
:100830008DF0080108014FB920EF84F022EF84F019
:1008400024EF84F0D6EF8DF04DEF88F00801080119
:10085000695124180EE1080108016851231809E1C3
:10086000080108016751221804E1080108016651D6
:100870002118D8B43EEF84F040EF84F06CEF84F0A0
:1008800021C05AF822C05BF823C05CF824C05DF890
:1008900066C821F067C822F068C823F069C824F050
:1008A00008016A6F010E08010801736F08016A519F
:1008B00008016B6F040E08010801726F08016B518B
:1008C0009FECA1F05AC821F05BC822F05CC823F06D
:1008D0005DC824F0D6EF8DF008016A6F070E176E21
:1008E00008016A512950075C08010801586F2A5015
:1008F00008580801596F0801080159AF82EF84F0C8
:1009000084EF84F09AEF84F000EE03F0EECF6AF803
:10091000EDCF6BF8015008016A5F025008016B5B74
:1009200008016A5108010801582708016B510801A4
:100930000801592308010801585121240801080120
:100940005E6F080108015951222008015F6F000EF7
:1009500023200801606F000E24200801616F080148
:1009600008016651080108015E5D08016A6F08010F
:1009700008016751080108015F5908016B6F080100
:100980000801685108010801605908016C6F0801ED
:100990000801695108010801615908016D6F0801DA
:1009A0006DAFD5EF84F0D7EF84F0EBEF84F0080162
:1009B0006A6F000E08010801736F08016A5108018F
:1009C0006B6F100E08010801726F08016B519FECEC
:1009D000A1F0D6EF8DF00950295C08016A6F0A502A
:1009E0002A5808016B6F08016C6B08016BBF6C071C
:1009F00008016C5108016D6F08016A51215C080102
:100A000008015E6F08016B51225808015F6F0801F1
:100A10006C5123580801606F08016D51245808017A
:100A2000616F00EE09F010EE29F0E652EE52ED5043
:100A3000E55C02E1EF50E75CD8B021EF85F023EFF1
:100A400085F043EF85F00150035C08016A6F0250A6
:100A5000045808016B6F08016C6B08016D6B08018D
:100A60006A51080108015E5F08016B510801080125
:100A70005F5B08016C5108010801605B08016D5162
:100A800008010801615B080108015E5108010801C5
:100A9000665D080108015E6F080108015F510801E9
:100AA0000801675908015F6F0801080160510801DA
:100AB000080168590801606F0801080161510801C7
:100AC000080169590801616F080108016151800A34
:100AD000800F0BE1000E0801605D07E1000E0801C8
:100AE0005F5D03E1010E08015E5DD8A07AEF85F03D
:100AF0007CEF85F07DEF86F00150035C08016A6FA2
:100B00000250045808016B6F08016C6B08016D6B93
:100B1000080108015E5108016A5D080108015F5182
:100B200008016B5908010801605108016C5908015E
:100B30000801615108016D59D8A0A1EF85F0A3EF1C
:100B400085F07DEF86F03F963F98199009C058F8E0
:100B50000AC059F8080108015E5109260801080178
:100B60005F510A22080108015851295C0801080157
:100B700059512A58D8A0BFEF85F0C1EF85F0EFEFAB
:100B800085F000EE09F010EE29F0E652EE52ED503D
:100B9000E55C02E1EF50E75CD8B0D1EF85F0D3EF30
:100BA00085F0EDEF85F000EE09F0EECF6AF8EDCFBD
:100BB0006BF8295008016A5F2A5008016B5B080135
:100BC0006A51212608016B512222000E2322000EB9
:100BD000242209C029F00AC02AF033EF86F000EE83
:100BE00003F0EECF6AF8EDCF6BF8015008016A5FB1
:100BF000025008016B5B295008016A2508010801B1
:100C0000586F2A5008016B210801596F09500801DB
:100C10000801585D0A50080108015959D8B013EF6E
:100C200086F015EF86F033EF86F000EE09F0EECF98
:100C30006AF8EDCF6BF808010801585108016A5FA6
:100C400008010801595108016B5B08016A5121260E
:100C500008016B512222000E2322000E242209C01B
:100C600029F00AC02AF000EE03F010EE09F0E65277
:100C7000EE52ED50E55C02E1EF50E75CD8A043EFA7
:100C800086F045EF86F057EF86F000EE03F0EECFEA
:100C90006AF8EDCF6BF8015008016A5F0250080155
:100CA0006B5B08016A51095E08016B510A5A00EE3C
:100CB00003F010EE29F0E652EE52ED50E55C02E151
:100CC000EF50E75CD8A067EF86F069EF86F07BEF26
:100CD00086F000EE03F0EECF6AF8EDCF6BF801502E
:100CE00008016A5F025008016B5B08016A51295EC6
:100CF00008016B512A5AF1EF86F000EE29F010EE50
:100D000009F0E652EE52ED50E518EFCFE8FFD8B407
:100D1000E718D8B48EEF86F090EF86F0F1EF86F00A
:100D20003FA695EF86F097EF86F0F0EF86F03FA8AC
:100D30009CEF86F09EEF86F0EFEF86F00950295C7D
:100D400008016A6F0A502A5808016B6F08016C6B22
:100D500008016BBF6C0708016C5108016D6F080139
:100D60006A51215E08016B51225A08016C51235AC5
:100D700008016D51245A00EE09F010EE29F0E652F8
:100D8000EE52ED50E55C02E1EF50E75CD8B0CBEFFE
:100D900086F0CDEF86F0EAEF86F00150035C0801A3
:100DA0006A6F0250045808016B6F08016C6B0801F0
:100DB0006BBF6C0708016C5108016D6F08016A5127
:100DC000215E08016B51225A08016C51235A080117
:100DD0006D51245A09C029F00AC02AF019843F88AD
:100DE0003F8600EE07F010EE09F0E652EE52ED50AD
:100DF000E518EFCFE8FFD8B4E718D8A402EF87F0E2
:100E000004EF87F047EF87F019B609EF87F00BEF93
:100E100087F024EF87F0C4EC43F0740E080108015A
:100E2000A1250F6E350E08010801A221106E060ED5
:100E300008010801A321116E000E08010801A42178
:100E4000126E189847EF87F00801080169512418BD
:100E50000EE1080108016851231809E108010801A1
:100E60006751221804E10801080166512118D8A42D
:100E70003CEF87F03EEF87F047EF87F03FA043EF6E
:100E800087F045EF87F047EF87F01898199600EE46
:100E900021F0EECF6AF8EDCF6BF80801080166513A
:100EA00008016A5F08010801675108016B5B0E0EBB
:100EB000080108014A25E96E000E080108014B21CE
:100EC000EA6EEECF6CF8EDCF6DF808016A510801BB
:100ED0006C5D08010801506F08016B5108016D59E4
:100EE0000801516F30502F10D8A479EF87F07BEFB5
:100EF00087F087EF87F00801080151515011D8B4ED
:100F000084EF87F086EF87F087EF87F0198250C86B
:100F10002FF051C830F01750080AD8A492EF87F08C
:100F200094EF87F0D4EF87F0080108016951241885
:100F30000EE1080108016851231809E108010801C0
:100F40006751221804E10801080166512118D8A44C
:100F5000ACEF87F0AEEF87F0D2EF87F03FA0B3EFB2
:100F600087F0B5EF87F0D2EF87F0C4EC43F0BA0E0C
:100F700008010801A1250F6E1A0E08010801A2211F
:100F8000106E030E08010801A321116E000E080166
:100F90000801A421126E188808016A6F090E176EE5
:100FA00008016A512DEF88F01750090AD8A4DBEF29
:100FB00087F0DDEF87F006EF88F0080108014FB1F8
:100FC000E4EF87F0E6EF87F004EF88F066C821F0E1
:100FD00067C822F068C823F069C824F008016A6F66
:100FE000000E08010801736F08016A5108016B6F58
:100FF000140E08010801726F08016B519FECA1F0FB
:101000006CEC33F0D6EF8DF02DEF88F017500A0A14
:10101000D8A40DEF88F00FEF88F02DEF88F00801CD
:101020000801695124180EE10801080168512318CC
:1010300009E1080108016751221804E108010801CB
:1010400066512118D8A427EF88F029EF88F02BEFFC
:1010500088F06CEC33F0D6EF8DF065EF88F0080186
:101060000801695124180EE108010801685123188C
:1010700009E1080108016751221804E1080108018B
:1010800066512118D8A447EF88F049EF88F04BEF5C
:1010900088F06CEC33F0D6EF8DF01750060A02E1C1
:1010A00026EF84F0010A01E11DD40F0A01E11AD4F0
:1010B000010A01E117D4030A01E114D4010A01E194
:1010C00011D4070ACCE02DEF88F0080108014FABDE
:1010D0006CEF88F06EEF88F070EF88F0D6EF8DF04F
:1010E00017500B0AD8A477EF88F079EF88F07BEFE0
:1010F00088F0D6EF8DF017500A0AD8A482EF88F056
:1011000084EF88F086EF88F0D6EF8DF017500C0A48
:10111000D8A48DEF88F08FEF88F091EF88F0D6EFAC
:101120008DF0080108014D514C11D8B49AEF88F0A8
:101130009CEF88F09AEF8CF0080108015751800A63
:10114000800F010ED8B4565DD8B0A9EF88F0ABEF90
:1011500088F032EF8AF00C0E080108014A25E96E8A
:10116000000E080108014B21EA6EEF380F0B080151
:101170006A6F6AC86BF808016C6BD89008016B370E
:101180006C37D89008016B376C370801080156514D
:1011900008016B5D08010801796F080108015751CA
:1011A00008016C5908017A6FF9EC42F00801080156
:1011B0005651080108014C27080108015751080140
:1011C00008014D23080108014C5108010801525D36
:1011D000080108014D51080108015359D8B0F3EF37
:1011E00088F0F5EF88F0F9EF88F052C84CF853C852
:1011F0004DF8080108014C512526080108014D5100
:101200002622000E2722000E282200EE0BF0EECF41
:101210006AF8EDCF6BF8080108014C5108016A2704
:10122000080108014D5108016B2308016A51055C52
:1012300008016B510658D8B020EF89F022EF89F0F1
:1012400096EF89F000EE05F0EECF6AF8EDCF6BF87F
:101250000B5008016A5F0C5008016B5B010E08011E
:101260006A2508010801586F000E08016B2108016A
:10127000596F58C8AAF859C8ABF808016A6F000E30
:1012800008010801A96F08016A51FF0E0801080151
:10129000A76FFF0E0801A86F1CC0A6F80BC0A4F82A
:1012A0000CC0A5F8A0EC23F0080108015851080172
:1012B00008014C5D08010801AA6F08010801595195
:1012C000080108014D590801AB6F08016A6F000E53
:1012D00008010801A96F08016A51FF0E0801080101
:1012E000A76FFF0E0801A86F1CC0A6F803C0A4F8E2
:1012F00004C0A5F8A0EC23F008014CC86AF8080166
:101300004DC86BF808010801585108016A5F0801CF
:101310000801595108016B5B035008016A250B6EE7
:10132000045008016B210C6EB9EF89F04CC8AAF883
:101330004DC8ABF808016A6F000E08010801A96FDB
:1013400008016A51FF0E08010801A76FFF0E08018E
:10135000A86F1CC0A6F80BC0A4F80CC0A5F8A0ECA0
:1013600023F0080108014C510B26080108014D51DA
:101370000C223D28D8B43E28D8B4C1EF89F0C3EF81
:1013800089F030EF8AF0080108014C513D5E0801F8
:1013900008014D513E5A3D50312408010801586F53
:1013A0003E5032200801596F0801080159AFDBEFA8
:1013B00089F0DDEF89F0E1EF89F03D683E6830EFBC
:1013C0008AF000EE3DF0EE52ED50800A800F010EE3
:1013D000D8B4EF5CD8B0EFEF89F0F1EF89F030EFDF
:1013E0008AF00801080158512526080108015951C1
:1013F0002622000E2722000E28220801080158513B
:101400000B260801080159510C2200EE0BF010EEDA
:1014100005F0E652EE52ED50E55C02E1EF50E75C7C
:10142000D8B015EF8AF017EF8AF02EEF8AF000EEB1
:1014300005F0EECF6AF8EDCF6BF8035008016A5F54
:10144000045008016B5B010E08016A27000E6B2334
:1014500008016A510B5E08016B510C5A3D683E68E9
:101460009AEF8CF0080108015751800A800F010E95
:10147000D8B4565DD8A03FEF8AF041EF8AF09AEFDA
:101480008CF008014CC86AF808014DC86BF80801D7
:101490000801565108016A2708010801575108013F
:1014A0006B2308016A5108010801525D08016B5164
:1014B000080108015359D8B060EF8AF062EF8AF052
:1014C00073EF8AF008010801565108010801525DC6
:1014D000080108014C6F0801080157510801080173
:1014E000535908014D6F0C0E080108014A25E96E99
:1014F000000E080108014B21EA6EEF380F0B0801BE
:101500006A6F6AC86BF808016C6BD89008016B377A
:101510006C37D89008016B376C376BC879F86CC89A
:101520007AF8F9EC42F000EE0BF0EECF6AF8EDCF6E
:101530006BF808010801565108016A2708010801E3
:10154000575108016B23080108014C5108016A2713
:10155000080108014D5108016B2308016A51055C1F
:1015600008016B510658D8B0B8EF8AF0BAEF8AF08C
:101570007DEF8BF000EE05F0EECF6AF8EDCF6BF863
:101580000B5008016A5F0C5008016B5B010E0801EB
:101590006A27000E6B2308010801565108016A5D95
:1015A00008010801586F08010801575108016B59DB
:1015B0000801596F0801080159BFE1EF8AF0E3EF14
:1015C0008AF031EF8BF058C8AAF859C8ABF8080177
:1015D0006A6F000E08010801A96F08016A51FF0E29
:1015E00008010801A76FFF0E0801A86F1CC0A6F82C
:1015F0000801080156510B2408010801A46F0801D5
:10160000080157510C200801A56FA0EC23F0080138
:1016100008015851080108014C5D08010801AA6F32
:10162000080108015951080108014D590801AB6F23
:1016300008016A6F000E08010801A96F08016A51CC
:10164000FF0E08010801A76FFF0E0801A86F1CC05C
:10165000A6F803C0A4F804C0A5F8A0EC23F07BEF23
:101660008BF04CC8AAF84DC8ABF808016A6F000EA1
:1016700008010801A96F08016A51FF0E080108015D
:10168000A76FFF0E0801A86F1CC0A6F800EE05F0BA
:10169000EECF6BF8EDCF6CF8035008016B5F045090
:1016A00008016C5B00EE0BF0EECF6DF8EDCF6EF83D
:1016B00008010801565108016D270801080157511A
:1016C00008016E2308016B5108016D5D08016F6F01
:1016D00008016C5108016E590801706FFF0E080176
:1016E0006F2508010801A46FFF0E08017021080191
:1016F000A56FA0EC23F0A1EF8BF04CC8AAF84DC861
:10170000ABF808016A6F000E08010801A96F080113
:101710006A51FF0E08010801A76FFF0E0801A86FAC
:101720001CC0A6F80801080156510B240801080145
:10173000A46F0801080157510C200801A56FA0EC07
:1017400023F03D28D8B43E28D8A4A9EF8BF0ABEF06
:101750008BF0B5EF8BF056C83DF057C83EF04CC843
:1017600031F04DC832F09AEF8CF03D50080108017D
:10177000565D3E50080108015759D8B0C2EF8BF0B2
:10178000C4EF8BF030EF8CF0080156C86AF80801FE
:1017900057C86BF8080108014C5108016A27080175
:1017A00008014D5108016B2300EE3DF0EECF6CF8BF
:1017B000EDCF6DF8315008016C27325008016D23D0
:1017C00008016A5108016C5D08016B5108016D59EF
:1017D000D8A0EDEF8BF0EFEF8BF00CEF8CF0080161
:1017E00056C86AF8080157C86BF8080108014C513F
:1017F00008016A27080108014D5108016B233D507B
:1018000008016A5D3E5008016B59D8B00AEF8CF0B0
:101810000CEF8CF012EF8CF04CC831F04DC832F068
:101820002AEF8CF000EE3DF0EECF6AF8EDCF6BF8CA
:10183000315008016A27325008016B230801080162
:10184000565108016A5D316E0801080157510801BF
:101850006B59326E56C83DF057C83EF09AEF8CF087
:10186000080156C86AF8080157C86BF80801080152
:101870004C5108016A27080108014D5108016B23EA
:1018800000EE3DF0EECF6CF8EDCF6DF83150080171
:101890006C27325008016D2308016A5108016C5D04
:1018A00008016B5108016D59D8B059EF8CF05BEF0E
:1018B0008CF09AEF8CF000EE3DF0EECF6AF8EDCFB1
:1018C0006BF8315008016A27325008016B23080178
:1018D0000801565108016A5D0801080157510801C5
:1018E0006B59D8A076EF8CF078EF8CF09AEF8CF0F3
:1018F000080156C86AF8080157C86BF808010801C2
:101900004C5108016A27080108014D5108016B2359
:101910003D5008016A5F3E5008016B5B3150080181
:101920006A5F325008016B5B08016A513126080179
:101930006B5132220801080155515411D8B4A3EF5C
:101940008CF0A5EF8CF0E4EF8CF01750070AD8B4B8
:10195000ACEF8CF0AEEF8CF0B2EF8CF00BC00DF072
:101960000CC00EF018AEB7EF8CF0B9EF8CF0CFEFE3
:101970008CF008016A6F010E08010801736F0801FD
:101980006A5108016B6F100E08010801726F08019F
:101990006B519FECA1F0B7EC24F0E4EF8CF0188EC3
:1019A00018BCD5EF8CF0D7EF8CF0E4EF8CF0188CEE
:1019B0005AEC42F00F0E08010801A125156E000E29
:1019C00008010801A221166E080108014FA1EBEFE2
:1019D0008CF0EDEF8CF0D6EF8DF00801080154513A
:1019E000080108015A2508016A6F080108015551CC
:1019F000080108015B2108016B6F000E0801080156
:101A00005C2108016C6F000E080108015D210801CE
:101A10006D6F010E252408016E6F000E262008014F
:101A20006F6F000E27200801706F000E282008013C
:101A3000716F08016D51080171190EE108016C51B7
:101A40000801701909E108016B5108016F1904E1DF
:101A500008016A5108016E19D8A431EF8DF033EFF7
:101A60008DF0D6EF8DF0010E2526000E2622000EF9
:101A70002722000E2822B9EF8DF008016A6F0C0EA4
:101A8000176E08016A5108016A6F010E080108010A
:101A9000736F08016A5108016B6F110E080108018C
:101AA000726F08016B519FECA1F0D6EF8DF0080129
:101AB0006A6F0B0E176E08016A515AEC42F01F0E46
:101AC00008010801A125156E000E08010801A221D8
:101AD000166EC4EF8DF008010801695124180EE15B
:101AE000080108016851231809E10801080167513C
:101AF000221804E10801080166512118D8A483EFD7
:101B00008DF085EF8DF09BEF8DF008016A6F000E70
:101B100008010801736F08016A5108016B6F100E0C
:101B200008010801726F08016B519FECA1F06CEC89
:101B300033F0D6EF8DF008016A6F0A0E176E0801B8
:101B40006A51C4EF8DF008016A6F000E08010801A8
:101B5000736F08016A5108016B6F100E08010801CC
:101B6000726F08016B519FECA1F06CEC33F0D6EF73
:101B70008DF01750060A81E0010A99E00F0AABE0E8
:101B8000010AE1E0A1EF8DF008016A6F010E080182
:101B90000801736F08016A5108016B6F100E08018C
:101BA0000801726F08016B519FECA1F0120008014F
:101BB000276F000E080108011E6F08012751000E53
:101BC000080108011E65E7EF8DF0E9EF8DF0EBEFFE
:101BD0008DF0F6EF93F01EC871F81DEC2BF00801A4
:101BE000276F000E08010801206F08012751080126
:101BF000276F000E080108011F6F08012751080117
:101C0000276F000E080108011D6F0801275119B246
:101C10000CEF8EF00EEF8EF015EF8EF019A413EF8F
:101C20008EF015EF8EF02DEF8EF0CBEC3DF000092D
:101C3000D8B41DEF8EF01FEF8EF02DEF8EF008015F
:101C4000276F100E08010801206F08012751000EB0
:101C500019B4010E080108011F6F18AA32EF8EF0A7
:101C600034EF8EF058EF8EF05AEC42F00801080184
:101C7000A151135C0801276F08010801A2511458F3
:101C80000801286F08012851800A800F010ED8B47E
:101C9000275DD8B04EEF8EF050EF8EF058EF8EF0FB
:101CA0000801276F100E08010801206F0801275155
:101CB00018AC5DEF8EF05FEF8EF083EF8EF05AEC94
:101CC00042F008010801A151155C0801276F0801C5
:101CD0000801A25116580801286F08012851800AEE
:101CE000800F010ED8B4275DD8B079EF8EF07BEF6E
:101CF0008EF083EF8EF00801276F100E08010801A7
:101D0000206F0801275117500B0AD8A48AEF8EF0D4
:101D10008CEF8EF0B6EF8EF05AEC42F0080108011D
:101D2000A151155C0801276F08010801A25116583E
:101D30000801286F08012851800A800F010ED8B4CD
:101D4000275DD8B0A6EF8EF0A8EF8EF0B6EF8EF03C
:101D50000801276F110E08010801206F08012751A3
:101D60000801276F0C0E176E080127511750040A3F
:101D7000D8A4BDEF8EF0BFEF8EF018EF90F0000EFC
:101D800008010801216F000E0801226F030E0801EF
:101D90000801215D000E08012259D8A0D2EF8EF073
:101DA000D4EF8EF0D6EF8EF018EF90F00801080116
:101DB0002151140DF3CF27F8100E08012727000139
:101DC0009F0E08012725E96EEA6A0001000EEA224B
:101DD000EE50ED10D8A4EFEF8EF0F1EF8EF0F3EFB0
:101DE0008EF018EF90F000EE1AF008010801215172
:101DF000140DF3CF27F8100E0801272700019F0EBE
:101E000008012725E16EE26A0001000EE222E65297
:101E1000EE52ED50E518EFCFE8FFD8B4E718D8A49C
:101E200014EF8FF016EF8FF006EF90F0B7EC24F080
:101E30000A0E08010801B06F000E0801B16F080119
:101E400008012151140D9F0E0801276F000E286F05
:101E5000F35008012727E86AF3BEE8680801282341
:101E600027C8AEF828C8AFF8330E08010801AC6FD8
:101E7000000E0801AD6F58EC3AF00801080121513D
:101E8000140DF3CF27F80A0E0801272700019F0E33
:101E900008012725E96EEA6A0001000EEA22EECF6A
:101EA0002BF0EDCF2CF0080108012151140DF3CFD8
:101EB00027F80C0E0801272700019F0E080127258F
:101EC000E96EEA6A0001000EEA22EECF28F8EECFB2
:101ED00029F8EECF2AF8EECF2BF8010E08012825BD
:101EE000256E000E08012921266E000E08012A2108
:101EF000276E000E08012B21286E00EE35F0EECF84
:101F000027F8EDCF28F8335008012727345008016F
:101F100028232B50080127272C50080128232D5057
:101F2000080127191A6E2E50080128191B6E080186
:101F3000276F120E08010801206F080127510801C0
:101F4000276F060E176E08012751140E08010801AD
:101F5000626F000E0801636F080108012151020839
:101F600008010801606F080108012251D8A0E82A81
:101F700000080801616F83EC3BF060C8AAF861C8F3
:101F8000ABF80801276F010E08010801A96F0801CD
:101F90002751080108012129140D9F0E0801286FFF
:101FA000000E296FF35008012827E86AF3BEE8689D
:101FB0000801292328C8A7F829C8A8F808012A6F0A
:101FC000010E08010801A66F08012A510801080145
:101FD0002151140D9F0E08012B6F000E2C6FF35032
:101FE00008012B27E86AF3BEE86808012C232BC8F8
:101FF000A4F82CC8A5F8A0EC23F0000E0001000105
:10200000D76F000E0001D86F18EF90F0080108019B
:10201000214B222B030E08010801215D000E08014F
:102020002259D8A016EF90F018EF90F0D6EF8EF06E
:10203000080108012051D8B420EF90F022EF90F071
:1020400035EF90F0080108011F51D8B42AEF90F045
:102050002DEF90F0010E2EEF90F0000E0801080118
:10206000736F20C872F89FECA1F018B83AEF90F0A7
:102070003CEF90F0BEEF90F01750070AD8A443EF62
:1020800090F045EF90F090EF90F0C4EC43F00F50DB
:1020900008010801A15D0801276F1050080108011F
:1020A000A2590801286F115008010801A35908011D
:1020B000296F125008010801A45908012A6F08016C
:1020C0002AAF65EF90F067EF90F069EF90F0E9EFDD
:1020D00093F01850070B060AD8A471EF90F073EF35
:1020E00090F092EF90F0000E18B6010E0801080172
:1020F000206F1EC82DF895EC12F01EC82DF895EC37
:1021000012F008010801206788EF90F08AEF90F044
:1021100090EF90F00801276F0E0E176E08012751FF
:10212000E9EF93F0B7EC24F00801276F020E0801E5
:102130000801736F080127510801286F100E08016C
:102140000801726F080128519FECA1F0C4EC43F024
:10215000740E08010801A1250F6E350E0801080153
:10216000A221106E060E08010801A321116E000EB7
:1021700008010801A421126EE9EF93F0C4EC43F0CA
:102180000F5008010801A15D0801276F10500801D8
:102190000801A2590801286F115008010801A3592C
:1021A0000801296F125008010801A45908012A6F7B
:1021B00008012AAFDEEF90F0E0EF90F0E2EF90F050
:1021C000E9EF93F0B7EC24F02DEF93F01DEC43F022
:1021D0000009D8B4EEEF90F0F0EF90F01BEF91F023
:1021E0000801276F010E176E080127513FA4FBEF6E
:1021F00090F0FDEF90F00DEF91F00801276F010EC8
:10220000080108012F6F0801275133C02DF834C091
:102210002EF848EC3BF01BEF91F00801276F010E00
:10222000080108012F6F0801275133C02DF834C071
:102230002EF80DEC3BF052EF93F00801230E08014D
:1022400008012D6F0801080E08012E6FD3EC94F0E1
:102250000009D8B42EEF91F030EF91F01BEF91F020
:10226000DCEC40F00009D8B438EF91F03AEF91F08F
:1022700072EF91F023C833F024C834F025C835F04C
:1022800026C836F00801276F020E176E0801275185
:1022900000EE35F0EECF27F8EDCF28F833500801E7
:1022A00027273450080128232B50080127272C50BA
:1022B000080128232D50080127191A6E2E500801F5
:1022C00028191B6E0801276F000E426E0801275166
:1022D000270E1D6E000E1E6E000E1F6E000E206E6D
:1022E0008EEF91F0C4EC43F0740E08010801A125B3
:1022F0000F6E350E08010801A221106E060E0801AE
:102300000801A321116E000E08010801A421126E1C
:102310000801276F000E176E0801275152EF93F046
:102320005AEC42F0A1C813F0A2C814F0330E080111
:1023300008014C6F000E08014D6F0EEC23F00801F0
:10234000276F030E176E0801275152EF93F0370ED7
:10235000080108014E6F000E08014F6F330E08018F
:1023600008014C6F000E08014D6FE7EC1AF00009F0
:10237000D8A4BDEF91F0BFEF91F0EEEF91F05AECE1
:1023800042F0135008010801A15F14500801080130
:10239000A25B08010801A1511D5C08010801A251BE
:1023A0001E58D8B0D6EF91F0D8EF91F01BEF91F016
:1023B000060E4260DEEF91F0E0EF91F0E6EF91F073
:1023C000422AD8901D361E361F3620360801276F48
:1023D000020E176E0801275152EF93F00801276F84
:1023E000020E08010801206F080127510801276F1C
:1023F000000E080108011F6F080127510801276F0F
:10240000050E176E0801275152EF93F00801276F50
:10241000020E08010801206F080127510801276FEB
:10242000010E080108011F6F0801275100EE42F05C
:10243000030EEF641EEF92F020EF92F01BEF91F08D
:102440000801276F040E426E08012751200E1D6EF1
:10245000EF0E1E6E090E1F6E000E206E52EF93F0EF
:10246000020E426036EF92F038EF92F04AEF92F0AF
:102470000801276F120E08010801206F080127517B
:102480000801276F010E080108011F6F080127517D
:102490001BEF91F018A64FEF92F051EF92F063EF1F
:1024A00092F00801276F140E08010801206F08013F
:1024B00027510801276F010E080108011D6F08014F
:1024C00027516BEF92F00801276F020E08010801F7
:1024D000206F0801275152EF93F0050E426073EF11
:1024E00092F075EF92F087EF92F00801276F100ECF
:1024F00008010801206F080127510801276F010E0C
:10250000080108011F6F080127511BEF91F0080116
:10251000276F080E176E080127510801276F110E4B
:1025200008010801206F0801275152EF93F0050EB2
:1025300042609DEF92F09FEF92F0B1EF92F00801B0
:10254000276F110E08010801206F080127510801AB
:10255000276F010E080108011F6F080127511BEFAB
:1025600091F00801276F140E08010801206F08017F
:1025700027510801276F010E080108011D6F08018E
:10258000275152EF93F00801276F140E080108013C
:10259000206F080127510801276F010E080108016B
:1025A0001D6F0801275152EF93F0050E4260DBEFDB
:1025B00092F0DDEF92F0EFEF92F00801276F100E2E
:1025C00008010801206F080127510801276F010E3B
:1025D000080108011F6F080127511BEF91F0080146
:1025E000276F140E08010801206F08012751080108
:1025F000276F010E080108011D6F0801275152EFD6
:1026000093F0050E426007EF93F009EF93F01BEF94
:1026100093F00801276F110E08010801206F0801CF
:1026200027510801276F010E080108011F6F0801DB
:1026300027511BEF91F00801276F140E08010801C4
:10264000206F080127510801276F010E08010801BA
:102650001D6F0801275152EF93F01750000A01E156
:10266000B5D5010A01E1E9D5030A01E159D6010A0C
:1026700001E16DD6060A01E1C9D6030A01E1F0D6EF
:10268000010A01E12AD70F0A01E151D7010A01E14C
:102690007AD7030A8AE0010A01E11FD7070AB1E0ED
:1026A0001BEF91F0080108012051D8B45AEF93F0C4
:1026B0005CEF93F0DDEF93F0080108011F51D8B4EF
:1026C00064EF93F066EF93F0D1EF93F0422AD89045
:1026D0001D361E361F3620360950295C08010801B8
:1026E000216F0A502A580801226F00EE09F010EEFF
:1026F00029F0E652EE52ED50E55C02E1EF50E75C66
:10270000D8B085EF93F087EF93F09DEF93F000EE54
:1027100003F0EECF27F8EDCF28F801500801275F2E
:1027200002500801285B08012751080108012127F0
:10273000080128510801080122230801080121513C
:102740000801276F0801080122510801286F0801BC
:10275000296B08012A6B08012751215E08012851C5
:10276000225A08012951235A08012A51245A0801E2
:10277000080121512F26080108012251302209C0E9
:1027800029F00AC02AF00801276F000E080108018D
:10279000736F0801275120C872F89FECA1F0DDEF9C
:1027A00093F00801276F010E08010801736F0801FB
:1027B000275120C872F89FECA1F0080108011D51B3
:1027C000D8B4E5EF93F0E7EF93F0E9EF93F06CEC1A
:1027D00033F0080108011E2B000E080108011E65D8
:1027E000F4EF93F0F6EF93F0EBEF8DF0000E0801AD
:1027F0000801216F000E0801226F030E0801080175
:10280000215D000E08012259D8A009EF94F00BEFCA
:1028100094F00DEF94F0D2EF94F0080108012151EB
:10282000140DF3CF27F8100E0801272700019F0E83
:1028300008012725E96EEA6A0001000EEA22EE503F
:10284000ED10D8A426EF94F028EF94F02AEF94F03E
:10285000D2EF94F0080108012151140DF3CF27F8AD
:10286000120E0801272700019F0E08012725E96E97
:10287000EA6A0001000EEA22EECF28F8EDCF29F82F
:102880005AEC42F00801285108010801A15D080135
:102890002A6F0801295108010801A25908012B6F6C
:1028A000DD0E08012A5D010E2B59D8A05AEF94F0D5
:1028B0005CEF94F0C0EF94F0140E08010801626F11
:1028C000000E0801636F0801080121510208080188
:1028D0000801606F080108012251D8A0E82A000809
:1028E0000801616F83EC3BF060C8AAF861C8ABF8DF
:1028F0000801276F010E08010801A96F080127517F
:10290000080108012129140D9F0E0801286F000EEF
:10291000296FF35008012827E86AF3BEE868080128
:10292000292328C8A7F829C8A8F808012A6F010E8A
:1029300008010801A66F08012A5108010801215168
:10294000140D9F0E08012B6F000E2C6FF350080121
:102950002B27E86AF3BEE86808012C232BC8A4F8EB
:102960002CC8A5F8A0EC23F0000E00010001D76FE1
:10297000000E0001D86F080108012107D8A0220726
:1029800008010801214B222B030E08010801215DDB
:10299000000E08012259D8A0D0EF94F0D2EF94F0A5
:1029A0000DEF94F0120059EF9BF00801486F000EF4
:1029B00007010701326F080148510801486F000EF6
:1029C00007010701386F080148510001780E08011E
:1029D00008014C6F0001000E08014D6F0EEC23F052
:1029E00007010701322BC4EC43F0A1C8C6F6A2C808
:1029F000C7F6A3C8C8F6A4C8C9F60801486F020EF6
:102A000007010701A66F080148517CEF9BF0040104
:102A1000B70E080108014E6F0401040E08014F6F44
:102A20000001780E080108014C6F0001000E08013A
:102A30004D6FE7EC1AF00009D8A421EF95F023EFD1
:102A400095F071EF95F0C4EC43F006010601C65114
:102A500008010801A15D0801486F06010601C75180
:102A600008010801A2590801496F06010601C85171
:102A700008010801A35908014A6F06010601C9515E
:102A800008010801A45908014B6FF30E485D9E0E22
:102A90004959000E4A59000E08014B59D8A053EF6E
:102AA00095F055EF95F06FEF95F00801486F010E26
:102AB00007010701A66F08014851020E070107012F
:102AC000326565EF95F067EF95F06FEF95F00801CF
:102AD000486F060E07010701A66F080148517CEFF9
:102AE0009BF078C0B3F479C0B4F47AC0B5F47BC07D
:102AF000B6F40801486F030E07010701A66F08012D
:102B00004851350E08010801536F000E0801546F3B
:102B1000000E08010801516F000E0801526F0801F4
:102B2000486F040E08010801506F08014851B30EA8
:102B30000801496F040E4A6F080149C84CF80801A2
:102B40004AC84DF8080108014E6B08014F6B22EC92
:102B5000D7F007010701A26F07010701A229D8A436
:102B6000B4EF95F0B6EF95F0B8EF95F07CEF9BF0F1
:102B70000801486F040E07010701A66F08014851BC
:102B8000A2C74CF893EC39F008014D514C11D8A470
:102B9000CCEF95F0CEEF95F0D0EF95F07CEF9BF079
:102BA00006010601E34BE42BE4C653F867EC3DF065
:102BB000E3C653F867EC3DF00801486F010E0801C9
:102BC0000801536F0801485167EC3DF00801486F58
:102BD000000E08010801536F0801485167EC3DF0F1
:102BE0000801486F000E08010801536F08014851A1
:102BF00067EC3DF00801486F010E08010801536FB2
:102C00000801485167EC3DF00801486F000E0801CB
:102C10000801536F0801485167EC3DF00801486F07
:102C2000000E08010801536F0801485167EC3DF0A0
:102C30000801486F000E08010801536F0801485150
:102C400067EC3DF00801486F000E08010801536F62
:102C50000801485167EC3DF00801486F000E08017B
:102C60000801536F0801485167EC3DF00801486FB7
:102C7000000E08010801536F0801485167EC3DF050
:102C80000701070107510611D8B449EF96F04BEF41
:102C900096F053EF96F006C74CF807C74DF836ECA0
:102CA0001AF059EF96F022C74CF823C74DF881EC83
:102CB00019F00801486F000E08010801536F080160
:102CC000485167EC3DF03CC753F867EC3DF0080114
:102CD000486F000E08010801536F0801485167EC66
:102CE0003DF00801486F010E08010801536F08010B
:102CF000485167EC3DF053EC21F0C4EC43F0A1C81F
:102D0000C6F6A2C8C7F6A3C8C8F6A4C8C9F6080183
:102D1000486F050E07010701A66F080148517CEFB7
:102D20009BF0A2C74CF8D9EC39F008014D514C1179
:102D3000D8A49DEF96F09FEF96F0DBEF96F0C4ECF1
:102D400043F006010601C65108010801A15D080112
:102D5000486F06010601C75108010801A259080180
:102D6000496F06010601C85108010801A35908016D
:102D70004A6F06010601C95108010801A45908015A
:102D80004B6FF30E485D9E0E4959000E4A59000ED6
:102D900008014B59D8A0CFEF96F0D1EF96F06FEF26
:102DA00095F00801486F060E07010701A66F08019C
:102DB00048517CEF9BF008013D0E080108014D6F62
:102DC0000801080E08014E6F35EC3DF008013C0E7D
:102DD000080108014D6F0801080E08014E6F35EC1F
:102DE0003DF006010601E451080108013D1906E124
:102DF00006010601E351080108013C19D8B403EFAC
:102E000097F005EF97F009EF97F08FEC41F07CEF2A
:102E10009BF008013F0E080108014D6F0801080EE4
:102E200008014E6F35EC3DF008013E0E0801080127
:102E30004D6F0801080E08014E6F35EC3DF008019A
:102E4000410E080108014D6F0801080E08014E6F80
:102E500035EC3DF00801400E080108014D6F0801F6
:102E6000080E08014E6F35EC3DF00801430E0801D5
:102E700008014D6F0801080E08014E6F35EC3DF05A
:102E80000801420E080108014D6F0801080E0801F3
:102E90004E6F35EC3DF00801450E080108014D6FFD
:102EA0000801080E08014E6F35EC3DF00801440E94
:102EB000080108014D6F0801080E08014E6F35EC3E
:102EC0003DF00801470E080108014D6F0801080E8A
:102ED00008014E6F35EC3DF00801460E080108016F
:102EE0004D6F0801080E08014E6F35EC3DF0A7EF5D
:102EF00097F0D5EC37F00801310E080108014D6F4D
:102F00000801080E08014E6F35EC3DF00801300E47
:102F1000080108014D6F0801080E08014E6F35ECDD
:102F20003DF00801310E080108014D6F0801080E3F
:102F300008014E6F35EC3DF00801300E0801080124
:102F40004D6F0801080E08014E6F35EC3DF0080189
:102F500008014007D8A0410708014029D8B44129F9
:102F6000D8A4B5EF97F0B7EF97F079EF97F098EF17
:102F700098F0D5EC37F00801330E080108014D6FC9
:102F80000801080E08014E6F35EC3DF00801320EC5
:102F9000080108014D6F0801080E08014E6F35EC5D
:102FA0003DF00801350E080108014D6F0801080EBB
:102FB00008014E6F35EC3DF00801340E08010801A0
:102FC0004D6F0801080E08014E6F35EC3DF0080109
:102FD000390E080108014D6F0801080E08014E6FF7
:102FE00035EC3DF00801380E080108014D6F08016D
:102FF000080E08014E6F35EC3DF00801370E080150
:1030000008014D6F0801080E08014E6F35EC3DF0C8
:103010000801360E080108014D6F0801080E08016D
:103020004E6F35EC3DF008013B0E080108014D6F75
:103030000801080E08014E6F35EC3DF008013A0E0C
:10304000080108014D6F0801080E08014E6F35ECAC
:103050003DF00801080132053311D8A432EF98F091
:1030600034EF98F07BEF98F0080108013405351132
:10307000D8A43DEF98F03FEF98F07BEF98F008016F
:1030800008013A51040A3B11D8A449EF98F04BEFDC
:1030900098F07BEF98F0070108830401B30E080154
:1030A00008014D6F0401040E08014E6F35EC3DF030
:1030B0000401B40E080108014D6F0401040E08015B
:1030C0004E6F35EC3DF00401B50E080108014D6F5F
:1030D0000401040E08014E6F35EC3DF00401B60EFC
:1030E000080108014D6F0401040E08014E6F35EC14
:1030F0003DF08AEF9AF088EF98F008012F0E080152
:1031000008014D6F0801080E08014E6F35EC3DF0C7
:10311000080108013A07D8A03B0708013A29D8B4AA
:103120003B29D8A496EF98F098EF98F07DEF98F0AF
:10313000080108014207D8A0430708014229D8B472
:103140004329D8A4A6EF98F0A8EF98F0B9EF97F02C
:1031500089EF99F0D5EC37F00801330E080108012A
:103160004D6F0801080E08014E6F35EC3DF0080167
:10317000320E080108014D6F0801080E08014E6F5C
:1031800035EC3DF00801350E080108014D6F0801CE
:10319000080E08014E6F35EC3DF00801340E0801B1
:1031A00008014D6F0801080E08014E6F35EC3DF027
:1031B0000801390E080108014D6F0801080E0801C9
:1031C0004E6F35EC3DF00801380E080108014D6FD7
:1031D0000801080E08014E6F35EC3DF00801370E6E
:1031E000080108014D6F0801080E08014E6F35EC0B
:1031F0003DF00801360E080108014D6F0801080E68
:1032000008014E6F35EC3DF008013B0E0801080146
:103210004D6F0801080E08014E6F35EC3DF00801B6
:103220003A0E080108014D6F0801080E08014E6FA3
:1032300035EC3DF00801080132053311D8A423EF25
:1032400099F025EF99F06CEF99F008010801340529
:103250003511D8A42EEF99F030EF99F06CEF99F07A
:10326000080108013A51040A3B11D8A43AEF99F039
:103270003CEF99F06CEF99F0070108830401B30E5D
:10328000080108014D6F0401040E08014E6F35EC72
:103290003DF00401B40E080108014D6F0401040E55
:1032A00008014E6F35EC3DF00401B50E0801080130
:1032B0004D6F0401040E08014E6F35EC3DF0040122
:1032C000B60E080108014D6F0401040E08014E6F8F
:1032D00035EC3DF08AEF9AF079EF99F008012F0E66
:1032E000080108014D6F0801080E08014E6F35EC0A
:1032F0003DF0080108013A07D8A03B0708013A2928
:10330000D8B43B29D8A487EF99F089EF99F06EEFF4
:1033100099F0080108014407D8A04507080144298D
:10332000D8B44529D8A497EF99F099EF99F0AAEF6E
:1033300098F07AEF9AF0D5EC37F00801330E0801D7
:1033400008014D6F0801080E08014E6F35EC3DF085
:103350000801320E080108014D6F0801080E08012E
:103360004E6F35EC3DF00801350E080108014D6F38
:103370000801080E08014E6F35EC3DF00801340ECF
:10338000080108014D6F0801080E08014E6F35EC69
:103390003DF00801390E080108014D6F0801080EC3
:1033A00008014E6F35EC3DF00801380E08010801A8
:1033B0004D6F0801080E08014E6F35EC3DF0080115
:1033C000370E080108014D6F0801080E08014E6F05
:1033D00035EC3DF00801360E080108014D6F08017B
:1033E000080E08014E6F35EC3DF008013B0E080158
:1033F00008014D6F0801080E08014E6F35EC3DF0D5
:1034000008013A0E080108014D6F0801080E080175
:103410004E6F35EC3DF00801080132053311D8A498
:1034200014EF9AF016EF9AF05DEF9AF00801080198
:1034300034053511D8A41FEF9AF021EF9AF05DEF13
:103440009AF0080108013A51040A3B11D8A42BEF65
:103450009AF02DEF9AF05DEF9AF0070108830401CE
:10346000B30E080108014D6F0401040E08014E6FF0
:1034700035EC3DF00401B40E080108014D6F040164
:10348000040E08014E6F35EC3DF00401B50E080145
:1034900008014D6F0401040E08014E6F35EC3DF03C
:1034A0000401B60E080108014D6F0401040E080165
:1034B0004E6F35EC3DF08AEF9AF06AEF9AF0080112
:1034C0002F0E080108014D6F0801080E08014E6F0C
:1034D00035EC3DF0080108013A07D8A03B07080188
:1034E0003A29D8B43B29D8A478EF9AF07AEF9AF029
:1034F0005FEF9AF0080108014607D8A047070801C6
:103500004629D8B44729D8A488EF9AF08AEF9AF0D0
:103510009BEF99F08FEC41F0A2C74CF8A3EC36F08A
:1035200007010701A2690801486F070E070107019B
:10353000A66F080148510701070108B3A2EF9AF0EE
:10354000A4EF9AF0B1EF9AF0000E04010401B36FFA
:10355000000E0401B46F000E0401B56F000E0401EB
:10356000B66F2DC8E9FF2EC8EAFF0401B3C4EEFF11
:103570000401B4C4EEFF0401B5C4EEFF0401B6C4F7
:10358000EEFF010E7FEF9BF0010E0701070138658A
:10359000CCEF9AF0CEEF9AF0DFEF9AF02DC8E9FF6A
:1035A0002EC8EAFF000EEE6E000EEE6E000EEE6EFE
:1035B000000EED6EED52ED52010E7FEF9BF0070114
:1035C0000701382B00017F517C117D117E11D8B489
:1035D000ECEF9AF0EEEF9AF06FEF95F0000100013A
:1035E0007C5100010001781B000100017D510001A8
:1035F0000001791B000100017E51000100017A1BCE
:10360000000100017F51000100017B1B000100014E
:103610007851000100017C1B00010001795100017B
:1036200000017D1B000100017A51000100017E1B99
:10363000000100017B51000100017F1B000100011E
:103640007C5100010001781B000100017D51000147
:103650000001791B000100017E51000100017A1B6D
:10366000000100017F51000100017B1B0801486F30
:10367000000E07010701326F0801485107010701D9
:10368000A229D8B446EF9BF048EF9BF04FEF9BF098
:10369000A2C74CF8A3EC36F007010701A2690801A4
:1036A000486F010E07010701A66F080148517CEF22
:1036B0009BF007010701A651000A02E1D5EF94F043
:1036C000010A02E1E5EF94F0030A02E107EF95F049
:1036D000010A02E181EF95F0070A02E1C0EF95F0DF
:1036E000010A02E191EF96F0030A01E14DD7010AC8
:1036F00001E121D77CEF9BF0000E7FEF9BF01200E1
:103700000201730E08010801896F0201020E08010F
:103710008A6F7BC8E9FF7CC8EAFF0801EECF8FF80B
:103720000801EECF90F80801EECF91F80801EECF36
:1037300092F87DC8E9FF7EC8EAFF0801EECFA3F842
:103740000801EECFA4F80801EECFA5F80801EECFEE
:10375000A6F87FC8E9FF80C8EAFF0801EECF9BF812
:103760000801EECF9CF80801EECF9DF80801EECFDE
:103770009EF881C8E9FF82C8EAFF0801EECF9FF8F2
:103780000801EECFA0F80801EECFA1F80801EECFB6
:10379000A2F883C8E9FF84C8EAFF0801EECF8BF8DE
:1037A0000801EECF8CF80801EECF8DF80801EECFBE
:1037B0008EF8730E0801AF6F020EB06F080108019A
:1037C0007A510801B01905E1080108017951080191
:1037D000AF19D8A4EEEF9BF0F0EF9BF070EF9CF0E8
:1037E0000801AF6F000E08010801886F0801AF5192
:1037F0000F0E08010801886500EF9CF002EF9CF0B5
:1038000004EF9CF06EEF9CF0030E0801080179258F
:10381000E96E000E080108017A21EA6EEF500801F6
:103820000801876F79C8E9FF7AC8EAFF030E08012B
:1038300008017925E16E000E080108017A21E26E87
:10384000EFCFE7FF79C8E9FF7AC8EAFF080187C828
:10385000EFFF010E080108017925E96E000E08014D
:1038600008017A21EA6EEF5008010801876F020E05
:10387000080108017925E96E000E080108017A2186
:10388000EA6E010E080108017925E16E000E0801BB
:1038900008017A21E26EEFCFE7FF020E080108016E
:1038A0007925E96E000E080108017A21EA6E080107
:1038B00087C8EFFF040E080108017927000E0801F0
:1038C0007A2308010801882B0F0E0801080188657A
:1038D0006CEF9CF06EEF9CF004EF9CF026EF9DF0F7
:1038E0000801AF6F000E08010801886F0801AF5191
:1038F0000F0E08010801886580EF9CF082EF9CF0B4
:1039000084EF9CF026EF9DF079C8E9FF7AC8EAFFC2
:10391000080108018851040DF3CFAFF8030E080128
:10392000AF270801AF510801080189250801B06FD0
:10393000E86A0801AFBFE868080108018A210801A8
:10394000B16FB0C8E1FFB1C8E2FFEFCFE7FF0801F8
:103950000801794B7A2B79C8E9FF7AC8EAFF080198
:1039600008018851040DF3CFAFF8020E0801AF270C
:103970000801AF510801080189250801B06FE86A04
:103980000801AFBFE868080108018A210801B16F8A
:10399000B0C8E1FFB1C8E2FFEFCFE7FF08010801BF
:1039A000794B7A2B79C8E9FF7AC8EAFF0801080148
:1039B0008851040DF3CFAFF8010E0801AF270801BD
:1039C000AF510801080189250801B06FE86A0801B4
:1039D000AFBFE868080108018A210801B16FB0C8CB
:1039E000E1FFB1C8E2FFEFCFE7FF08010801794B23
:1039F0007A2B79C8E9FF7AC8EAFF080108018851E3
:103A0000040DF3500801080189250801AF6FE86A29
:103A1000F3BEE868080108018A210801B06FAFC849
:103A2000E1FFB0C8E2FFEFCFE7FF08010801794BE3
:103A30007A2B08010801882B0F0E08010801886500
:103A400024EF9DF026EF9DF084EF9CF00801AF6F0E
:103A50000D0E08010801876F0801AF510801AF6F13
:103A6000080E08010801866F0801AF510801AF6F09
:103A7000020E08010801856F0801AF510801AF6F00
:103A8000000E08010801886F0801AF514F0E0801B0
:103A9000080188654EEF9DF050EF9DF052EF9DF0CC
:103AA0003FEFA1F0140E0801080188615AEF9DF064
:103AB0005CEF9DF0D1EF9DF00801A3C8AFF80801BD
:103AC000A4C8B0F80801A5C8B1F80801A6C8B2F8A2
:103AD0000801AF1FB01FB11FB21F080108019F519D
:103AE0000801AF150801B36F08010801A0510801D2
:103AF000B0150801B46F08010801A1510801B11502
:103B00000801B56F08010801A2510801B2150801AA
:103B1000B66F080108019B5108010801A3150801AF
:103B2000B76F080108019C5108010801A41508019C
:103B3000B86F080108019D5108010801A515080189
:103B4000B96F080108019E5108010801A615080176
:103B5000BA6F0801B3510801B71108010801936F4A
:103B60000801B4510801B8110801946F0801B5515A
:103B70000801B9110801956F0801B6510801BA1181
:103B80000801966F990E08010801976F790E0801D8
:103B9000986F820E0801996F5A0E08019A6F2FEFE5
:103BA0009FF0130E080108018865D9EF9DF0DBEF47
:103BB0009DF031EF9EF0280E080108018861E3EFC7
:103BC0009DF0E5EF9DF031EF9EF0080108019B515B
:103BD00008010801A3190801AF6F080108019C51F1
:103BE00008010801A4190801B06F080108019D51DE
:103BF00008010801A5190801B16F080108019E51CB
:103C000008010801A6190801B26F080108019F51B7
:103C10000801AF1908010801936F08010801A051BC
:103C20000801B0190801946F08010801A1510801A9
:103C3000B1190801956F08010801A2510801B219D4
:103C40000801966FA10E08010801976FEB0E08019D
:103C5000986FD90E0801996F6E0E08019A6F2FEFB9
:103C60009FF0270E08010801886539EF9EF03BEFB1
:103C70009EF0E5EF9EF03C0E08010801886143EFDD
:103C80009EF045EF9EF0E5EF9EF0080108019F5180
:103C9000080108019B150801AF6F08010801A05138
:103CA000080108019C150801B06F08010801A15125
:103CB000080108019D150801B16F08010801A25112
:103CC000080108019E150801B26F080108019F5103
:103CD00008010801A3150801B36F08010801A051EC
:103CE00008010801A4150801B46F08010801A151D9
:103CF00008010801A5150801B56F08010801A251C6
:103D000008010801A6150801B66F080108019B51BA
:103D100008010801A3150801B76F080108019C51AB
:103D200008010801A4150801B86F080108019D5198
:103D300008010801A5150801B96F080108019E5185
:103D400008010801A6150801BA6F0801B35108015E
:103D5000B7110801BB6F0801B4510801B81108017F
:103D6000BC6F0801B5510801B9110801BD6F080108
:103D7000B6510801BA110801BE6F0801AF51080120
:103D8000BB1108010801936F0801B0510801BC1173
:103D90000801946F0801B1510801BD110801956F28
:103DA0000801B2510801BE110801966FDC0E08012E
:103DB0000801976FBC0E0801986F1B0E0801996FE0
:103DC0008F0E08019A6F2FEF9FF0080108019B5199
:103DD00008010801A3190801AF6F080108019C51EF
:103DE00008010801A4190801B06F080108019D51DC
:103DF00008010801A5190801B16F080108019E51C9
:103E000008010801A6190801B26F080108019F51B5
:103E10000801AF1908010801936F08010801A051BA
:103E20000801B0190801946F08010801A1510801A7
:103E3000B1190801956F08010801A2510801B219D2
:103E40000801966FD60E08010801976FC10E080190
:103E5000986F620E0801996FCA0E08019A6F0F0ED3
:103E600008010801886537EF9FF039EF9FF056EFA2
:103E7000A0F0080108018751040DF3500801080162
:103E800089250801AF6FE86AF3BEE86808010801F8
:103E90008A210801B06FAFC8E9FFB0C8EAFF080186
:103EA000EECFA7F80801EECFA8F80801EECFA9F8E9
:103EB0000801EECFAAF8080108018651040DF3505D
:103EC0000801080189250801AF6FE86AF3BEE868B8
:103ED000080108018A210801B06FAFC8E9FFB0C826
:103EE000EAFF0801EECFABF80801EECFACF808010D
:103EF000EECFADF80801EECFAEF808010801AB51E6
:103F000008010801A71B08010801AC5108010801BC
:103F1000A81B08010801AD5108010801A91B0801EF
:103F20000801AE5108010801AA1B080108018551CA
:103F3000040DF3500801080189250801AF6FE86AF4
:103F4000F3BEE868080108018A210801B06FAFC814
:103F5000E9FFB0C8EAFF0801EECFABF80801EECFE9
:103F6000ACF80801EECFADF80801EECFAEF80801CD
:103F70000801AB5108010801A71B08010801AC5159
:103F800008010801A81B08010801AD51080108013A
:103F9000A91B08010801AE5108010801AA1B08016C
:103FA000080188510F0B040DF35008010801892501
:103FB0000801AF6FE86AF3BEE868080108018A21CA
:103FC0000801B06FAFC8E9FFB0C8EAFF0801EECF43
:103FD000ABF80801EECFACF80801EECFADF8080160
:103FE000EECFAEF808010801AB5108010801A71B8C
:103FF00008010801AC5108010801A81B08010801CB
:10400000AD5108010801A91B08010801AE510801C2
:104010000801AA1B0801AF6F010E08010801C66F55
:104020000801AF51A7C8C2F8A8C8C3F8A9C8C4F806
:10403000AAC8C5F814EC33F00801080188510F0B29
:10404000040DF3500801080189250801B06FE86AE2
:10405000F3BEE868080108018A210801B16FB0C801
:10406000E9FFB1C8EAFF0801C2C8EEFF0801C3C8F2
:10407000EEFF0801C4C8EEFF0801C5C8EDFFED5210
:10408000ED5208010801872B08010801862B080161
:104090000801852B0F0E0801080187170F0E080174
:1040A000080186170F0E080108018517080108018D
:1040B00088510F0B040DF3500801080189250801F0
:1040C000AF6FE86AF3BEE868080108018A210801B9
:1040D000B06FAFC8E9FFB0C8EAFFEECFB1F8EECFDE
:1040E000B2F8EECFB3F8EECFB4F80801B56F050E15
:1040F00008010801C66F0801B5518FC8C2F890C801
:10410000C3F891C8C4F892C8C5F814EC33F008019C
:10411000B15108010801C2250801B66F0801B2516A
:1041200008010801C3210801B76F0801B351080154
:104130000801C4210801B86F0801B4510801080141
:10414000C5210801B96F0801080193510801B6257E
:104150000801BA6F0801080194510801B72108014C
:10416000BB6F0801080195510801B8210801BC6F17
:104170000801080196510801B9210801BD6F080125
:1041800008018B510801BA250801BE6F080108011A
:104190008C510801BB210801BF6F080108018D5136
:1041A0000801BC210801C06F080108018E510801F7
:1041B000BD210801C16F0801080197510801BE2502
:1041C00008010801A76F0801080198510801BF21E3
:1041D0000801A86F0801080199510801C0210801D0
:1041E000A96F080108019A510801C1210801AA6FAD
:1041F0009FC88BF8A0C88CF8A1C88DF8A2C88EF80B
:104200009BC89FF89CC8A0F89DC8A1F89EC8A2F8BA
:104210000801AF6F1E0E08010801C66F0801AF51FB
:10422000A3C8C2F8A4C8C3F8A5C8C4F8A6C8C5F8EE
:1042300014EC33F0C2C89BF8C3C89CF8C4C89DF8FE
:10424000C5C89EF88FC8A3F890C8A4F891C8A5F86F
:1042500092C8A6F8A7C88FF8A8C890F8A9C891F87E
:10426000AAC892F808010801882B4F0E080108011E
:1042700088653DEFA1F03FEFA1F052EF9DF07BC8C4
:10428000E9FF7CC8EAFF080108018F51EE2608010A
:104290009051EE2208019151EE2208019251ED2237
:1042A000ED52ED527DC8E9FF7EC8EAFF0801080122
:1042B000A351EE260801A451EE220801A551EE22D9
:1042C0000801A651ED22ED52ED527FC8E9FF80C8EA
:1042D000EAFF080108019B51EE2608019C51EE22DD
:1042E00008019D51EE2208019E51ED22ED52ED5242
:1042F00081C8E9FF82C8EAFF080108019F51EE2644
:104300000801A051EE220801A151EE220801A2519C
:10431000ED22ED52ED5283C8E9FF84C8EAFF08019F
:1043200008018B51EE2608018C51EE2208018D51B7
:10433000EE2208018E51ED22ED52ED521200B7EC43
:1043400024F00801080172A1A8EFA1F0AAEFA1F0E2
:10435000AEEFA1F01986080108017291189A189C15
:10436000189E199219941990B6EFA1F0CBEC3DF07C
:104370000009D8B4BEEFA1F0C0EFA1F0B6EFA1F0F4
:10438000080108017251060BD8B4C9EFA1F0CBEFB8
:10439000A1F0D4EFA1F0000E08010801766F000E25
:1043A0000801776F74EFA3F000EE29F010EE07F02C
:1043B000E652EE52ED50E518EFCFE8FFD8B4E7181B
:1043C000D8A4E5EFA1F0E7EFA1F0F0EFA1F0000E27
:1043D00008010801766F000E0801776F44EFA3F023
:1043E00000EE07F010EE29F0E652EE52ED50E55CDB
:1043F00002E1EF50E75CD8B000EFA2F002EFA2F0CC
:1044000057EFA2F02950075C08010801766F2A5087
:1044100008580801776F0801080176512F5C0801E0
:10442000080177513058D8B018EFA2F01AEFA2F077
:104430001EEFA2F02FC076F830C077F8080108010F
:104440007651405C0801080177514158D8B02BEFF4
:10445000A2F02DEFA2F032EFA2F040C076F841C0FA
:1044600077F8198476C8AAF877C8ABF81CC0A9F801
:1044700029C0A7F82AC0A8F808019C6F000E0801FF
:104480000801A66F08019C51050E08010801A46FE0
:104490000B0E0801A56FA0EC23F00801080176516E
:1044A00029260801080177512A2244EFA3F0295058
:1044B000035C08010801866F2A5004580801876FC1
:1044C000080108EE86F0EECF9CF8EDCF9DF807507E
:1044D00008019C27085008019D23015008019C5D9C
:1044E00008010801766F025008019D590801776F95
:1044F0000801080176512F5C0801080177513058F6
:10450000D8B085EFA2F087EFA2F08BEFA2F02FC01A
:1045100076F830C077F8080108017651405C080150
:10452000080177514158D8B098EFA2F09AEFA2F065
:104530009FEFA2F040C076F841C077F819840801D7
:104540000801865108010801765D080108018751BC
:10455000080108017759D8B0B0EFA2F0B2EFA2F08D
:10456000B6EFA2F076C886F877C887F886C8AAF8AA
:1045700087C8ABF81CC0A9F829C0A7F82AC0A8F8BA
:1045800008019C6F000E08010801A66F08019C51EC
:10459000050E08010801A46F0B0E0801A56FA0EC21
:1045A00023F008010801865108010801765D080121
:1045B0000801866F08010801875108010801775931
:1045C0000801876F0801080187518611D8B4EBEF05
:1045D000A2F0EDEFA2F018EFA3F086C8AAF887C802
:1045E000ABF81CC0A9F801C0A7F802C0A8F80801E0
:1045F0009C6F000E08010801A66F08019C5100EE97
:1046000003F0EECF9DF8EDCF9EF8295008019D5F95
:104610002A5008019E5B050E08019D25080108012E
:10462000A46F0B0E08019E210801A56FA0EC23F0DA
:1046300008010801765129260801080177512A222C
:1046400000EE03F010EE29F0E652EE52ED50E55C7C
:1046500002E1EF50E75CD8A030EFA3F032EFA3F017
:1046600044EFA3F000EE03F0EECF9CF8EDCF9DF801
:10467000015008019C5F025008019D5B08019C519C
:10468000295E08019D512A5A19A649EFA3F04BEF64
:10469000A3F074EFA3F000EE2FF00801EE52080132
:1046A0007751ED18080176C8E8FFD8B4EF18D8B4F0
:1046B0005CEFA3F05EEFA3F074EFA3F000EE40F028
:1046C0000801EE5208017751ED18080176C8E8FF9D
:1046D000D8B4EF18D8B46FEFA3F071EFA3F074EF74
:1046E000A3F00801080172810801080177517611D1
:1046F000D8A47DEFA3F07FEFA3F08AEFA3F0080129
:1047000008017251030BD8B488EFA3F08AEFA3F02D
:10471000D0EFA3F00801080176512F5E08010801CF
:104720007751305A0801080177517611D8B49BEFC0
:10473000A3F09DEFA3F0A0EFA3F00801080172879A
:104740000801080173A1A7EFA3F0A9EFA3F0B7EF49
:10475000A3F008019C6F000E426E08019C51F20EFE
:104760001D6E9E0E1E6E000E1F6E000E206EC4EC9F
:1047700043F01D5008010801A1250F6E1E500801CD
:104780000801A221106E1F5008010801A321116E1B
:10479000205008010801A421126E18882DEFA4F002
:1047A0000801080173A3D7EFA3F0D9EFA3F0F9EF45
:1047B000A3F0010E08019C6F1850070B08019D6FB4
:1047C00008019C5108019D27185008019D19F80BFC
:1047D00008019D19186E2106000E225A235A245AE8
:1047E000010E08010801766F000E0801776F2DEFAA
:1047F000A4F018A8FEEFA3F000EFA4F02DEFA4F0B2
:104800000801080173B107EFA4F009EFA4F017EF56
:10481000A4F04250D8B40FEFA4F011EFA4F017EFBA
:10482000A4F04206D89020321F321E321D32C4EC52
:1048300043F01D5008010801A1250F6E1E5008010C
:104840000801A221106E1F5008010801A321116E5A
:10485000205008010801A421126E2DC088F82EC036
:1048600089F82BC08AF82CC08BF821C08CF822C0A4
:104870008DF823C08EF824C08FF825C090F826C08C
:1048800091F827C092F828C093F83F0E08019517B9
:104890000801949108019493080194950801949754
:1048A0000B000E0072C895F8000E080108019A6FFF
:1048B000000E08019B6F08010801765121260801AE
:1048C000080177512222000E2322000E2422080123
:1048D000080172A36EEFA4F070EFA4F0A2EFA4F0B1
:1048E0000801080172B977EFA4F079EFA4F086EF20
:1048F000A4F0000E08010801906F000E0801916FEE
:10490000000E0801926F000E0801936F3FA28BEF1B
:10491000A4F08DEFA4F099EFA4F0080108018C0732
:10492000000E08018D5B08018E5B08018F5BA2EF12
:10493000A4F0010E2126000E2222000E2322000EDA
:1049400024223F820801080172A1A9EFA4F0ABEF75
:10495000A4F0C7EFA4F03FA0B0EFA4F0B2EFA4F032
:10496000BEEFA4F0080108018C07000E08018D5B62
:1049700008018E5B08018F5BC7EFA4F0010E2126B2
:10498000000E2222000E2322000E24223F8000EE81
:104990000DF010EE0BF0E652EE52ED50E55C02E148
:1049A000EF50E75CD8A0D7EFA4F0D9EFA4F000EF68
:1049B000A5F000EE0BF0EECF9CF8EDCF9DF80D507A
:1049C00008019C5F0E5008019D5B00EE05F0EECFE4
:1049D0009EF8EDCF9FF8035008019E5F0450080138
:1049E0009F5B08019C5108019E5D08010801966FBC
:1049F00008019D5108019F590801976F17EFA5F015
:104A000000EE0DF0EECF9CF8EDCF9DF80B500801B5
:104A10009C5F0C5008019D5BFF0E08019C2508015E
:104A20000801966FFF0E08019D210801976FC3ECE6
:104A300025F0A0C874F8A1C875F8400E0801080157
:104A4000745D000E08017559D8B029EFA5F02BEF61
:104A5000A5F034EFA5F0000E08010801746F000EF8
:104A60000801756F3BEFA5F0400E08010801745F67
:104A7000000E0801755B0801080196510801080144
:104A8000745D080108019751080108017559D8B0F3
:104A90004CEFA5F04EEFA5F052EFA5F074C896F8D4
:104AA00075C897F80801880E08010801A06F080171
:104AB000080E0801A16FC7EC07F0140E08010801E9
:104AC0007627000E08017723080194510F0B500937
:104AD0000801946F0801080172A371EFA5F073EF4C
:104AE000A5F0ABEFA5F0040E080108017627000E33
:104AF0000801772308019C6F020E08010801786FF6
:104B000008019C5108019C6F040E08010801796F8F
:104B100008019C51020E080108017A6F180E080165
:104B20007B6F010E08019C6F0801080194390F0B7F
:104B300008019D6F08019C5108019D2708019D3BBC
:104B400008010801945108019D190F0B08019D19D6
:104B500008010801946F6CC07CF86DC07DF86EC0D0
:104B60007EF86FC07FF833C080F834C081F835C05C
:104B700082F836C083F808019C6F000E0801080116
:104B8000846F08019C5108019C6F060E0801080102
:104B9000856F08019C5176C886F877C887F886C863
:104BA000BCF887C8BDF82FEC43F0BCC886F8BDC878
:104BB00087F80C0E08010801BC6F000E0801BD6FDC
:104BC00008017C0E08010801BA6F0801080E0801EF
:104BD000BB6FF2EC1EF008010801BA1D08010801C4
:104BE000986F08010801BB1D0801996FDD0E0801CF
:104BF0000801AC6F0A0E0801AD6F0BEC44F076C8EB
:104C0000A3F877C8A4F808019C6F060E08010801F4
:104C1000A26F08019C51330E08010801A06F000E1D
:104C20000801A16FCAEC18F0140E08010801C26F48
:104C3000000E0801C36F0801880E08010801C06F4B
:104C40000801080E0801C16FBBEC40F00801080123
:104C500072A32DEFA6F02FEFA6F041EFA6F0040E01
:104C600008010801C26F000E0801C36F0801780E29
:104C700008010801C06F0801080E0801C16FBBECF4
:104C800040F0F10E08010801AC6F0A0E0801AD6F8B
:104C90002CEC44F076C8A0F877C8A1F80EEC10F020
:104CA000A0C874F8A1C875F8010E08010801AC6F1E
:104CB0000B0E0801AD6F0BEC44F0020E0801080169
:104CC000C26F000E0801C36F0801740E08010801CD
:104CD000C06F0801080E0801C16FBBEC40F003EC87
:104CE00039F0120008011E6F000E080108011D6F47
:104CF00008011E51000E080108011D6582EFA6F093
:104D000084EFA6F086EFA6F0C7EFAAF07CEFAAF03A
:104D1000BAEFAAF0430E08010801536F000E080114
:104D2000546F440E08010801516F000E0801526FC4
:104D300008011E6F000E08010801506F08011E5186
:104D4000000E080108014C6F000E08014D6F000EA7
:104D500008014E6F000E08014F6F22ECD7F0446E31
:104D60004428D8A4B6EFA6F0B8EFA6F0BAEFA6F0A4
:104D7000BAEFAAF008011E6F020E00010001456F94
:104D800008011E51000E000100014B6F000E0001D2
:104D90004C6F000E00014D6F000E00014E6F3C0E77
:104DA000000100014F6F000E0001506F000E000166
:104DB000516F000E0001526F08011E6F000E0001BE
:104DC00000016B6F08011E510001469100014695DC
:104DD00097EC42F00009D8A4F0EFA6F0F2EFA6F0AD
:104DE000F4EFA6F0BAEFAAF044C04CF893EC39F017
:104DF0002C0E080108014C5D010E08014D59D8B078
:104E000004EFA7F006EFA7F008EFA7F0BAEFAAF0BB
:104E1000000146790A0E080108015D6F000E0801C5
:104E20005E6FFF0E080108015B6F000E08015C6FEA
:104E30004450170D0201000EF32408010801596FB8
:104E400008015A6B0201020E08015A2353EC40F08C
:104E500008011E6F000E08010801236F08011E5192
:104E600008011F6F010E08010801226F08011F5180
:104E7000CCECBCF0C4EC43F0A1C847F0A2C848F0A9
:104E8000A3C849F0A4C84AF000014E514B114C117F
:104E90004D11D8A44EEFA7F050EFA7F05AEFA7F0AE
:104EA000C4EC43F0A1C84BF0A2C84CF0A3C84DF02D
:104EB000A4C84EF008011E6F030E00010001456FEB
:104EC00008011E51BAEFAAF044C04CF8D9EC39F0F1
:104ED000FA0E080108014C5D000E08014D59D8B0CA
:104EE00074EFA7F076EFA7F0BFEFA7F0C4EC43F0A4
:104EF00000010001475108010801A15D08011E6F72
:104F000000010001485108010801A25908011F6F62
:104F100000010001495108010801A3590801206F4F
:104F2000000100014A5108010801A4590801216F3C
:104F3000E40E1E5D3D0E1F59010E2059000E0801A2
:104F40002159D8A0A6EFA7F0A8EFA7F088EFA6F008
:104F500008011E6F020E00010001456F08011E517D
:104F6000000E00010001576F000E0001586F000E87
:104F70000001596F000E00015A6FBAEFAAF000014C
:104F80004687C8ECAAF0020AD8B4C9EFA7F0CBEF65
:104F9000A7F0CDEFA7F0BAEFAAF008011E6F040E3C
:104FA00000010001456F08011E51000E00010001C3
:104FB0004B6F000E00014C6F000E00014D6F000E94
:104FC00000014E6F44C04CF893EC39F0020E08011A
:104FD00008014C5D010E08014D59D8B0F2EFA7F061
:104FE000F4EFA7F0F6EFA7F0BAEFAAF00A0E080167
:104FF00008015D6F000E08015E6FFF0E08010801D9
:105000005B6F000E08015C6F4450170D0201000E2B
:10501000F32408010801596F08015A6B0201020EBE
:1050200008015A2353EC40F008011E6F000E0801DE
:105030000801236F08011E5108011F6F030E0801AC
:105040000801226F08011F51CCECBCF0C4EC43F006
:10505000A1C847F0A2C848F0A3C849F0A4C84AF0C4
:1050600000010001452BBAEFAAF044C04CF8D9EC7E
:1050700039F0FA0E080108014C5D000E08014D5987
:10508000D8B045EFA8F047EFA8F08FEFA8F0C4EC38
:1050900043F000010001475108010801A15D08012A
:1050A0001E6F00010001485108010801A2590801C2
:1050B0001F6F00010001495108010801A3590801AF
:1050C000206F000100014A5108010801A45908019C
:1050D000216F2E0E1E5D500E1F59090E2059000E15
:1050E00008012159D8A077EFA8F079EFA8F088EF50
:1050F000A6F0000100EE45F0EF2A0B0EEF6483EFFF
:10510000A8F085EFA8F08DEFA8F008011E6F020E41
:1051100000010001456F08011E51BAEFAAF01AEF15
:10512000A9F044C04CF8A3EC36F04468C4EC43F05A
:10513000A1C847F0A2C848F0A3C849F0A4C84AF0E3
:1051400008011E6F0C0E00010001456F08011E5181
:105150000001468300014681000100016BA1B3EF0D
:10516000A8F0B5EFA8F0BDEFA8F057C06CF058C09C
:105170006DF059C06EF05AC06FF0000100016BA5D0
:10518000C4EFA8F0C6EFA8F0CEEFA8F05FC070F0B3
:1051900060C071F061C072F062C073F00001000184
:1051A0006BA3D5EFA8F0D7EFA8F0DFEFA8F05BC0B6
:1051B00074F05CC075F05DC076F05EC077F0000101
:1051C00000016BA7E6EFA8F0E8EFA8F0F0EFA8F079
:1051D00063C078F064C079F065C07AF066C07BF097
:1051E000000E000100017C6F000E00017D6F000EBB
:1051F00000017E6F000E00017F6F000100016BA9AE
:1052000004EFA9F006EFA9F00EEFA9F067C07CF05B
:1052100068C07DF069C07EF06AC07FF088EFA6F0BC
:1052200008011E6F020E00010001456F08011E51AA
:1052300088EFA6F0C8ECAAF0050A01E172D7030ACC
:10524000EFE088EFA6F0C4EC43F000010001475105
:1052500008010801A15D08011E6F0001000148510D
:1052600008010801A25908011F6F000100014951FE
:1052700008010801A3590801206F000100014A51EB
:1052800008010801A4590801216FF20E1E5D9E0E4F
:105290001F59000E2059000E08012159D8B053EFB4
:1052A000A9F055EFA9F057EFA9F0BAEFAAF0020E56
:1052B00000014F5D000E00015059000E00015159D0
:1052C000000E000100015259D8A069EFA9F06BEF60
:1052D000A9F084EFA9F0F20E0001000147279E0E0D
:1052E00000014823000E00014923000E00014A235B
:1052F000000100014F07000E0001505B0001515BEF
:105300000001525BBAEFAAF0430E08010801536F87
:10531000000E0801546F440E08010801516F000E81
:105320000801526F08011E6F000E08010801506F3E
:1053300008011E51000E080108014C6F000E080103
:105340004D6F000E08014E6F000E08014F6F22ECEA
:10535000D7F0446E4428D8A4B0EFA9F0B2EFA9F07A
:10536000B4EFA9F0BAEFAAF008011E6F0D0E00010C
:105370000001456F08011E5144C04CF893EC39F010
:10538000020E080108014C5D010E08014D59D8B00C
:10539000CCEFA9F0CEEFA9F0D0EFA9F0BAEFAAF0C8
:1053A00008011E6F010E08010801236F08011E513C
:1053B00008011F6F030E08010801226F08011F5129
:1053C000CCECBCF000014695C4EC43F0A1C847F01A
:1053D000A2C848F0A3C849F0A4C84AF000010001DF
:1053E000452BBAEFAAF044C04CF8D9EC39F0FA0ECC
:1053F000080108014C5D000E08014D59D8B003EFBB
:10540000AAF005EFAAF04DEFAAF0C4EC43F00001BA
:105410000001475108010801A15D08011E6F00014C
:105420000001485108010801A25908011F6F00013D
:105430000001495108010801A3590801206F00012A
:1054400000014A5108010801A4590801216F2E0EDC
:105450001E5D500E1F59090E2059000E08012159DA
:10546000D8A035EFAAF037EFAAF088EFA6F0000138
:1054700000EE45F0EF2A120EEF6441EFAAF043EF81
:10548000AAF04BEFAAF008011E6F020E0001000106
:10549000456F08011E51BAEFAAF074EFAAF044C09C
:1054A0004CF8A3EC36F04468C4EC43F0A1C847F0D4
:1054B000A2C848F0A3C849F0A4C84AF008011E6F6A
:1054C0000C0E00010001456F08011E5100014683CA
:1054D00088EFA6F008011E6F020E00010001456F63
:1054E00008011E5188EFA6F0C8ECAAF0050AD7E023
:1054F000030AF0E088EFA6F0000100014551000A20
:1055000001E106D4010A01E105D4030A01E147D40F
:10551000010A01E1D9D4070A01E154D5010A01E1E8
:10552000A4D5030A01E14ED5010A01E19ED50F0A77
:1055300001E148D5010A01E198D5030A01E142D50C
:10554000010A01E192D5070A01E17DD6010A01E1D4
:1055500013D7030A01E147D7010A01E10DD71F0A5A
:1055600001E141D7010A01E107D7030A01E13BD775
:10557000BAEFAAF0080108011D2B000E080108016E
:105580001D65C5EFAAF0C7EFAAF086EFA6F01200DE
:1055900008012B6F000E08010801236F08012B5131
:1055A0000801250E080108014D6F0801080E0801C9
:1055B0004E6F35EC3DF0080108012551020AD8A4D0
:1055C000E4EFAAF0E6EFAAF069EFAEF01C0E0801D6
:1055D00008014E6F000E08014F6F83EC42F0080186
:1055E0002B6F000E08010801266F08012B51050ED4
:1055F000080108012665FFEFAAF001EFABF003EF09
:10560000ABF036EFABF00801250E080108014D6F35
:105610000801080E08014E6F35EC3DF026C82BF846
:105620002D0E08012B2700016C0E08012B25E96EB9
:10563000EA6A0001000EEA22EF500801080125196C
:10564000D8B425EFABF027EFABF029EFABF0B1EF1B
:10565000AEF008010801262B050E08010801266599
:1056600034EFABF036EFABF003EFABF0000100012D
:1056700046B53DEFABF03FEFABF05CEFABF0100E9B
:10568000080108014E6F000E08014F6F83EC42F0D5
:10569000040E080108014F6F000E0801506F000151
:1056A000570E080108014D6F0001000E08014E6FF2
:1056B000F8EC2BF000016B81F00E080108014E6F31
:1056C000000E08014F6F83EC42F008012B6F000EB3
:1056D00008010801226F08012B510801250E08015D
:1056E00008014D6F0801080E08014E6F35EC3DF0C2
:1056F0000009D8A47EEFABF080EFABF08AEFABF0FF
:1057000008012B6F010E08010801226F08012B51BF
:1057100069EFAEF045EFAEF00801250E0801080173
:105720004D6F0801080E08014E6F35EC3DF0080181
:1057300008012505D8A49FEFABF0A1EFABF0C4EFB3
:10574000ABF00801230E080108014D6F0801080E97
:1057500008014E6F35EC3DF00001000146A5B3EFA6
:10576000ABF0B5EFABF0C2EFABF00801080123518D
:10577000020AD8A4BEEFABF0C0EFABF0C2EFABF0C3
:10578000B1EFAEF0C6EFABF0B1EFAEF05FEFAEF061
:105790000801250E080108014D6F0801080E0801D7
:1057A0004E6F35EC3DF0080108012551040AD8A4DC
:1057B000DCEFABF0DEEFABF0C4EFABF000010001CB
:1057C00046A5E5EFABF0E7EFABF015EFACF0080165
:1057D0002B6F000E08010801266F08012B51030EE4
:1057E000080108012665F7EFABF0F9EFABF0FBEF2E
:1057F000ABF013EFACF00801250E080108014D6F66
:105800000801080E08014E6F35EC3DF00801080153
:10581000262B030E08010801266511EFACF013EFEB
:10582000ACF0FBEFABF029EFACF0040E080108017F
:105830004F6F000E0801506F00015F0E0801080154
:105840004D6F0001000E08014E6FF8EC2BF00001C7
:105850006B85C6EFABF00801240E080108014D6FFF
:105860000801080E08014E6F35EC3DF0030E0801EB
:10587000080124653EEFACF040EFACF0C4EFABF0B4
:105880000001000146A547EFACF049EFACF077EF1F
:10589000ACF008012B6F000E08010801266F08010B
:1058A0002B51030E08010801266559EFACF05BEFA0
:1058B000ACF05DEFACF075EFACF00801250E08011F
:1058C00008014D6F0801080E08014E6F35EC3DF0E0
:1058D00008010801262B030E08010801266573EF55
:1058E000ACF075EFACF05DEFACF08BEFACF0040E0C
:1058F000080108014F6F000E0801506F00015B0E98
:10590000080108014D6F0001000E08014E6FF8EC10
:105910002BF000016B838DEFACF0040E0801080141
:10592000245F9EEFACF00801250E080108014D6FC1
:105930000801080E08014E6F35EC3DF00801080122
:10594000240708012429D8A4A8EFACF0AAEFACF0F2
:1059500093EFACF05FEFAEF00801240E08010801F0
:105960004D6F0801080E08014E6F35EC3DF0040E36
:10597000080108012461BFEFACF0C1EFACF0C3EF48
:10598000ACF0B1EFAEF00001000146B5CAEFACF0EB
:10599000CCEFACF0E4EFACF0040E080108014F6F5F
:1059A000000E0801506F0001630E080108014D6FE1
:1059B0000001000E08014E6FF8EC2BF000016B8720
:1059C000040E08010801245F030E08010801246584
:1059D000ECEFACF0EEEFACF00FEFADF0000100013A
:1059E00046B5F5EFACF0F7EFACF00FEFADF0040E0D
:1059F000080108014F6F000E0801506F0001670E8B
:105A0000080108014D6F0001000E08014E6FF8EC0F
:105A10002BF000016B89040E08010801245F1CEFC4
:105A2000ADF00801250E080108014D6F0801080EB0
:105A300008014E6F35EC3DF008010801240708010C
:105A40002429D8A426EFADF028EFADF011EFADF08A
:105A50005FEFAEF00801250E080108014D6F080147
:105A6000080E08014E6F35EC3DF008010801255184
:105A7000040AD8A43EEFADF040EFADF0C4EFABF0B8
:105A800008012A0E080108014D6F0801080E0801DF
:105A90004E6F35EC3DF00801290E080108014D6FED
:105AA0000801080E08014E6F35EC3DF00801280E84
:105AB000080108014D6F0801080E08014E6F35EC12
:105AC0003DF00801270E080108014D6F0801080E7E
:105AD00008014E6F35EC3DF0C6EFABF008012B6FBF
:105AE000010E08010801226F08012B515FEFAEF093
:105AF0000801250E080108014D6F0801080E080174
:105B00004E6F35EC3DF0080108012551040AD8A478
:105B10008CEFADF08EEFADF0C4EFABF00001000103
:105B200046A595EFADF097EFADF0C5EFADF00801EC
:105B30002B6F000E08010801266F08012B51030E80
:105B4000080108012665A7EFADF0A9EFADF0ABEFB6
:105B5000ADF0C3EFADF00801250E080108014D6F4F
:105B60000801080E08014E6F35EC3DF008010801F0
:105B7000262B030E080108012665C1EFADF0C3EF27
:105B8000ADF0ABEFADF01DEFAEF00001520E08012D
:105B900008014D6F0001000E08014E6F35EC3DF01D
:105BA0000001510E080108014D6F0001000E0801AF
:105BB0004E6F35EC3DF00001500E080108014D6FAD
:105BC0000001000E08014E6F35EC3DF000014F0E54
:105BD000080108014D6F0001000E08014E6F35EC01
:105BE0003DF000014FC02BF8000150C02CF800011F
:105BF00051C02DF8000152C02EF8060E06EFAEF08F
:105C0000D89008012E332D332C332B33E82E00EFA0
:105C1000AEF008012B51000100014F5F08012C512B
:105C200000010001505B08012D5100010001515B92
:105C300008012E5100010001525BC6EFABF00801D4
:105C4000240E080108014D6F0801080E08014E6F6F
:105C500035EC3DF037EFAEF00801250E08010801E4
:105C60004D6F0801080E08014E6F35EC3DF008013C
:105C70000801240708012429D8A441EFAEF043EF1E
:105C8000AEF02CEFAEF05FEFAEF008010801255149
:105C9000010A01E17DD5020A01E1DDD5050A01E134
:105CA0005BD6350A01E124D7060A01E135D5030A9E
:105CB00001E1D0D6C90A01E111D71FEFAEF008010A
:105CC00008012251D8B467EFAEF069EFAEF06DEF86
:105CD000ABF0080108012351020AD8A472EFAEF01C
:105CE00074EFAEF080EFAEF027C853F028C854F040
:105CF00029C855F02AC856F000014685AAEFAEF033
:105D0000080108012A5100010001561914E1080197
:105D1000080129510001000155190DE10801080190
:105D2000285100010001541906E10801080127511A
:105D3000000100015319D8B4A0EFAEF0A2EFAEF00D
:105D4000AAEFAEF008012B6F000E08010801236FC7
:105D500008012B518FEC41F0080108012351B6EFE7
:105D6000AEF08FEC41F0000EB6EFAEF01200DDEFBA
:105D7000B0F0080108010D51D8B4C1EFAEF0C3EF87
:105D8000AEF0DFEFAEF0550E080108010E65CBEF67
:105D9000AEF0CDEFAEF0DFEFAEF05C0E0801080123
:105DA0000E61D5EFAEF0D7EFAEF0DFEFAEF0080149
:105DB0001F6F010E070107010A6F08011F51F4EF61
:105DC000B0F01B0E080108010E65E9EFAEF0EBEF35
:105DD000AEF0FFEFAEF0200E080108010E61F3EF08
:105DE000AEF0F5EFAEF0FFEFAEF008011F6F030E5F
:105DF000070107010A6F08011F51F4EFB0F02A0EE6
:105E0000080108010E6507EFAFF009EFAFF01DEFD5
:105E1000AFF02F0E080108010E6111EFAFF013EF84
:105E2000AFF01DEFAFF008011F6F040E070107016F
:105E30000A6F08011F51F4EFB0F005EC36F0F4EFF3
:105E4000B0F01A0E080108010E6529EFAFF02BEF34
:105E5000AFF01DEFAFF0200E080108010E6133EF27
:105E6000AFF035EFAFF01DEFAFF008011F6F050E7B
:105E7000070107010A6F08011F51F4EFB0F0030E8C
:105E8000080108010E6547EFAFF049EFAFF01DEFD5
:105E9000AFF0090E080108010E6151EFAFF053EFAA
:105EA000AFF01DEFAFF008011F6F070E07010701EC
:105EB0000A6F08011F51F4EFB0F006010601D66722
:105EC00064EFAFF066EFAFF0A6EFAFF0010E0801A0
:105ED00008010E656EEFAFF070EFAFF084EFAFF03A
:105EE000050E080108010E6178EFAFF07AEFAFF010
:105EF00084EFAFF008011F6F010E06010601D66F97
:105F000008011F51F4EFB0F0040E080108010E65FE
:105F10008CEFAFF08EEFAFF0A2EFAFF0080E0801FC
:105F200008010E6196EFAFF098EFAFF0A2EFAFF07F
:105F300008011F6F020E06010601D66F08011F51EE
:105F4000F4EFB0F005EC36F0F4EFB0F00601060126
:105F5000D605D8A4AEEFAFF0B0EFAFF0DCEFAFF006
:105F6000040E080108010E65B8EFAFF0BAEFAFF00C
:105F70001DEFAFF0080E080108010E61C2EFAFF08F
:105F8000C4EFAFF01DEFAFF008011F6F000E060168
:105F90000601D66F08011F5107010701164B172B89
:105FA0000701D89007019037070191370701923711
:105FB00007019337F4EFB0F006010601D651020A4B
:105FC000D8A4E5EFAFF0E7EFAFF019EFB0F0010EB6
:105FD000080108010E65EFEFAFF0F1EFAFF01DEF34
:105FE000AFF0050E080108010E61F9EFAFF0FBEF0D
:105FF000AFF01DEFAFF008011F6F000E06010601A4
:10600000D66F08011F5107010701164B172B070117
:1060100007019051070107010C130701D8900701F0
:106020009037070191370701923707019337F4EF53
:10603000B0F005EC36F0F4EFB0F006010601D667DB
:1060400024EFB0F026EFB0F066EFB0F0030E0801D9
:1060500008010E652EEFB0F030EFB0F044EFB0F075
:10606000090E080108010E6138EFB0F03AEFB0F008
:1060700044EFB0F008011F6F010E06010601D66F54
:1060800008011F51F4EFB0F0080E080108010E6579
:106090004CEFB0F04EEFB0F062EFB0F0100E080130
:1060A00008010E6156EFB0F058EFB0F062EFB0F0BB
:1060B00008011F6F020E06010601D66F08011F516D
:1060C000F4EFB0F005EC36F0F4EFB0F006010601A5
:1060D000D605D8A46EEFB0F070EFB0F09CEFB0F042
:1060E000080E080108010E6578EFB0F07AEFB0F005
:1060F0001DEFAFF0100E080108010E6182EFB0F045
:1061000084EFB0F01DEFAFF008011F6F000E060125
:106110000601D66F08011F5107010701164B172B07
:106120000701D8900701903707019137070192378F
:1061300007019337F4EFB0F006010601D651020AC9
:10614000D8A4A5EFB0F0A7EFB0F0D9EFB0F0030EF0
:10615000080108010E65AFEFB0F0B1EFB0F01DEF30
:10616000AFF0090E080108010E61B9EFB0F0BBEF06
:10617000B0F01DEFAFF008011F6F000E0601060121
:10618000D66F08011F5107010701164B172B070196
:1061900007019051070107010C130701D89007016F
:1061A0009037070191370701923707019337F4EFD2
:1061B000B0F005EC36F0F4EFB0F0070107010A513A
:1061C000000A01E1D6D5010A01E1FBD5020A01E18D
:1061D00074D6070A01E135D6010A01E150D6020A58
:1061E00001E12BD7F4EFB0F0070107011651080ABF
:1061F0001711D8A4FEEFB0F000EFB1F07CEFB1F0D2
:1062000006010601E82B050E06010601E8610BEF09
:10621000B1F00DEFB1F068EFB1F0070107010C51DB
:1062200005010501FC2505010501FC6F000E0501B6
:106230000501FD210501FD6F000E05010501FE218F
:106240000501FE6F000E05010501FF210501FF6F2D
:10625000040E06010601E86130EFB1F032EFB1F053
:1062600045EFB1F00501FCC520F80501FDC521F899
:106270000501FEC522F808011F6B1FC8FCF520C8E8
:10628000FDF521C8FEF522C8FFF5070107010C51F5
:1062900006010601CA2506010601CA6F000E0601A5
:1062A0000601CB210601CB6F000E06010601CC21B1
:1062B0000601CC6F000E06010601CD210601CD6F4F
:1062C00008011F6F000E070107010C6F08011F5125
:1062D000000E07010701166F000E0701176F010E70
:1062E00007010701906F000E0701916F000E070173
:1062F000926F000E0701936F070107010A51030A0D
:10630000D8A485EFB1F087EFB1F0DBEFB1F0060173
:106310000601E851040AD8A490EFB1F092EFB1F071
:10632000DBEFB1F0FCC50FF8FDC510F8FEC511F8A4
:10633000FFC512F805EC36F00BEC43F0A50E080192
:1063400008012E6FFF0E08012F6F2D0E08010801A6
:106350002C6FFF0E08012D6FF5EC43F0E60E0801DF
:1063600008012E6FFE0E08012F6FAB0E0801080109
:106370002C6FFF0E08012D6FF5EC43F00FC82EF8BF
:1063800010C82FF811C830F812C831F8B10E080142
:1063900008012C6FFF0E08012D6F71EC43F008010E
:1063A0001F6F010E080108012C6F08011F515CECE2
:1063B00041F090EFB2F0070107010A51070AD8A493
:1063C000E4EFB1F0E6EFB1F08EEFB2F006010601B6
:1063D000E851050AD8A4EFEFB1F0F1EFB1F08EEF7C
:1063E000B2F0070107010C5108010801136F080101
:1063F000146B0801156B0801166BCAC617F8CBC6DB
:1064000018F8CCC619F8CDC61AF8FCC51BF8FDC59E
:106410001CF8FEC51DF8FFC51EF805EC36F0080196
:106420000801135108010801172508011F6F080111
:10643000080114510801080118210801206F080102
:10644000080115510801080119210801216F0801EF
:1064500008011651080108011A210801226FFF0ED8
:1064600008011F150801236F000E080120150801FF
:10647000246F000E080121150801256F000E080188
:1064800022150801266F0801230524112511261164
:10649000D8B44DEFB2F04FEFB2F051EFB2F090EF51
:1064A000B2F00BEC43F0A50E080108012E6FFF0EB1
:1064B00008012F6F2D0E080108012C6FFF0E080137
:1064C0002D6FF5EC43F0BB0E080108012E6FFE0E98
:1064D00008012F6FAB0E080108012C6FFF0E080199
:1064E0002D6FF5EC43F01BC82EF81CC82FF81DC803
:1064F00030F81EC831F8B10E080108012C6FFF0EEC
:1065000008012D6F71EC43F008011F6F010E0801A7
:1065100008012C6F08011F515CEC41F090EFB2F0C4
:106520001200020E080108014A25E96E000E08015A
:1065300008014B21EA6EEE50ED10D8A4A2EFB2F0A4
:10654000A4EFB2F0A7EFB2F0000E18EFB6F008011A
:10655000546FFE0E080108014E6F08015451020EDF
:10656000080108014A25E96E000E080108014B21C7
:10657000EA6EEECF54F8EDCF55F84AC8E9FF4BC8A4
:10658000EAFFEECF56F8EDCF57F84CC8E9FF4DC8FB
:10659000EAFFEECF58F8EDCF59F8020E08010801D6
:1065A0004C25E96E000E080108014D21EA6EEECF80
:1065B0005AF8EDCF5BF80801585108015A25080137
:1065C0005C6F0801595108015B2108015D6F0801EA
:1065D000565108015C2508015E6F080157510801FA
:1065E0005D2108015F6F0801545108015E1908011F
:1065F0000801506F0801555108015F190801516FDA
:106600000801546F000E080108014F6F0801545132
:10661000000E080108014F6510EFB3F012EFB3F060
:1066200014EFB3F0C4EFB3F04FC871F81DEC2BF0CA
:1066300017500D0AD8A41FEFB3F021EFB3F023EFEA
:10664000B3F0B7EFB3F01750040AD8A42AEFB3F0B1
:106650002CEFB3F04BEFB3F0020E080108014A250E
:10666000E96E000E080108014B21EA6E10EE1AF0E7
:10667000E652EE52ED50E518EFCFE8FFD8B4E71838
:10668000D8A445EFB3F047EFB3F049EFB3F04FC8EC
:106690004EF8B7EFB3F000EE1AF00801EE52080121
:1066A0005151ED18080150C8E8FFD8B4EF18D8B41C
:1066B0005CEFB3F05EEFB3F060EFB3F0B7EFB3F0C1
:1066C000B7EC24F000EE2DF0020E080108014A2577
:1066D000E16E000E080108014B21E26EE652EE5217
:1066E000ED50E518EFCFE8FFD8B4E718D8A47BEF5A
:1066F000B3F07DEFB3F0B7EFB3F000EE2BF04AC884
:10670000E1FF4BC8E2FFE652EE52ED50E518EFCF45
:10671000E8FFD8B4E718D8A490EFB3F092EFB3F045
:10672000B7EFB3F04CC8E9FF4DC8EAFFEECF54F81D
:10673000EECF55F8EECF56F8EECF57F836500801A9
:1067400057190BE135500801561907E1345008017B
:10675000551903E1335008015419D8A4B2EFB3F02E
:10676000B4EFB3F0B7EFB3F0010E18EFB6F00801D5
:1067700008014F2B000E080108014F65C2EFB3F06E
:10678000C4EFB3F014EFB3F0080108014E51FE0A54
:10679000D8B4CDEFB3F0CFEFB3F015EFB4F04EC8EF
:1067A00071F81DEC2BF0B7EC24F0080108014E51F4
:1067B000FE0AD8B4DEEFB3F0E0EFB3F015EFB4F0BB
:1067C00050C81AF051C81BF00A0E08010801B06F3A
:1067D000000E0801B16F4CC8AEF84DC8AFF8330ECB
:1067E00008010801AC6F000E0801AD6F58EC3AF0DB
:1067F0004AC8E9FF4BC8EAFFEECF2BF0EDCF2CF0F3
:10680000020E080108014A25E96E000E0801080180
:106810004B21EA6EEECF2DF0EDCF2EF001C029F026
:1068200002C02AF0010E18EFB6F00D0E08010801A3
:106830004A25E96E000E080108014B21EA6EEF506F
:106840000801546F080154B328EFB4F02AEFB4F0F4
:106850002DEFB4F0000E18EFB6F000010001D85192
:10686000D711D8B436EFB4F038EFB4F03BEFB4F052
:10687000000E18EFB6F0000E08010801526F000E6E
:106880000801536F030E08010801525D000E080154
:106890005359D8A04EEFB4F050EFB4F052EFB4F02B
:1068A0002EEFB5F0080108015251140DF3CF54F842
:1068B000100E0801542700019F0E08015425E96EAF
:1068C000EA6A0001000EEA22EE50ED10D8A46BEF48
:1068D000B4F06DEFB4F06FEFB4F02EEFB5F0020E40
:1068E000080108014A25E96E000E080108014B2144
:1068F000EA6E080108015251140DF3CF54F8100E3E
:106900000801542700019F0E08015425E16EE26A38
:106910000001000EE222E652EE52ED50E518EFCFF4
:10692000E8FFD8B4E718D8B498EFB4F09AEFB4F011
:106930009CEFB4F01CEFB5F04AC8E9FF4BC8EAFF82
:10694000080108015251140DF3CF54F80A0E080142
:10695000542700019F0E08015425E16EE26A0001F0
:10696000000EE222E652EE52ED50E518EFCFE8FFBE
:10697000D8B4E718D8B4BFEFB4F0C1EFB4F0C3EFA8
:10698000B4F01CEFB5F04CC8E9FF4DC8EAFFEECFFC
:1069900054F8EECF55F8EECF56F8EECF57F8080181
:1069A00008015251140D00019F0EF324E96EEA6AAA
:1069B0000001000EEA22EECF58F8EECF59F8EECFE4
:1069C0005AF8EECF5BF80801575108015B190EE148
:1069D0000801565108015A1909E1080155510801E9
:1069E000591904E10801545108015819D8B4FBEFB2
:1069F000B4F0FDEFB4F0FFEFB4F01CEFB5F05AECDB
:106A000042F0080108015251140DF3CF54F8120E50
:106A10000801542700019F0E08015425E96EEA6A17
:106A20000001000EEA220801A1C8EEFF0801A2C879
:106A3000EDFF000E18EFB6F008010801524B532B82
:106A4000030E08010801525D000E08015359D8A039
:106A50002CEFB5F02EEFB5F052EFB4F00801546F03
:106A6000000E080108014F6F08015451000E080183
:106A700008014F653EEFB5F040EFB5F042EFB5F0DD
:106A800015EFB6F04FC871F81DEC2BF018B64BEFB0
:106A9000B5F04DEFB5F04FEFB5F008EFB6F0B7EC4D
:106AA00024F0020E080108014A25E96E000E0801D3
:106AB00008014B21EA6E10EE2DF0E652EE52ED5039
:106AC000E518EFCFE8FFD8B4E718D8B46AEFB5F00F
:106AD0006CEFB5F06EEFB5F008EFB6F00A0E0801F6
:106AE0000801B06F000E0801B16F4CC8AEF84DC878
:106AF000AFF8080108015251140D00019F0EF32454
:106B000008010801AC6F0801AD6B0001000E08011F
:106B1000AD2358EC3AF04AC8E9FF4BC8EAFF080138
:106B200008015251140DF3CF54F80A0E08015427EE
:106B300000019F0E08015425E16EE26A0001000E7B
:106B4000E222EECFE6FFEDCFE5FF040E08010801DB
:106B50004A25E96E000E080108014B21EA6E080182
:106B600008015251140DF3CF54F80C0E08015427AC
:106B700000019F0E08015425E16EE26A0001000E3B
:106B8000E222EECFE6FFEECFE6FFEECFE6FFEDCF5F
:106B9000E5FFE552E552020E080108014A25E96EBB
:106BA000000E080108014B21EA6E0801080152514C
:106BB000140DF3CF54F8100E0801542700019F0E56
:106BC00008015425E16EE26A0001000EE222EECFD8
:106BD000E6FFEDCFE5FF5AEC42F008010801525103
:106BE000140DF3CF54F8120E0801542700019F0E24
:106BF00008015425E96EEA6A0001000EEA22080144
:106C0000A1C8EEFF0801A2C8EDFF000E18EFB6F014
:106C1000080108014F2B000E080108014F6513EF12
:106C2000B6F015EFB6F042EFB5F0000E18EFB6F083
:106C300012000801096F000E080108011D6F08010C
:106C4000095153EC44F00009D8A429EFB6F02BEF1A
:106C5000B6F063EFB6F00801096F000E08010801F5
:106C60000D6F08010951EAEC43F00801096FFF0EAE
:106C7000080108010D6F0801095100EC44F00601FC
:106C80000601E551D8B447EFB6F049EFB6F061EF31
:106C9000B6F0A1C72DF895EC12F0A1C70DF8EEECF7
:106CA00041F00801096FFE0E07010701A16F0801FD
:106CB00009510801096F000E06010601E56F080180
:106CC000095188EFB9F0A1C70DF83DEC41F000097A
:106CD000D8A46DEFB6F06FEFB6F08BEFB6F0010E03
:106CE00006010601E56577EFB6F079EFB6F08BEFB8
:106CF000B6F0060E06010601E56181EFB6F083EFFE
:106D0000B6F08BEFB6F00801096F060E060106011A
:106D1000E56F0801095169EFB9F059EC44F0000939
:106D2000D8A495EFB6F097EFB6F0ADEFB6F0080146
:106D3000096FFF0E080108010D6F08010951EAEC07
:106D400043F00801096FFF0E080108010D6F0801EB
:106D5000095100EC44F088EFB9F00801096FFF0E0B
:106D6000080108010D6F08010951EAEC43F0080120
:106D7000096F000E080108010D6F0801095100ECB0
:106D800044F00801096F000E08010801146F0801A2
:106D9000095127C712F828C713F808010A6F010E16
:106DA00008010801116F08010A51C80E08010B6F94
:106DB000010E0C6F08010BC80DF808010CC80EF885
:106DC000080108010F6B0801106B3FECDAF00701B6
:106DD0000701A16F0801096F010E06010601E56FA9
:106DE00008010951C4EC43F0A1C8C0F6A2C8C1F61D
:106DF000A3C8C2F6A4C8C3F688EFB9F0A1C70DF8BE
:106E00003DEC41F00009D8A408EFB7F00AEFB7F065
:106E100046EFB7F0C4EC43F006010601C05108018B
:106E20000801A15D0801096F06010601C1510801B1
:106E30000801A25908010A6F06010601C2510801A2
:106E40000801A35908010B6F06010601C35108018F
:106E50000801A45908010C6F5D0E095DA00E0A59C6
:106E6000120E0B59000E08010C59D8A03AEFB7F0DA
:106E70003CEFB7F044EFB7F00801096F060E0601CA
:106E80000601E56F0801095188EFB9F0C4EC43F041
:106E9000A1C802F7A2C803F7A3C804F7A4C805F75E
:106EA0000801096F020E06010601E56F080109518C
:106EB00088EFB9F00801096F000E080108010D6F95
:106EC00008010951EAEC43F00801096F000E0801BE
:106ED00008010D6F0801095100EC44F0C0ECE4F02A
:106EE0000801096F030E06010601E56F080109514B
:106EF00088EFB9F0C4EC43F006010601E95108013E
:106F00000801A15D0801096F06010601EA510801A7
:106F10000801A25908010A6F06010601EB51080198
:106F20000801A35908010B6F06010601EC51080185
:106F30000801A45908010C6F710E095D810E0A59F0
:106F40004A0E0B59000E08010C59D8A0AAEFB7F051
:106F5000ACEFB7F0B0EFB7F077EC40F088EFB9F0F6
:106F6000C4EC43F007010701025108010801A15DCB
:106F70000801096F07010701035108010801A2591F
:106F800008010A6F07010701045108010801A3590C
:106F900008010B6F07010701055108010801A459F9
:106FA00008010C6F510E095D840E0A59DF0E0B5952
:106FB000000E08010C59D8A0E0EFB7F0E2EFB7F0EF
:106FC000ECEFB7F00801096F080E06010601E56F46
:106FD0000801095188EFB9F0A1C713F894EC2DF01E
:106FE000080114511311D8B4F8EFB7F0FAEFB7F065
:106FF0000EEFB8F0C4EC43F0A1C8C0F6A2C8C1F6C9
:10700000A3C8C2F6A4C8C3F60801096F040E06019E
:107010000601E56F0801095188EFB9F088EFB9F072
:10702000C4EC43F006010601C05108010801A15D4E
:107030000801096F06010601C15108010801A259A2
:1070400008010A6F06010601C25108010801A3598F
:1070500008010B6F06010601C35108010801A4597C
:1070600008010C6FE50E095D3D0E0A59010E0B5922
:10707000000E08010C59D8A040EFB8F042EFB8F06C
:107080004EEFB8F065EC3FF00801096F030E060102
:107090000601E56F0801095188EFB9F0A1C713F89F
:1070A00094EC2DF0080114511311D8A45AEFB8F044
:1070B0005CEFB8F05EEFB8F088EFB9F0A1C713F855
:1070C00094EC2DF0080114511311D8A46AEFB8F014
:1070D0006CEFB8F06EEFB8F00EEFB8F00801080EE4
:1070E000080108010E6F0801080E08010F6FA1C703
:1070F0000DF84BEC28F00009D8A481EFB8F083EF2D
:10710000B8F085EFB8F00EEFB8F008C80DF8C1EC94
:10711000DBF0C4EC43F0A1C8C0F6A2C8C1F6A3C816
:10712000C2F6A4C8C3F661EC43F00009D8B49BEFE3
:10713000B8F09DEFB8F0A7EFB8F00801096F050EA1
:1071400006010601E56F080109510EEFB8F05EEF88
:10715000B8F0C4EC43F0A1C802F7A2C803F7A3C873
:1071600004F7A4C805F7C8EC15F065EC3FF008017A
:10717000096F030E06010601E56F0801095188EF4A
:10718000B9F0A1C72DF895EC12F0A1C70DF8EEECFF
:1071900041F00801096F080E06010601E56F0801BC
:1071A000095188EFB9F09BEC03F07F0E080108014C
:1071B0001617000E080117170A0E080108011625F8
:1071C00007010701246F000E0801080117210701BC
:1071D000256FC4EC43F0A1C8C0F6A2C8C1F6A3C88D
:1071E000C2F6A4C8C3F6D7EC41F00801096F000E3F
:1071F000080108010D6F0801095100EC44F0080175
:10720000096F090E06010601E56F0801095188EFB3
:10721000B9F0C4EC43F006010601C05108010801B1
:10722000A15D0801096F06010601C15108010801AD
:10723000A25908010A6F06010601C251080108019E
:10724000A35908010B6F06010601C351080108018B
:10725000A45908010C6FF20E08010801116F9E0E6F
:107260000801126F000E0801136F000E0801146F61
:107270000701080124C70DF80701080125C70EF80A
:107280000801000E08010EBFFF0E08010F6F080174
:10729000106FBBEC32F008010951080108010D5DC7
:1072A00008010A51080108010E5908010B51080193
:1072B00008010F5908010C51080108011059D8B0F4
:1072C00064EFB9F066EFB9F00EEFB8F0FF0088EFA9
:1072D000B9F006010601E551000A01E11ED5010AD7
:1072E00001E18CD5030A01E1E5D5010A01E102D6ED
:1072F000070A01E195D6010A01E12BD7030A01E152
:1073000040D70E0A01E14FD7010A83E088EFB9F0B8
:10731000120058C8E9FF59C8EAFF0801EECF61F82A
:107320000801EECF62F80801EECF63F80801EECF56
:1073300064F8040E080108015825E96E000E0801E2
:1073400008015921EA6E0801EECF65F80801EECF79
:1073500066F80801EECF67F80801EECF68F8080E6E
:10736000080108015825E96E000E0801080159219D
:10737000EA6E0801EECF69F80801EECF6AF808015D
:10738000EECF6BF80801EECF6CF80C0E0801080187
:107390005825E96E000E080108015921EA6E08011E
:1073A000EECF6DF80801EECF6EF80801EECF6FF862
:1073B0000801EECF70F8100E080108015825E96E9B
:1073C000000E080108015921EA6E0801EECF71F89C
:1073D0000801EECF72F80801EECF73F80801EECF86
:1073E00074F8180E080108015825080108015F6F9C
:1073F000000E0801080159210801606F140E0801F0
:1074000008015825E96E000E080108015921EA6EAD
:10741000EF500801756F3F0E08017517080175518F
:10742000080108015F250801766FE86A080175BF49
:10743000E8680801080160210801776F76C85DF8E7
:1074400077C85EF80801756F000E080108015C6FCF
:107450000801755143EFBAF05FC8E9FF60C8EAFF61
:107460000201730E080108015C25E16EE26A020167
:10747000020EE222EFCFE7FF080108015F4B602B0D
:10748000080108015C2B080108015E510801080190
:10749000601906E1080108015D51080108015F1942
:1074A000D8A455EFBAF057EFBAF02CEFBAF00201BA
:1074B000730E080108015C25E96EEA6A0201020EFA
:1074C000EA22800EEF6E080108015C2B380E0801DD
:1074D00008015C656EEFBAF070EFBAF0D5EFBAF064
:1074E0003F0E080108015C6578EFBAF07AEFBAF058
:1074F0007CEFBAF095EFBAF00201730E08010801B3
:107500005C25E96EEA6A0201020EEA22000EEF6EC5
:10751000080108015C2B3F0E080108015C6593EF30
:10752000BAF095EFBAF07CEFBAF00801710E0801DD
:107530000801836F0801080E0801846F08016D0EB1
:1075400008010801816F0801080E0801826F080117
:10755000690E080108017F6F0801080E0801806F9D
:107560000801650E080108017D6F0801080E080179
:107570007E6F0801610E080108017B6F0801080E8B
:1075800008017C6F0201730E08010801796F020186
:10759000020E08017A6F80EC9BF00801756F000EF7
:1075A000080108015C6F08017551370E08010801D8
:1075B0005C65DDEFBAF0DFEFBAF0E1EFBAF0FAEFB9
:1075C000BAF00201730E080108015C25E96EEA6A4F
:1075D0000201020EEA22000EEF6E080108015C2B88
:1075E000370E080108015C65F8EFBAF0FAEFBAF05F
:1075F000E1EFBAF0140E080108015825E96E000EFB
:10760000080108015921EA6EEF500801756F080161
:10761000D89075370801D89075370801D89075351E
:1076200002010201B26F140E080108015825E96E2B
:10763000000E080108015921EA6EEECF75F8EECF71
:1076400076F8EECF77F8EECF78F8060E2EEFBBF097
:10765000D89008017833773376337533E82E28EFE6
:10766000BBF00801755102010201B16F140E08014F
:1076700008015825E96E000E080108015921EA6E3B
:10768000EECF75F8EECF76F8EECF77F8EECF78F84C
:107690000E0E51EFBBF0D890080178337733763374
:1076A0007533E82E4BEFBBF0080175510201020162
:1076B000B06F140E080108015825E96E000E08018C
:1076C00008015921EA6EEECF75F8EECF76F8EECFCD
:1076D00077F8EECF78F8160E74EFBBF0D89008016B
:1076E0007833773376337533E82E6EEFBBF00801CD
:1076F000755102010201AF6F140E080108015825EF
:10770000E96E000E080108015921EA6EEECF75F806
:10771000EECF76F8EECF77F8EECF78F81E0E97EF33
:10772000BBF0D89008017833773376337533E82E81
:1077300091EFBBF00801755102010201AE6F080123
:10774000756F000E02010201AD6F0801755108014D
:10775000756F000E02010201AC6F0801755108013E
:10776000756F000E02010201AB6F0801755108012F
:10777000710E08010801836F0801080E0801846F6B
:1077800008016D0E08010801816F0801080E08014B
:10779000826F0801690E080108017F6F0801080E59
:1077A0000801806F0801650E080108017D6F08015E
:1077B000080E08017E6F0801610E080108017B6F49
:1077C0000801080E08017C6F0201730E0801080110
:1077D000796F0201020E08017A6F80EC9BF05AC8A3
:1077E000E9FF5BC8EAFF080164C8EFFF0801080170
:1077F0005A4B5B2B5AC8E9FF5BC8EAFF080163C814
:10780000EFFF080108015A4B5B2B5AC8E9FF5BC820
:10781000EAFF080162C8EFFF080108015A4B5B2B21
:107820005AC8E9FF5BC8EAFF080161C8EFFF080119
:1078300008015A4B5B2B5AC8E9FF5BC8EAFF0801F5
:1078400068C8EFFF080108015A4B5B2B5AC8E9FFD3
:107850005BC8EAFF080167C8EFFF080108015A4B3F
:107860005B2B5AC8E9FF5BC8EAFF080166C8EFFF57
:10787000080108015A4B5B2B5AC8E9FF5BC8EAFFB5
:10788000080165C8EFFF080108015A4B5B2B5AC875
:10789000E9FF5BC8EAFF08016CC8EFFF08010801B7
:1078A0005A4B5B2B5AC8E9FF5BC8EAFF08016BC85B
:1078B000EFFF080108015A4B5B2B5AC8E9FF5BC870
:1078C000EAFF08016AC8EFFF080108015A4B5B2B69
:1078D0005AC8E9FF5BC8EAFF080169C8EFFF080161
:1078E00008015A4B5B2B5AC8E9FF5BC8EAFF080145
:1078F00070C8EFFF080108015A4B5B2B5AC8E9FF1B
:107900005BC8EAFF08016FC8EFFF080108015A4B86
:107910005B2B5AC8E9FF5BC8EAFF08016EC8EFFF9E
:10792000080108015A4B5B2B5AC8E9FF5BC8EAFF04
:1079300008016DC8EFFF080108015A4B5B2B5AC8BC
:10794000E9FF5BC8EAFF080174C8EFFF08010801FE
:107950005A4B5B2B5AC8E9FF5BC8EAFF080173C8A2
:10796000EFFF080108015A4B5B2B5AC8E9FF5BC8BF
:10797000EAFF080172C8EFFF080108015A4B5B2BB0
:107980005AC8E9FF5BC8EAFF080171C8EFFF0801A8
:1079900008015A4B5B2B1200000E08010801296FE9
:1079A000000E08012A6F000E08012B6F000E08015F
:1079B0002C6F00014E514B114C114D11D8B4E3EF17
:1079C000BCF0E5EFBCF01FEFBDF0C4EC43F00001EC
:1079D00000014B5108010801A15D080108012E6F4B
:1079E000000100014C5108010801A25908012F6F44
:1079F000000100014D5108010801A3590801306F31
:107A0000000100014E5108010801A4590801316F1D
:107A1000F20E08010801326F9E0E0801336F000E4E
:107A20000801346F000E0801356F90EC1FF02EC86E
:107A300029F82FC82AF830C82BF831C82CF80801CB
:107A40002D6F010E08010801536F08012D5167ECDD
:107A50003DF008012D6F010E08010801536F080168
:107A60002D5167EC3DF008012D6F060E080108014D
:107A7000536F08012D5167EC3DF008012D6F000E8A
:107A800008010801536F08012D5167EC3DF0080112
:107A90002D6F120E08010801536F08012D5167EC7C
:107AA0003DF008012D6F230E08010801536F0801F6
:107AB0002D5167EC3DF008012D6F340E08010801CF
:107AC000536F08012D5167EC3DF008012D6F560EE4
:107AD00008010801536F08012D5167EC3DF02AC8D9
:107AE00053F867EC3DF029C853F867EC3DF0080106
:107AF0002D6F800E08010801536F08012D51000100
:107B0000000146A986EFBDF088EFBDF090EFBDF013
:107B100008012D6F000E08010801536F08012D5157
:107B200067EC3DF008012D6F000E08010801536F4E
:107B300008012D5167EC3DF0080108012251030AAC
:107B4000D8A4A5EFBDF0A7EFBDF0C5EFBDF00801CB
:107B500008012351D8B4AFEFBDF0B1EFBDF0C5EFD0
:107B6000BDF0040E08010801556F000E0801566FA4
:107B70000001570E08010801536F0001000E0801B3
:107B8000546FF9EC30F0EDEFBDF008012D6F000EF1
:107B900008010801536F08012D5167EC3DF0080101
:107BA0002D6F000E08010801536F08012D5167EC7D
:107BB0003DF008012D6F000E08010801536F080108
:107BC0002D5167EC3DF008012D6F000E08010801F2
:107BD000536F08012D5167EC3DF008012D6F000E29
:107BE00008010801246F08012D510B0E080108013E
:107BF0002465FDEFBDF0FFEFBDF001EFBEF018EF23
:107C0000BEF008012D6F000E08010801536F080136
:107C10002D5167EC3DF008010801242B0B0E0801E3
:107C20000801246516EFBEF018EFBEF001EFBEF0BC
:107C3000060E08010801556F000E0801566F00017D
:107C4000990E08010801536F0001000E0801546FDE
:107C5000F9EC30F008012D6F000E08010801246FC7
:107C600008012D51C90E0801080124653AEFBEF044
:107C70003CEFBEF03EEFBEF055EFBEF008012D6FB9
:107C8000000E08010801536F08012D5167EC3DF00B
:107C900008010801242BC90E08010801246553EFCF
:107CA000BEF055EFBEF03EEFBEF008012D6F630E43
:107CB00008010801536F08012D5167EC3DF00801E0
:107CC0002D6F820E08010801536F08012D5167ECDA
:107CD0003DF008012D6F530E08010801536F080194
:107CE0002D5167EC3DF008012D6F630E080108016E
:107CF000536F08012D5167EC3DF008012D6F350ED3
:107D000008010801536F08012D5167EC3DF008018F
:107D10002D6F010E08010801536F08012D5167EC0A
:107D20003DF022C853F867EC3DF008010801220538
:107D3000D8A49DEFBEF09FEFBEF0A1EFBEF0000112
:107D40004695080108012251030AD8A4AAEFBEF003
:107D5000ACEFBEF0D9EFBEF0080108012367B3EF26
:107D6000BEF0B5EFBEF0D9EFBEF008012D6F360EB4
:107D700008010801536F08012D5167EC3DF008011F
:107D80002D6F040E08010801536F08012D5167EC97
:107D90003DF056C053F867EC3DF055C053F867EC22
:107DA0003DF054C053F867EC3DF053C053F867EC16
:107DB0003DF008012D6F370E08010801536F0801CF
:107DC0002D5167EC3DF008012D6F040E08010801EC
:107DD000536F08012D5167EC3DF008012D6F010E26
:107DE00008010801536F08012D5167EC3DF00801AF
:107DF0002D6F030E08010801536F08012D5167EC28
:107E00003DF008012D6F060E08010801536F0801AF
:107E10002D5167EC3DF008012D6F0C0E0801080193
:107E2000536F08012D5167EC3DF008010801225104
:107E3000030AD8A41EEFBFF020EFBFF02AEFBFF077
:107E4000080108012351D8B428EFBFF02AEFBFF092
:107E500040EFBFF0080108012205D8A432EFBFF0BF
:107E600034EFBFF066EFBFF000015A5157115811BF
:107E70005911D8B43EEFBFF040EFBFF066EFBFF04E
:107E800008012D6F320E08010801536F08012D51B2
:107E900067EC3DF008012D6F040E08010801536FD7
:107EA00008012D5167EC3DF0040E08010801556FE3
:107EB000000E0801566F0001570E08010801536FAC
:107EC0000001000E0801546FF9EC30F008012D6F2D
:107ED000FF0E08010801536F08012D5167EC3DF0BA
:107EE0007CEFBFF008012D6F000E08010801536FF1
:107EF00008012D5167EC3DF02C0E06010601BC5D1A
:107F0000010E0601BD59D8A088EFBFF08AEFBFF07F
:107F100072EFBFF06CC025F86DC026F86EC027F870
:107F20006FC028F808010801236799EFBFF09BEFA5
:107F3000BFF0A8EFBFF0000E000100016C6F000E53
:107F400000016D6F000E00016E6F000E00016F6F7B
:107F500053EC21F025C86CF026C86DF027C86EF0F0
:107F600028C86FF012000801226F000E08010801F6
:107F70001D6F08012251040E080108011D65C3EFA1
:107F8000BFF0C5EFBFF0C7EFBFF071EFC2F008015F
:107F900008011D51170DF3CF22F80E0E08012227FC
:107FA0000201000E08012225E96EEA6A0201020EB2
:107FB000EA22EF50050AD8B4E0EFBFF0E2EFBFF0DD
:107FC000FCEFBFF0080108011D51170DF3CF22F897
:107FD0000E0E080122270201000E08012225E96E7B
:107FE000EA6A0201020EEA22040EEF62FAEFBFF023
:107FF000FCEFBFF0FEEFBFF064EFC2F03EEFC2F067
:108000001DEC43F00009D8B408EFC0F00AEFC0F04F
:1080100075EFC0F0080108011D51170DF3CF22F8CC
:108020000E0E080122270201000E08012225E96E2A
:10803000EA6A0201020EEA22000EEF6E0801080150
:108040001D51170DF3CF22F8140E0801222702014B
:10805000000E08012225E96EEA6A0201020EEA22F8
:10806000EF500801236F080123A139EFC0F03BEF67
:10807000C0F059EFC0F00801226F010E080108019D
:108080002F6F08012251080108011D51170D02012F
:10809000000EF324E96EEA6A0201020EEA220801E8
:1080A000EECF2DF80801EDCF2EF848EC3BF075EF40
:1080B000C0F00801226F010E080108012F6F0801AE
:1080C0002251080108011D51170D0201000EF32471
:1080D000E96EEA6A0201020EEA220801EECF2DF8EB
:1080E0000801EDCF2EF80DEC3BF064EFC2F0080173
:1080F0001E0E080108012D6F0801080E08012E6FE1
:10810000D3EC94F00009D8B488EFC0F08AEFC0F047
:1081100075EFC0F0DCEC40F00009D8B492EFC0F08D
:1081200094EFC0F0F2EFC0F0080108011D51170DE7
:108130000201000EF324E96EEA6A0201020EEA224D
:1081400008011EC8EEFF08011FC8EEFF080120C885
:10815000EEFF080121C8EEFF080108011D51170DAF
:10816000F3CF22F80E0E080122270201000E0801AB
:108170002225E96EEA6A0201020EEA22020EEF6E81
:10818000080108011D51170DF3CF22F8130E080145
:1081900022270201000E08012225E96EEA6A020187
:1081A000020EEA22000EEF6E080108011D51170DA4
:1081B000F3CF22F80F0E080122270201000E08015A
:1081C0002225E96EEA6A0201020EEA22270EEE6E0D
:1081D000000EEE6E000EEE6E000EED6EED52ED52E4
:1081E00006EFC1F0080108011D51170DF3CF22F869
:1081F0000E0E080122270201000E08012225E96E59
:10820000EA6A0201020EEA22010EEF6E64EFC2F08A
:108210005AEC42F0080108011D51170DF3CF22F866
:10822000150E080122270201000E08012225E96E21
:10823000EA6A0201020EEA220801A1C8EEFF080163
:10824000A2C8EDFF080108011D51170D0201000E23
:10825000F324080108014C6F08014D6B0201020E66
:1082600008014D230EEC23F0080108011D51170DE4
:10827000F3CF22F80E0E080122270201000E08019A
:108280002225E96EEA6A0201020EEA22030EEF6E6F
:1082900064EFC2F0080108011D51170DF3CF22F859
:1082A000040E080122270201000E08012225080100
:1082B00008014E6F08014F6B0201020E08014F23A7
:1082C000080108011D51170D0201000EF3240801D9
:1082D00008014C6F08014D6B0201020E08014D238D
:1082E000E7EC1AF00009D8A478EFC1F07AEFC1F0FA
:1082F00026EFC2F0080108011D51170DF3CF22F837
:10830000150E080122270201000E08012225E96E40
:10831000EA6A0201020EEA22EECF23F8EDCF24F83A
:108320005AEC42F00801235108010801A15D08013F
:10833000256F0801245108010801A2590801266F80
:10834000080108011D51170DF3CF27F80F0E080182
:1083500027270201000E08012725E96EEA6A0201BB
:10836000020EEA22EECF28F8EDCF29F808012551B8
:108370000801285D0801265108012959D8B0C3EF2A
:10838000C1F0C5EFC1F024EFC2F0080108011D5192
:10839000170DF3CF22F8130E080122270201000E59
:1083A00008012225E96EEA6A0201020EEA22EF5074
:1083B0000801236F060E0801235DD8B0E2EFC1F07B
:1083C000E4EFC1F010EFC2F0080108011D51170DD4
:1083D000F3CF22F8130E080122270201000E080134
:1083E0002225E96EEA6A0201020EEA22EF2A08015A
:1083F00008011D51170DF3CF22F80F0E0801222797
:108400000201000E08012225E96EEA6A0201020E4D
:10841000EA22D890EE36EE36EE36ED36ED52ED52DB
:10842000080108011D51170DF3CF22F80E0E0801A7
:1084300022270201000E08012225E96EEA6A0201E4
:10844000020EEA22020EEF6E75EFC0F0080108017D
:108450001D51170DF3CF22F80E0E0801222702013D
:10846000000E08012225E96EEA6A0201020EEA22E4
:10847000050EEF6E64EFC2F064EFC2F00801080170
:108480001D51170DF3CF22F80E0E0801222702010D
:10849000000E08012225E96EEA6A0201020EEA22B4
:1084A000EF50000A01E123D6010A01E1A9D5030A30
:1084B00001E1AED6010A01E1EDD6070A01E115D6C8
:1084C000010ADAE03CEFC2F0080108011D2B040E9E
:1084D000080108011D656FEFC2F071EFC2F0C7EF30
:1084E000BFF01200080108010D51D8B47AEFC2F0B4
:1084F0007CEFC2F081EFC2F0080108010E2B84EF7F
:10850000C2F0080108010E07DDEFC4F0050E0801F6
:1085100008010E658EEFC2F090EFC2F09FEFC2F03F
:108520000C0E080108010E6198EFC2F09AEFC2F03C
:108530009FEFC2F007010701102BEEEFC4F00D0E04
:10854000080108010E65A7EFC2F0A9EFC2F0CFEF56
:10855000C2F0160E080108010E61B1EFC2F0B3EFD0
:10856000C2F0CFEFC2F0140E070107011065BBEF98
:10857000C2F0BDEFC2F0CFEFC2F008010F6F010EE5
:10858000070107012A6F08010F5108010F6F030E41
:1085900007010701106F08010F51EEEFC4F0E0EC86
:1085A0003FF0EEEFC4F00D0E080108010E65DBEFA1
:1085B000C2F0DDEFC2F0CFEFC2F0160E08010801E5
:1085C0000E61E5EFC2F0E7EFC2F0CFEFC2F00701B6
:1085D00007011007070107011067F1EFC2F0F3EF81
:1085E000C2F002EFC3F0000E06010601E16F000EBB
:1085F0000601E26F08010F6F020E070107012A6FE3
:1086000008010F51EEEFC4F00EC812F80DC811F8B2
:108610004CEC1EF011C8BAF612C8BBF606010601F2
:10862000BB29FE0ED8B4BA19D8A419EFC3F01BEFBA
:10863000C3F01FEFC3F0E0EC3FF0EEEFC4F0060133
:108640000601BA29D8B4BB29D8A429EFC3F02BEF6F
:10865000C3F02DEFC3F0EEEFC4F006010601E251C6
:10866000E111D8A436EFC3F038EFC3F042EFC3F006
:1086700006010601BA5106010601E26F0601E16B2F
:10868000E8EFC3F006010601BA5106010601E11345
:1086900006010601BB5106010601E2137DEFC3F09E
:1086A00008010F6F070E070107019A6F08010F51AC
:1086B000D8EFC3F008010F6F050E070107019A6F8D
:1086C00008010F51D8EFC3F008010F6F080E070122
:1086D00007019A6F08010F51D8EFC3F008010F6F1F
:1086E000090E070107019A6F08010F51D8EFC3F077
:1086F000070107019A69D8EFC3F00601E1C60FF838
:108700000601E2C610F80801C2EFC3F008010F51DC
:10871000840ADAE0100AD8E078EFC3F008010F51BC
:10872000200ABEE078EFC3F008010F51140ACCE034
:1087300078EFC3F008010F51100AB2E078EFC3F0F0
:1087400008010F51600ACAE078EFC3F008010F5129
:10875000440AB0E078EFC3F008010F51740AAAE0B0
:1087600078EFC3F008010F51400AA4E0300AA2E0FC
:1087700078EFC3F008010F51240A92E0900A90E0CC
:1087800078EFC3F008011051190AC0E0040AC6E0EE
:10879000340ACAE0040ACEE0700AD2E0950AD6E0B4
:1087A000100ADAE0340ADEE0140AE4E078EFC3F0FD
:1087B00008010F6F030E070107012A6F08010F510F
:1087C00008010F6F000E070107011C6F08010F5110
:1087D000EEEFC4F00EC812F80DC811F84CEC1EF004
:1087E00011C8BAF612C8BBF606010601BB29FE0E77
:1087F000D8B4BA19D8A4FFEFC3F001EFC4F047EF23
:10880000C4F0070107019AAF08EFC4F00AEFC4F003
:10881000CFEFC2F0080108010D6711EFC4F013EFAC
:10882000C4F0CFEFC2F0D89006010601C5310801AF
:10883000106F06010601C43108010F6F380E0801E0
:108840000F5D000E1059D8A028EFC4F02AEFC4F035
:10885000CFEFC2F01E0E080108010E6532EFC4F022
:1088600034EFC4F0CFEFC2F008010F6F000E070124
:1088700007019A6F08010F51000E06010601BA6F39
:10888000000E0601BB6F45EFC4F058EFC4F00601BF
:108890000601BA29D8B4BB29D8A451EFC4F053EFCC
:1088A000C4F055EFC4F0EEEFC4F0070107019A07DA
:1088B0000601A90E070107011C25E96EEA6A0601F7
:1088C000060EEA220601BAC6EFFF070107011C2BBC
:1088D000070107019A676FEFC4F071EFC4F0CBEFA7
:1088E000C4F0E0EC3FF00BEC43F0850E080108010A
:1088F0002E6FFF0E08012F6F930E080108012C6FD9
:10890000FF0E08012D6FF5EC43F0700E0801080111
:108910002E6FFF0E08012F6F2D0E080108012C6F1E
:10892000FF0E08012D6FF5EC43F006010801E1C6CA
:108930002EF806010801E2C62FF808010801306B85
:108940000801316BAB0E080108012C6FFF0E080106
:108950002D6F71EC43F01CC726F80601A90E080123
:108960000801246F0601060E0801256FB10E0801EB
:108970000801226FFF0E0801236FB7EC43F00801D6
:108980000F6F010E080108012C6F08010F515CECFC
:1089900041F0EEEFC4F0910E06010601C45D010E38
:1089A0000601C559D8A0D7EFC4F0D9EFC4F002EF43
:1089B000C3F0E0EC3FF0EEEFC4F0070107012A51ED
:1089C000000A01E1A3D5010A01E1EDD5030A01E1A5
:1089D0001BD6010A01E1FED6EEEFC4F01200080139
:1089E000096F000E080108011D6F0801095153ECC1
:1089F00044F00009D8A4FFEFC4F001EFC5F027EF61
:108A0000C5F0070107011D51D8B409EFC5F00BEF00
:108A1000C5F025EFC5F09EC72DF895EC12F09EC766
:108A20000DF8EEEC41F00801096FFE0E0701070199
:108A30009E6F08010951BDEC3BF00801096F000E63
:108A4000070107011D6F0801095119EFC7F006EF73
:108A5000C7F00801096F010E070107011D6F08012A
:108A600009510801096F000E08010801146F08017F
:108A70000951500E08010801126F000E0801136F12
:108A800008010A6F010E08010801116F08010A515F
:108A90006A0E08010B6F070E0C6F08010BC80DF86A
:108AA00008010CC80EF8080108010F6B0801106BD3
:108AB0003FECDAF0070107019E6F070107019E51A5
:108AC000FE0AD8A466EFC5F068EFC5F072EFC5F0F6
:108AD0000801096F000E070107011D6F0801095108
:108AE00019EFC7F0C4EC43F0A1C8F5F6A2C8F6F63A
:108AF000A3C8F7F6A4C8F8F619EFC7F09EC70DF89B
:108B00003DEC41F00009D8A488EFC5F08AEFC5F02C
:108B1000C6EFC5F0C4EC43F006010601F5510801AB
:108B20000801A15D0801096F06010601F65108015F
:108B30000801A25908010A6F06010601F751080150
:108B40000801A35908010B6F06010601F85108013D
:108B50000801A45908010C6F5D0E095DA00E0A59A9
:108B6000120E0B59000E08010C59D8A0BAEFC5F02F
:108B7000BCEFC5F0C4EFC5F00801096F040E070192
:108B800007011D6F0801095119EFC7F00801096FAE
:108B9000020E070107011D6F0801095119EFC7F007
:108BA0009EC768F8BEEC20F07D0E08010801685DE4
:108BB000000E08016959D8B0E0EFC5F0E2EFC5F04A
:108BC000E4EFC5F019EFC7F0D90E08010801576F9F
:108BD000FF0E0801586F9EC756F830EC42F0160E93
:108BE00008010801576FFE0E0801586F9EC756F81E
:108BF00030EC42F00801096F000E06010601E76F34
:108C000008010951050E06010601E7650AEFC6F0E5
:108C10000CEFC6F00EEFC6F049EFC6F00001DB0E18
:108C200006010601E725E96EEA6A0001000EEA2264
:108C3000EF5008010801586F0DEC3FF008010801E2
:108C4000576F9EC756F801EC15F00001DB0E0601C8
:108C50000601E725E96EEA6A0001000EEA22EF50FC
:108C600008010801646FE1EC3EF008010801576F4C
:108C70009EC756F801EC15F006010601E72B050E1C
:108C800006010601E76547EFC6F049EFC6F00EEFB3
:108C9000C6F0A90E08010801576FFE0E0801586FB3
:108CA0009EC756F830EC42F007016A0E0801080131
:108CB000576F0701070E0801586F9EC756F845EC1D
:108CC00042F0910E08010801576FFE0E0801586F1F
:108CD0009EC756F830EC42F09EC768F8F6EC3BF0C1
:108CE0000801096F000E06010601E76F080109512E
:108CF0000801096F030E070107011D6F08010951E3
:108D000019EFC7F00801080E080108010E6F0801ED
:108D1000080E08010F6F9EC70DF84BEC28F00009F4
:108D2000D8A495EFC6F097EFC6F099EFC6F0CEEF56
:108D3000C6F0030E06010601E765A1EFC6F0A3EF3A
:108D4000C6F0A9EFC6F008C80DF86CEC0DF0CCEF3A
:108D5000C6F00801080108510A0AD8B4B2EFC6F0FB
:108D6000B4EFC6F0BFEFC6F00801080108510D0AC4
:108D7000D8A4BDEFC6F0BFEFC6F0C4EFC6F0060141
:108D80000601E72BCCEFC6F00801096F000E0601C3
:108D90000601E76F0801095182EFC6F09EC70DF882
:108DA0003DEC41F00009D8A4D8EFC6F0DAEFC6F0E8
:108DB000E2EFC6F00801096F040E070107011D6FFD
:108DC0000801095119EFC7F09EC72DF895EC12F074
:108DD0009EC70DF8EEEC41F00801096FFE0E070189
:108DE00007019E6F080109510801096F010E070173
:108DF00007012E6F080109510801096F050E0701CF
:108E000007011D6F0801095119EFC7F0070107019C
:108E10001D51000A01E11DD6010A01E16FD6030AC6
:108E200001E1BED6010A01E16DD7070ACDE019EFD5
:108E3000C7F0120008010C6F000E08010801086F4E
:108E400008010C5133EFC8F09BC735F8BEC633F8A4
:108E5000BFC634F887EC3EF0D8A031EFC7F033EF4F
:108E6000C7F086EFC7F0960E06010601D4653BEF0A
:108E7000C7F03DEFC7F043EFC7F0BEC696F7BFC6D9
:108E800097F79BC79CF706010601D451D8B44BEF66
:108E9000C7F04DEFC7F071EFC7F0D4C60EF8080168
:108EA0000C6F000E080108010D6F08010C5155EC04
:108EB000D0F0D4C60EF808010C6F000E08010801AE
:108EC0000D6F08010C5172ECC2F0D4C60EF8080107
:108ED0000C6F000E080108010D6F08010C51B7EC72
:108EE000AEF006010601FB2B08010C6F000E060117
:108EF0000601D46F08010C5108010C6F000E070128
:108F00000701376F08010C51CEEFC7F006010601CB
:108F1000D4678DEFC7F08FEFC7F095EFC7F0BEC6EF
:108F200094F7BFC695F79BC7DAF606010601FB5119
:108F3000D8B49DEFC7F09FEFC7F0C3EFC7F0FBC6F3
:108F40000EF808010C6F010E080108010D6F0801F1
:108F50000C5155ECD0F0FBC60EF808010C6F010E59
:108F6000080108010D6F08010C5172ECC2F0FBC63C
:108F70000EF808010C6F010E080108010D6F0801C1
:108F80000C51B7ECAEF006010601D42B08010C6FB2
:108F9000000E06010601FB6F08010C510701D89075
:108FA0009B33070107019B67D8EFC7F0DAEFC7F0E3
:108FB000F9EFC7F008010C6F800E070107019B6FE6
:108FC00008010C5106010601BE4BBF2B060106012C
:108FD000BF51020ABE11D8A4F0EFC7F0F2EFC7F0FC
:108FE000F9EFC7F0000E06010601BE6F000E060184
:108FF000BF6F06010601BF5107010701971906E17E
:1090000006010601BE51070107019619D8A40BEF0E
:10901000C8F00DEFC8F01EEFC8F0070107019B5123
:10902000070107019C6317EFC8F019EFC8F01EEFA6
:10903000C8F0070107019669070197690601060153
:10904000D451960AD8A427EFC8F029EFC8F033EF1F
:10905000C8F008010C6F010E08010801086F080133
:109060000C5147EFC8F006010601D951060106016F
:10907000BF1906E106010601D85106010601BE1915
:10908000D8A445EFC8F047EFC8F024EFC7F00801B7
:10909000080108674EEFC8F050EFC8F052EFC8F073
:1090A00010EFC9F0070107013751D8B45AEFC8F0E3
:1090B0005CEFC8F05EEFC8F010EFC9F094C70FF88E
:1090C00095C710F896C70DF897C70EF8E1EC2FF08A
:1090D0000DC80AF80EC80BF8080108010BBF73EFA2
:1090E000C8F075EFC8F086EFC8F0080108010B5111
:1090F000800A800F320ED8B40A5DD8B082EFC8F073
:1091000084EFC8F086EFC8F010EFC9F0080108013D
:109110000B51800A800F9E0ED8B40A5DD8A093EF41
